:020000040800F2
:1000000000500020A58400085185000805700008F4
:100010005185000851850008518500080000000046
:1000200000000000000000000000000051850008F2
:10003000518500080000000051850008F56F000898
:100040005185000851850008518500085185000838
:100050005185000851850008518500085185000828
:100060005185000851850008518500085185000818
:100070005185000851850008616F0008518500080E
:1000800051850008518500085185000851850008F8
:1000900051850008518500085185000851850008E8
:1000A000518500085185000851850008AD6E000893
:1000B000A56E0008996E00088D6E0008A56F0008F7
:1000C0009D6F0008A16F0008996F00085185000816
:1000D00051850008256F0008B96E00085185000899
:1000E0005185000851850008518500080000000076
:1000F0000000000000000000000000000000000000
:0C01000000000000000000005FF808F1A3
:100110002DE9F04F664B674C99B023600023636074
:1001200003F042F8A24618B906F078FB03F05EF837
:1001300004F01AFD002308935F4C09930A934FF4CF
:10014000E0130B9323685D4943F480338A7B23607B
:10015000A36943F01003A361236803F400330993F8
:10016000089B01330893099B1BB9089BB3F5A06F4B
:10017000F2D12168504B11F4003101D0022315E077
:10018000186840F0010018600891236803F002032A
:100190000993089B01330893099B1BB9089BB3F58E
:1001A000A06FF2D12368990738D501230A93444BF5
:1001B000444E196841F010011960196821F00301DB
:1001C0001960196841F0020119606368636063682F
:1001D0006360636843F4806363603B4B196821F09C
:1001E000704119603949B161616821F47C11616025
:1001F000196841F000411960996821F40041996043
:1002000059680B0449BF324B4FF4E013B3614FF40C
:1002100080130B930A9B012B01D117E0FEE7022B01
:1002200018D16AB10B9BB3F5801F02D14FF4A01314
:1002300005E00B9BB3F5E01F02D14FF400130B93C5
:1002400062680B9B134343F4803302E0636843F41A
:1002500060136360236843F0807323602268164B49
:100260009701FBD55A6822F003025A605A6842F09F
:1002700002025A606368104A03F00C03082B0693CD
:10028000F8D15168134B01F00C01042903D008295F
:1002900004D00E4A00E0B2691A6027E05168506845
:1002A000C1F38341C50301F1020117D40A4A1BE0DF
:1002B000CD21000800050020001002400C0F002096
:1002C00000200240100000200410014000127A00BB
:1002D000001BB7007800002000093D00526812F4AE
:1002E000003FB26918BF5208514319606368DFF8D4
:1002F0001C83C3F30313334493F81C90B44B18AD21
:100300001A68002722FA09F9C3F80090B14BB248E5
:10031000C8F80C30A36943F00103A361636A43F09A
:1003200080736362A36943F01C03A3614FF6FF73FC
:1003300025F82C3D29468DF8367002F071FAA74851
:10034000294602F06DFAA648294602F069FAA54B43
:100350005A6842F000725A60A34B0FCB85E80F0039
:10036000A3699F4843F01003A361A3690EA943F05A
:100370001003A3614FF4005303614FF48043036102
:100380000D9802F04DFA10A90F9802F049FA28468C
:1003900004F028F90D9B954A3846B3FBF2F34FF46D
:1003A0007A72CAF80830B9FBF2F9914B09F1FF32C1
:1003B0005A604FF00709F02288F823209F60C3F8A5
:1003C000009004F021FA642001F0F1FD8949DFF882
:1003D0004082D1F808B040460BF400630493102328
:1003E0001A46394603930AF098F8039B0222ADF8A7
:1003F0003030042388F800301BF4004F4FF0010325
:100400008DF833708DF8322088F8023088F8039028
:10041000474609D01221ADF830103B717B71BB719A
:1004200087F80790904600E098466B480CA904F0C6
:1004300089F9049B93B1022368480CA9ADF83030C8
:1004400004F080F9092301223B73BA7308F1010318
:10045000072287F80D80FA735FFA83F863696648AC
:1004600043F001036361A369DFF88C9143F40073E7
:10047000A36101F0E2FA614B00240D93604BB8F1E7
:10048000010F0E930CBF2346802312934FF4807309
:1004900013934FF480631493202329461593484601
:1004A0004FF4005316930F94CDF840801194179495
:1004B00001F0A5FAD9F80030B8F1010F43F00103BB
:1004C000C9F800304F4B98BF00215A6888BF0121FE
:1004D00022F4702222F4807242EA01225A60996862
:1004E000494A0A4042F4602242F002029A60D96A04
:1004F00008F1FF3221F47001D2B241EA0252DA620D
:100500002146012378188278002A5AD07A5C5C1C34
:10051000092A90F803E0E4B23A4811D9A2F10A0599
:1005200005EB45054FF0070808FA05F80EFA05F542
:10053000D0F80CC02CEA080C4CEA0505C5600EE0AA
:1005400002EB42054FF0070808FA05F80EFA05F528
:10055000D0F810C02CEA080C4CEA05050561062B02
:1005600028480ED8013B03EB83034FF01F0E0EFA11
:1005700003FE9A40456B25EA0E0545EA02034363F4
:1005800020E00C2B0ED8073B03EB83034FF01F0E2C
:100590000EFA03FE9A40056B25EA0E0545EA0203B2
:1005A00003630FE00D3B03EB83034FF01F0E0EFAC6
:1005B00003FE9A40C56A25EA0E0545EA0203C362B6
:1005C00000E01C460431102924D023469AE700BFDE
:1005D000780000200005FA0500080140000C0140E9
:1005E000001001400000014088C1000840420F0097
:1005F00010E000E00C0F0020080002404C240140F5
:10060000D003002000240140FDF7F1FF00ED00E0E1
:10061000C0030020B24B9A6842F480729A609A68D4
:1006200042F001029A609A6842F008029A60996862
:10063000AB4A0807FBD4936843F004039360A84ACD
:10064000936813F00403FAD1916841F4A00191601A
:10065000A44AB2F8E60050B9B2F9E83033B9B2F9B9
:10066000EA30D3F1010338BF002300E0034613F062
:10067000010340F0968086F82C3000B206F02AFE86
:1006800095A3D3E9002306F08BFE07F0BBF8954E47
:100690000546B6F9E80006F01DFE8FA3D3E9002356
:1006A00006F07EFE07F0AEF80446B6F9EA0006F062
:1006B00011FE89A3D3E9002306F072FE07F0A2F829
:1006C000804628460AF058F9064628460AF0C8F936
:1006D000074620460AF050F9054620460AF0C0F9C0
:1006E000044640460AF048F9814640460AF0B8F907
:1006F00031468046484607F0E3F931468346404696
:1007000007F0DEF949460490384607F0D9F941462A
:100710000590384607F0D4F929460790484607F077
:10072000CFF94146CAF80C0005F1004007F0C8F9BE
:100730002146CAF81000CAF81440059807F0C0F91D
:100740000146049807F0B4F82146CAF81800079843
:1007500007F0B6F90146584607F0A8F82946CAF846
:100760001C0007F1004007F0ABF92146CAF8200051
:10077000584607F0A5F90146079807F097F8214673
:10078000CAF82400049807F09BF90146059807F081
:100790008FF83146CAF82800284607F091F9CAF8C0
:1007A0002C00514EDFF8688133684E4C43F00A0349
:1007B0003360D8F800304D4DB3F85A304FF000098F
:1007C000B4F8EEB094F8ED70059385F8009005F05C
:1007D0000FF90490002800F00D81454B4549BBF10D
:1007E000140F19604449454D596045499846D960F0
:1007F00019D006D8BBF1050F19D0BBF10A0F14D0E0
:100800000FE0BBF1BC0F0AD0BBF5807F04D0BBF179
:10081000620F06D102230BE085F82D9015E001232D
:1008200006E0032304E0042302E0052300E006239E
:1008300085F82D3009E0082F0DD08FB1314B1B7892
:10084000002B7ED1002F78D01F462F4B0022022F85
:100850001A70F0D104E0336823F002033360EDE74F
:1008600005F0C6F80028E9D006210DAB68200A463D
:1008700004F0D0F89DF837309DF839B003F001034B
:100880005B000BF0010B43EA8B0B9DF8353003F056
:1008900001035BEA030B0CD0BBF1010F03D1002372
:1008A0008AF8303039E0BBF1020F0DD10122174B2D
:1008B00031E00CAB68200C21012204F0ABF89DF86C
:1008C000303013F00F0301D1052094E0042B0F4BBF
:1008D00020D183F830B020E0399D52A246DF913F0D
:1008E000002401400C0F0020F401002036020020FB
:1008F00020020020DD580008BF5100081000002031
:1009000090C1793DF51300209E02002000050020D3
:100910001C020020012283F83020B14BB14A1A603A
:10092000B14A5A609AF83020002A14BF6E226F2212
:100930001A72AE4B02221A7080E7336823F002036A
:10094000336094F8E2300BB1A948037094F8E330B7
:100950000BB1A84A137094F8E4300BB1A64A137097
:100960003368990702D59E4B1B689847D8F800302A
:10097000984718AF002307F82C3D1E200A210122BA
:100980003B4604F047F838B19DF83430482B03D18A
:10099000994B03221A7003E0336823F00803336095
:1009A0003368DFF8989213F0080F1FD005994FF0C5
:1009B000640A0AB292FBFAFB5846039207F02CF83D
:1009C000039A03460AFB1B2000B2039307F024F8A6
:1009D0008A4907F075F8039B0146184606F068FF40
:1009E000874907F06DF8C9F8340006E00023C9F81C
:1009F000343002E0032001F023FB824A4FF48043AD
:100A000053614FF4005313614FF00A0ADFF8F49179
:100A10001920D9F80C300AF1FF3A83F48043C9F861
:100A20000C30D9F80C3083F40053C9F80C3001F0C5
:100A3000BEFA192001F0BBFA1AF0FF0AE6D14FF412
:100A40000053C9F810304FF48043C9F810306E4B92
:100A5000DFF8ECB11B6893F90C0006F03BFC5CA3DB
:100A6000D3E9002306F09CFC06F0CCFE09F084FFDD
:100A70008246BBF8000006F0CFFF514607F020F891
:100A800009F0B0FF614BDFF8B4A11880BBF800009B
:100A900006F0C2FF01465E4807F0C6F85D4907F060
:100AA000C3F8CAF83800D8F80C0006F025FC48A3B3
:100AB000D3E9002306F074FC47A3D3E9002306F032
:100AC0006FFC06F09FFE544B62791860534B5449FB
:100AD0001A70544B01EBC202527CCAF83C30524BA4
:100AE0001A60A268920644BF01221A603368180790
:100AF00040F11B814FF48043C9F81430AA694B4977
:100B00008A4214D103F1804303F5E8339A694848D7
:100B100042F008029A614FF48053ADF8303002235E
:100B20008DF8333004238DF832300CA90BE04149A5
:100B30008A420AD1404A3348916941F010019161DB
:100B400018A921F8303D01F06BFE322001F02FFA98
:100B5000002111221E2004F079FE012160221E20B6
:100B600004F074FE642001F022FA4FF000083846C9
:100B700004F004FFC2460A23C346022101221E20BC
:100B8000039304F063FE322001F011FA384604F0BA
:100B9000F5FEBDF93410BDF93600BDF938208B449F
:100BA0008842B8BF014690449142B8BF0A4612F548
:100BB000805F8244039B45DDD9F80C20013B82F421
:100BC0008042C9F80C20D8D101273CE0AFF3008067
:100BD000399D52A246DF913F000000A0F7C6B03E0B
:100BE0008C0200206519000881510008F5130020CF
:100BF000360200209E020020F21300208988883CE3
:100C00000000204100100140D8020020FC0200201A
:100C10000AE81C4100401C46D4020020F4040020D5
:100C200088C100081C0F0020F004002000127A0088
:100C3000000C0140001BB70000100240000500201E
:100C40000000002000271E200021122204F0FEFDDB
:100C50000A23022101221E20039304F0F7FD322013
:100C600001F0A5F90DA804F089FEBDF93410BDF915
:100C70003600BDF93820C1EB0B0B8842B8BF0146E6
:100C8000C2EB08089142B8BF0A4612F5805FC0EB7C
:100C90000A0A039B08DDD9F80C20013B82F480424C
:100CA000C9F80C20D5D100E00027784B58460393B3
:100CB00006F0B2FE0146764806F0B6FF20F000408E
:100CC0002863504606F0A8FE0146714806F0ACFFC6
:100CD00020F000406863404606F09EFE01466D48E5
:100CE00006F0A2FF20F00040A863002170221E2021
:100CF00004F0ACFD012120221E2004F0A7FD0221FA
:100D000000221E2004F0A2FD642001F050F9039B94
:100D100027B94FF07E521A635A639A634FF48043A7
:100D2000C9F810305C4B01221A7000214FF4A072F8
:100D30005A4809F0F2FB5A4B5A4FDA6942F007025F
:100D4000DA619A6942F4006242F00C029A61564BF1
:100D50003B6003F087FA3A68544B05921846FF212E
:100D6000152209F0DAFB002202703268DFF840E158
:100D7000012112F0020F8EF80010734604D041706A
:100D80000321197002218170510704D519784E1C76
:100D90001E700326465412F00A0F0CD01A78042154
:100DA0008154511CC9B205264654D11C0232197017
:100DB000D2B206218154A1688A0604D51A78561C3D
:100DC0001E70072686546279082A01D00E2A04D1A3
:100DD0001A78561C1E700B2686541A784F0702F19B
:100DE0000106F6B21E704FF00C03835405D5304B4C
:100DF00002321A702D4B10229A552D4B12271A7859
:100E0000875494F84101561CF6B200280CBF00210B
:100E100001F001011E7021B102321A70234B13221E
:100E20009A5524480021982209F077FB4FF00008DA
:100E3000059B4FF000095A680026009601203146B4
:100E4000032305F0C1FF074638B9B9F1000F33D1CC
:100E50004FF496424FF00109EEE7B8F1010FE7D8E1
:100E60004C2202FB08FBDFF84C9008F1010C0BEB65
:100E70000908404631465FFA8CFA09F04EFB01231F
:100E80004BF8097088F84A30D046D1E710000020AE
:100E900000406F4601C05E4614020020400500205D
:100EA00000100240B004002034100020B7040020DD
:100EB000B604002010040020297ABB4B02291E68CA
:100EC000BA4B40F056835968B94DC5F8801139B90D
:100ED00000910220B268032305F076FFC5F8800177
:100EE0000DA80021122209F018FB63790E2B01D006
:100EF000082B02D101238DF83D30A66816F4005668
:100F000018D1AC4A0023B05CD75CD118874203D01B
:100F10001033602BF8D1002102F004F983681B78AC
:100F2000012B04D01036602EEBD1002004900499E0
:100F30008DF83710A368A049C3F340028DF838201C
:100F40000968C3F380128DF83920C3F340320031B1
:100F50008DF834209948C3F3C03218BF01218DF8B1
:100F60003620C3F300428DF83A208DF83B1003F091
:100F7000010201688DF8352091F82611B4F8E000DF
:100F8000C1F380018DF83C10ADF84000B4F8DE10DC
:100F90004FF47A70ADF84200D804ADF83E1004D595
:100FA000874BB3F8DA30ADF84230B1F5FA7F844EB2
:100FB00084BF0023ADF84230B6F818318149ADF84E
:100FC000443096F8203185F88431002385F8853146
:100FD0004B709DF83D30002B14BF0223002302B15B
:100FE0000133794A002702EB8303D3F82831BA464C
:100FF00004930499CB5B4FF6FF718B42DAB20AD1AE
:1010000095F8853185F88731704B1F78162F40F0A1
:101010003F8100242FE19DF8371019B1911E01295D
:1010200040F215819DF8391019B1111F032940F2C2
:101030000E81DFF8B8919DF83A104FEA021809EBDB
:10104000080429B159F808106148814200F0FF8076
:101050009DF8361011B1012A00F0F9801B0A022B0D
:1010600005D19DF83410002908BF002303E0012BAF
:1010700008BF9DF835309DF83B1039B19DF83D1003
:1010800021B9A2F10801012998BF04239DF83C1061
:1010900031B19DF83D1019B9043A032A40F2C080DD
:1010A000012B35D1FF2385F8CC3185F8CD31A368EC
:1010B0004FF0000BE27B6068ADF830300CA90223E2
:1010C00085F8D0B1C5F8DC418DF833308DF8322089
:1010D00085F888B1C5F88CB1C5F890B1C5F894B160
:1010E000C5F8C8B185F8CEB185F8CFB101F098FB4D
:1010F000217B5A4659F8080003F04FF9204605F0C5
:101100003DF820465946334A334B02F057FE9EE0E5
:10111000022B30D1DFF8D8E05FFA8AFB4FEA0B11DF
:101120000EEB010000224FF0010C8270827280F8F9
:1011300001B00EF801C0E17BC460A0688DF83210E8
:10114000ADF830000CA960688DF83330039201F0DF
:1011500067FB217B039A59F8080003F01EF920462B
:1011600005F00CF8204659461C4A1D4B02F026FE9D
:101170000AF1010A6BE0032B50D1BDF83E2095F82F
:101180008681B2F5FA7FBDF8423033D91549204641
:10119000B1FBF2F292B2082102F0A6FE05EB880341
:1011A000C3F85002104B32E0B004002010000020C1
:1011B0000005002050C20008F00400201C0200209E
:1011C0000C0F00208506002088C10008F4040020D0
:1011D000000400401918000821190008954500086E
:1011E000F518000800127A004119000858D30008C9
:1011F000D00600208D492046B1FBF2F292B20121C7
:1012000002F072FE05EB8803C3F85002884B83603E
:1012100095F88631013385F8863118E0042B16D114
:10122000BDF84030814A204692FBF3F20121BDF81F
:10123000443092B295F8858102F056FE05EB8803A2
:10124000C3F8800295F88531013385F8853102377E
:101250001C2F7FF4CEAED3E6764B04EB030E98E85A
:101260000F008EE80F00744B10341A78C02C02F176
:1012700001021A7008D0EB6B0021185903EB040827
:1012800006F0B2FD0028E7D0B368D9041ED419E0F7
:101290006A49694A01EBC70393F810C0D3F8148078
:1012A00082F800C0B8F1000FEED000246445EBDAFC
:1012B000604A230103EB020E43440FCB01348EE856
:1012C0000F00F3E7082F5E4C28D129E05A4B93F822
:1012D0000090B9F1010FF5D95A4C4FF00008C845FC
:1012E00004F11004EEDA54F8100C4FF07C5106F0C3
:1012F000E7FB4FF07C5144F8100C54F8140C06F046
:10130000DFFB4FF07C5144F8140C54F80C0C06F041
:10131000D7FB08F1010844F80C0CE0E70E2F03D1CD
:10132000237843F0100302E0237823F010032370A6
:1013300002F008F8444A45484549464B0260464891
:10134000C5F8643301600023B6F81801C5F86013CE
:10135000A5F86A3385F86C33C5F870233F495852B5
:101360000233242BFAD13E4B1A60B3681A0740F1BE
:10137000A7803C4B002293F81631042B00F29A8090
:10138000DFE803F003032A448400012B4FF003013C
:10139000354A08D185F87413072185F8763385F826
:1013A00075130C2308E0022385F87433002385F8B5
:1013B000763385F8751307231370002300930820F4
:1013C00001232A494FF4E13205F0FEFC284BC5F811
:1013D0007803C5F87C3369E0012300932549052390
:1013E0000820254A05F0F0FCB6F81811C5F880036E
:1013F000A1F5777149000023204A99500433302B1E
:10140000FAD11F4B0C22C5F87C334DE0009201232A
:101410004FF4E13208201B4905F0D6FC1A4BC5F801
:101420008403C5F87C3310223EE000BF40420F0029
:1014300031190008A0070020CC13002088C1000843
:1014400002020020A80700206408002004040020F5
:101450001A100020C0C20008F40000204A03002037
:10146000E80100200C0F0020CC040020311E0008F1
:10147000D11500083D1F0008A086010014010020BE
:1014800085160008C91E0008751600080092012381
:101490004FF4E1320820404905F096FC3F4BC5F877
:1014A0008803C5F87C3308223D4B1A70003018BF02
:1014B000012028B9082001F077F90023C5F87C3312
:1014C000B268374B12F4804F04D0082119703549A7
:1014D000C5F87C1342F20101114002F0010002F450
:1014E000005741B1304AC5F87C230FB108221A7069
:1014F00008B10C221A701A78043A5A7000F07EFC77
:101500002A4B18607379052B03D1294B4FF4C8720D
:101510001A80284B4FF47A721A80237843F008031C
:101520002370254B1A7822F002021A70B3689B07C9
:101530002ED5224B224A1C461A6000F0D3FB2820ED
:1015400000F035FD069901390691F6D121681D4B51
:1015500048781D7802460123954203D30133082BB6
:101560000244F9D1184A13708A785343174A1380FA
:101570000EE01A7D022A09D08D073FF5A4AC02F0D7
:10158000020202F0FF01002A3FF49EAC0C339AE401
:1015900019B0BDE8F08F00BF7D1E0008611600087D
:1015A000CC04002099160008A5160008440300206A
:1015B000A0020020F0130020F4130020B403002048
:1015C00010100020B103002074000020B20300209E
:1015D0001E4B2DE9F0431A781D460AB31C4B0778C1
:1015E0001E781C4B93F800C002231B4A03F101082C
:1015F000D45C344104F00F04BC420CD20B2C0AD84A
:1016000012F8039012F8088002EB840209EA0C0435
:1016100008EB042414610233102BE6D100232B7055
:1016200003788B420FD90C4B93F8400060B10B4A02
:10163000890012780B44186902B1400800F57770F0
:1016400080B2BDE8F0830020BDE8F083F800002000
:1016500074080020750800208C08002076080020FF
:1016600007299ABF024B33F821000020704700BFC2
:10167000C4010020024B53F82100C0F3CF00704793
:101680006C010020034B53F82100400800F57770EF
:1016900080B2704714010020014B33F811007047ED
:1016A0004A030020014B33F811007047340A002030
:1016B000032810B5114B0FD8114A126894888C4238
:1016C0000AD2D2888A4207D9012202FA00F093F89E
:1016D0004120104383F8410093F841300F2B0CD187
:1016E000064B002283F84120064B998808B2142843
:1016F00002DD1439998010BD9A8010BD8C0800203D
:10170000500A002064080020024B9A8801329A8017
:10171000704700BF64080020074B1A68074B117818
:10172000B3F9040053780B4403EB83039842D4BF0E
:1017300000200120704700BF500A002064080020EC
:10174000064BB3F90400064B1B681B7803EB8303BD
:101750009842D4BF00200120704700BF64080020D9
:10176000500A002010B50446FFF7EAFF002814BF16
:101770002046002000F0010010BD024B01221A7229
:10178000704700BF64080020014B187A704700BF03
:1017900064080020034BB3F90400D0F1010038BF06
:1017A0000020704764080020014B00229A80704797
:1017B00064080020016B0346C26810B5406941B15E
:1017C000196C541A005D013918BF0A46C0B21A6478
:1017D00010BD196A405C0131B1FBF2F402FB141236
:1017E000C0B21A6210BD026B03691AB15168013BA5
:1017F000026C02E0C169026A013B881A1840C0B25B
:101800007047436B13B190F844007047826A436A93
:10181000D31A584258417047334A10B5136C906838
:101820001944081A40F68C2398429160D0605160A8
:1018300013463CD9127893F945108A420BD1111FF7
:10184000082908D893F84610182901D8013103E077
:1018500083F8442002E0002183F8461093F94410F5
:101860008A421CD1204991F84710C1B10021914210
:101870001E4806DA03EB8104246920F81140013187
:10188000F5E7511E00EB41011630814203D00024E0
:1018900021F8024FF9E7164908780130087083F8FB
:1018A0004520002201211A7083F8471010BD92F8DC
:1018B0004710B9B1A0F2EF2440F2DA518C4208D8B7
:1018C00011780B2905D80B1D0131117042F8230046
:1018D00010BD002283F84720991804320020302AD6
:1018E0000861F9D110BD00BF88060020340A00202D
:1018F000DC0A0020084B03EB0010837A0133DBB2D3
:101900000A2B837207D983781BB94178034A22F8DE
:101910001130002383727047D0060020340A002063
:10192000024B1A6C11441964704700BF88060020EE
:10193000024B53F820301B68198070475007002075
:10194000074BA1F57A7153F820304FF47A701A687A
:101950009B884B4393FBF0F39BB21380704700BF0F
:1019600050070020064B1B7813B1012B03D07047A2
:101970004FF4006201E04FF48052024B1A8070472E
:10198000300500200000002038B50C6805462046D0
:1019900008F004FE214602462868BDE8384008F0F9
:1019A00005BE094BDA68D10709D4DA68520708D4B2
:1019B000DB6813F0100F0CBF0420032070470120D8
:1019C00070470220704700BF00200240826A816990
:1019D000436B1144D960416A914203D98A1A5A6013
:1019E000816204E001698A1A5A6000228262002240
:1019F00080F844201A6842F001021A6070478A6831
:101A000010B50C6A036814430A6923F4FF431443B6
:101A10004A6923F0700314438A691443CA69144362
:101A20004A6A14438A6A224313430360CB684360C3
:101A30000B6883604B68C36010BD02684FF6FE738D
:101A4000134003600023036043608360C3602A4B3C
:101A5000984222D0294B984229D0294B984230D025
:101A6000284B984237D0284B98423ED0274B98427B
:101A700006D153F8682C42F4700243F8682C704782
:101A8000234B984206D153F87C2C42F0706243F805
:101A90007C2C70471F4B984206D153F8042C42F01F
:101AA0000F0243F8042C70471B4B984206D153F8A1
:101AB000182C42F0F00243F8182C7047174B98424C
:101AC00006D153F82C2C42F4706243F82C2C70474A
:101AD000134B984206D153F8402C42F4704243F81D
:101AE000402C70470F4B984205D153F8542C42F4C8
:101AF000702243F8542C7047080002401C0002403A
:101B00003000024044000240580002406C00024095
:101B100080000240080402401C04024030040240DD
:101B2000440402405804024010B5104B4178DB6871
:101B30008478DB43C3F30223C3F1040201FA02F207
:101B40000F21D94021401143094B02780901C9B244
:101B50001A4482F8001302780120510902F01F0292
:101B600000FA02F243F8212010BD00BF00ED00E0B2
:101B700000E100E02DE9F843574B0C460168013ABB
:101B8000C3F842108188A3F84610072A42D8DFE83C
:101B900002F0040A101822292F35B3F842202280BF
:101BA000B3F8442013E0B3F844202280B3F8422075
:101BB00005E0B3F8422052422280B3F8442052425A
:101BC00005E0B3F8442052422280B3F842206280FC
:101BD000B3F846301DE0B3F8422052422280B3F8F9
:101BE000442012E0B3F844202280B3F842200CE0F5
:101BF000B3F842202280B3F8442005E0B3F8442033
:101C000052422280B3F8422052426280B3F84630FA
:101C10005B42A380314B1B78002B5AD1B4F90000F2
:101C200005F0FAFE8046B4F9020005F0F5FE07461D
:101C3000B4F9040005F0F0FE294D06462968404637
:101C400005F03EFFE9688146384605F039FF014658
:101C5000484605F02DFEA9698146304605F030FF63
:101C60000146484605F024FE08F0BCFE6968208065
:101C7000404605F025FF29698146384605F020FFDA
:101C80000146484605F014FEE9698146304605F0F4
:101C900017FF0146484605F00BFE08F0A3FEA968B1
:101CA0006080404605F00CFF69698046384605F0C3
:101CB00007FF0146404605F0FBFD296A074630460E
:101CC00005F0FEFE0146384605F0F2FD08F08AFEFA
:101CD000A080BDE8F88300BF8C0800203C000020F5
:101CE0000C05002010B5194B93F84820511C83F8BF
:101CF0004810174902F007024878164903EB4203DF
:101D000031F81010A3F84A1000231846124A9A5AC4
:101D100002331044102B80B2F8D1C00805F07CFECD
:101D20000E4905F0CDFE0E4905F07EFF0D4B044631
:101D30001B68187805F070FE0146204605F0C0FECD
:101D400006F0AAF8084B187010BD00BF8C080020E0
:101D5000C0030020D0030020D608002033335340B6
:101D600000F07F45B4030020B1030020034B1B6843
:101D7000DA79511CD9711344187A7047A8040020ED
:101D800010B5FFF7F3FF0446FFF7F0FF04EB002068
:101D900080B210BDF0B5137C012B29D80C255D4312
:101DA000144C013305EB040C9CF8086030421DD044
:101DB0002D5D1DB1012D14BF022501250E4C4E7B5A
:101DC00004EB051416B1277B3E420FD04F686668BE
:101DD000B7420BD38F68A668B74207D815709460D6
:101DE000C2F804C0D16013741046F0BDDBB2D3E773
:101DF0000020F0BD1000002080C7000810B5094A7F
:101E0000094913688C6812689342F8D1074A106830
:101E100011684FF47A725043001BB0FBF1F002FBE3
:101E2000030010BD080F002010E000E008050020AE
:101E300038B5104C0123054684F84030FFF7DEFF2B
:101E4000E36D41F28832C31A9342236684BF0023B4
:101E500084F8643094F86430EDB20F2BE065E554FB
:101E600003D1054B01221A7038BD024A013382F8B2
:101E7000643038BD8C080020F800002010B50446FE
:101E8000FFF7BCFF0D4B41F288319A6E9866821ABB
:101E90008A42DA6684BF002283F8702093F870309B
:101EA000074A142BD45403D1064B01221A7010BDDB
:101EB000024A013382F8703010BD00BF8C08002048
:101EC000AD010020AC01002010B50446FFF796FFDD
:101ED000164A536F5067C31AB3F57A6F84BF002355
:101EE00082F8783092F8783023B9A82C1CD11049A8
:101EF0000B7006E0022B02D10E490C7001E0242B7E
:101F000001D80D49CC540133DBB282F87830094A4C
:101F1000127852000532934206D1044B002283F816
:101F20007820034B01221A7010BD00BF8C080020DE
:101F3000440100206A0100204501002038B5044614
:101F4000FFF75CFF114B40F6C411DA6FD867821AB5
:101F50008A4284BF002283F8802093F880200AB947
:101F60000F2C11D10A480021017052B1094D182AD5
:101F7000154405F8014C04D1012283F88010027049
:101F800038BD013283F8802038BD00BF8C080020A6
:101F9000F9000020FA00002038B50446FFF72EFFB4
:101FA0000546FFF72BFF401BA042FAD338BD10B502
:101FB00004462CB14FF47A70FFF7EEFF013CF8E7CE
:101FC00010BD2DE9F04106460F4690460025EBB2C4
:101FD000434512D20024E3B2B34209D2084B38463B
:101FE000DA68013482F40052DA60FFF7E0FFF2E7CA
:101FF0003C20FFF7DCFF0135E9E7BDE8F08100BFD9
:10200000001001400B490B7813F0010F03F004029C
:102010000AD072B9980707D443F004030B70064B3B
:102020001A88064B1A8070471AB90220FF21012234
:10203000C7E77047F413002018030020A80300200E
:1020400040F2DB1568430C4C08B54FF480436361E4
:102050004FF400532361851EE368284683F48043D0
:10206000E360E36883F40053E360FFF7A0FF192007
:10207000FFF79DFFF0E700BF0010014008B50368BF
:102080001B68984708BD064B10B5044621461868E2
:10209000FFF7F4FF034B1B689A7954409C7110BD05
:1020A000AC040020A804002038B5044624200D46C6
:1020B000FFF7E9FF4D20FFF7E6FF002C084C0CBFAF
:1020C0003E202120FFF7DFFF2368002228469A7177
:1020D000FFF7D9FF236893F84900BDE83840D2E7FD
:1020E000A804002001460020DEE7F8B50E4E0F4C94
:1020F0000F4DC1B20746306884F88110FFF7BEFF6C
:102100002B6894F881109A7930684A409A71C7F325
:10211000072184F88110FFF7B1FF2B6894F8811034
:102120009A794A409A71F8BDAC0400208C080020CE
:10213000A8040020F8B51B4D1B4C1C4F0646C1B22D
:10214000286884F88210FFF799FF3B6894F88210A2
:102150009A7928684A409A71C6F3072184F8821058
:10216000FFF78CFF3B6894F882109A7928684A4000
:102170009A71C6F3074184F88210FFF77FFF3B682E
:1021800094F882109A7928684A409A71310E84F83E
:102190008210FFF773FF3B6894F882109A794A40E7
:1021A0009A71F8BDAC0400208C080020A80400201F
:1021B00010B5441E14F8011F21B1034B1868FFF736
:1021C0005DFFF7E710BD00BF80060020014B1868D7
:1021D00054E700BF600B002010B50024094BE0B2AB
:1021E0001B7883420CD9084B33F81010074B53F877
:1021F00020301BB10B2801D89B6898470134EDE7CC
:1022000010BD00BFCC130020CE13002050070020CB
:10221000054B1B6803EBC00090F9063019420CBF58
:1022200001204FF0FF307047540A00200A4B1A6813
:1022300002EBC002D379FF2B07D0084909789942F5
:1022400003D9074A32F8130004E00728D4BF908866
:1022500040F2DC5000B27047540A0020CC04002049
:102260004A0300202DE9F04F0C68836889B0D0F84C
:1022700000A0D0F804800646204603938B4608F061
:102280007BFB0746204608F0EBFBDBF80440814669
:10229000204608F071FB0546204608F0E1FBDBF81C
:1022A000082004461046019208F066FB019A834616
:1022B000104608F0D5FB39460290584605F000FC60
:1022C00039460490029805F0FBFB594605904846B4
:1022D00005F0F6FB02990690484605F0F1FB294609
:1022E0000790584605F0ECFB0146504605F0E8FB28
:1022F00021468346069805F0E3FB0146059805F064
:10230000D7FA0146404605F0DBFB0146584605F08A
:10231000CFFA21468346049805F0D2FB0146079880
:1023200005F0C4FA0146039805F0CAFB0146584679
:1023300005F0BEFA3060029905F1004005F0C0FBDF
:102340000146504605F0BCFB21468346079805F040
:10235000B7FB0146049805F0A9FA0146404605F08E
:10236000AFFB0146584605F0A3FA2146834605987F
:1023700005F0A6FB0146069805F09AFA0146039877
:1023800005F09EFB0146584605F092FA2146706022
:10239000504605F095FB2946044609F1004005F03A
:1023A0008FFB0146404605F08BFB0146204605F0B9
:1023B0007FFA39460446284605F082FB0146039819
:1023C00005F07EFB0146204605F072FAB06009B0C8
:1023D000BDE8F08F2DE9F84F374E04463768384690
:1023E00008F0CAFA0546384608F03AFB7668804697
:1023F000304608F0C1FA8346304608F031FBD4F885
:10240000049006462946484605F05AFBA7688246CE
:102410004146384605F054FB0146504605F046FA61
:1024200021688246584605F04BFB41460446484623
:1024300005F046FB314605F043FB0146204605F01A
:1024400037FA31460446384605F03AFB294605F08E
:1024500037FB0146204605F02BFA0146504608F0AE
:102460008DFB164905F02CFB04F046FF10A3D3E9C1
:10247000002305F0BFF8124B044618680D4604F01F
:102480003BFF02460B462046294604F0D7FD0022BA
:102490000C4B05F0AFF805F0B5F908F0A3FA83B2DC
:1024A0001A0444BF00F5B4739BB218B2BDE8F88FAC
:1024B000182D4454FB210940000300200000E14492
:1024C000340500200000244080EAE073A3EBE073B1
:1024D0008B4206DB002801DD401A704702D0084419
:1024E000704700207047044B1A78510744BF22F010
:1024F00004021A70704700BFF413002070B5FFF794
:102500001FF938B3144C237A0BB9A38070BD134D57
:102510002E78C6F38000FFF725F990B1104B46F0F6
:1025200002061A680F4B51892E7019805189598003
:1025300052899A800C4A12685288DA80E388013303
:10254000E380FFF7E9F810B92B785B0702D4BDE808
:102550007040C8E770BD00BF64080020F41300207D
:10256000600800204A030020500A00202DE9F041B5
:1025700002780346202A00F10100F9D0092AF7D099
:102580002D2A02D10346414D04E02B2A08BF034601
:102590004FF07E551E460024334616F8012BA2F15B
:1025A0003007F9B209290DD83949204605F088FAD3
:1025B0000446384605F030FA0146204605F078F921
:1025C0000446E9E72E2A17D1314F334616F8010B9E
:1025D0003038C2B2092A0FD805F01EFA394605F084
:1025E00023FB0146204605F063F929490446384695
:1025F00005F066FA0746E8E71A7802F0DF02452A96
:1026000038D15A782D2A02D10233012604E02B2A30
:1026100014BF013302330026013B002713F8012FBA
:10262000303AD1B2092903D80A2101FB0727F5E77F
:10263000B7F59A7F28BF4FF49A77B8464FF07E518E
:10264000B8F1070F07D90846124905F039FAA8F181
:1026500008080146F4E707F0070737B108460C49B8
:1026600005F02EFA013F0146F7E72EB1204605F0AE
:10267000DBFA04E04FF07E51204605F021FA0146D6
:10268000284605F01DFABDE8F08100BF000080BFBC
:102690000000204120BCBE4CF0B50124B0FBF4F595
:1026A0008D4201D34C43F9E70026DCB1B0FBF4F5D1
:1026B00004FB1500B4FBF1F41EB9002D01DC002C65
:1026C000F3D1092D03F101075FFA85FC04DD002A2F
:1026D0000CBF5725372500E0302565441D700136B5
:1026E0003B46E2E71C70F0BDF0B50124B0FBF4F509
:1026F0008D4201D34C43F9E70026DCB1B0FBF4F581
:1027000004FB1500B4FBF1F41EB9002D01DC002C14
:10271000F3D1092D03F101075FFA85FC04DD002ADE
:102720000CBF5725372500E0302565441D70013664
:102730003B46E2E71C70F0BD70B50646B6FBF2F40E
:102740000846154614B12046FFF7F6FF05FB146452
:10275000024B1B5D00F8013B70BD00BF38D4000880
:102760002DE9F041069C002B06460F460CBF4FF0AA
:1027700020084FF03008234613F8011B09B915460D
:1027800003E0002AFBDD013AF6E7002D04DD3046C8
:102790004146B847013DF8E714F8011B11B1304636
:1027A000B847F9E7BDE8F081024B9A6822EA0000D9
:1027B000986070470C0F002010B50023094CDAB266
:1027C00004EB8204246A01338442F7D10023064CCF
:1027D000D8B234F8104001338C42F8D102EB8000BB
:1027E000C0B210BD80C70008B0C70008044B53F842
:1027F00020301BB107289CBF1B681980704700BFA1
:102800008007002010B5054C00202188FFF7EEFF5F
:1028100061880120BDE81040E8E700BF60000020AB
:102820002DE9F0410F88002347FA03F2D2072BD598
:102830008A7803F0070512F0100F18BF91F803C053
:1028400002F00F0618BF46EA0C06AD004FF00F0C61
:102850000CFA05FC06FA05F5DC0850F82480282A55
:1028600028EA0C0C45EA0C0540F8245005D1012259
:102870009A40C46824EA020205E0482A04D10122F1
:102880009A40C4682243C2600133102BCCD1BDE80A
:10289000F08100BFAFF30080426A10B58469A15493
:1028A000416A02690131B1FBF2F402FB1412426287
:1028B000426B32B11368DB0708D4BDE81040FFF764
:1028C00085B8036DDA6842F08002DA6010BD0FB49B
:1028D0002DE9F04F684A89B012AB1668674A53F881
:1028E000045B176804939B462978002900F0B880A0
:1028F000252902D001353046B0E06C78302C03D069
:1029000002354FF0000903E0AC784FF001090335C0
:10291000A4F13003092B4FF000081AD8A4F13003BA
:10292000DAB2092A07D80A2B13DC0A2202FB08387C
:1029300015F8014BF2E7A4F16103052B02D8A4F1CD
:102940005703F0E7A4F14103052B02D8A4F13703A4
:10295000E9E76C2C03BF2C78012201350022632C9F
:1029600066D006D8252C77D0582C3FD0002C77D0B5
:10297000BAE7732C63D002D8642C11D0B4E7752C5D
:1029800002D0782C32D0AFE70BF1040A05ACDBF8AB
:1029900000000A2112B10022234613E0234620E062
:1029A0000BF1040A05ACDBF8000072B1002806DA6E
:1029B0002D238DF8143040420DF1150300E023461D
:1029C0000A210022FFF790FE0DE0002806DA2D23F1
:1029D0008DF8143040420DF1150300E023460A2122
:1029E0000022FFF759FED34600941AE00BF10403CE
:1029F00003930DF1140ADBF80000102132B1583CAA
:102A0000624262415346FFF76FFE06E0B4F158039D
:102A10005A425A415346FFF73FFEDDF80CB0CDF85D
:102A200000A03046394642464B46FFF799FE5BE729
:102A300030469BF800100BF10404B8470AE0DBF8BD
:102A40000030304600933946424600230BF104041F
:102A5000FFF786FEA34647E730462146B84743E7DF
:102A6000074B186803681B6998470028F8D009B01D
:102A7000BDE8F04F04B070470405002000050020B9
:102A8000600B002037B502790D46110604468368B5
:102A900006D526494FF4947091F8BC1400FB01331D
:102AA00002F03F02042A12D006D8012A0DD0022AD1
:102AB0002FD193F900102DE0102A0AD0202A0AD035
:102AC000082A26D1B3F9001024E0197822E01988E9
:102AD00020E019681EE06946186801F0E9FB01462C
:102AE0001348FFF7F4FEF5B1E06804F095FF69467E
:102AF00001F0DEFB01460F48FFF7E9FE206904F014
:102B00008BFF694601F0D4FB01460A48FFF7DFFE60
:102B100009E000210848FFF7DAFE25B10748E1681F
:102B20002269FFF7D4FE03B030BD00BF0C0F0020B8
:102B30008FDB00088EDB000861D400085DD400083C
:102B40007FB5044607F02AFD082824D100231F4939
:102B5000E25C09681144497801F00301022908BFC9
:102B6000203AE2540133082BF1D10025665D184864
:102B7000314607F006FD28B101356019314607F0EE
:102B800000FD18B11348FFF713FB1CE0082DEDD131
:102B9000204601F0EFFA1048FFF70AFB00230F4A26
:102BA00004A91A4492F80E210A440949595C0133D8
:102BB000082B02F80C1CF2D10023094801A98DF85A
:102BC0000C30FFF784FE04B070BD00BF8000002011
:102BD000E8DA000864D4000884D400080C0F002050
:102BE000E1DB00082DE9F047054607F0D7FC324B42
:102BF0000446D3F808809A4690B93048FFF7D8FACF
:102C00002F4B53F8241049B10123A34013EA080FB6
:102C100002D02C48FFF75BFE0134F1E72A4821E09F
:102C200028462A49224607F0C1FC58B92848FFF730
:102C3000BFFA284C54F8041F0029EFD02148FFF7B1
:102C400046FEF7E72B7800262D2B03BF013504F154
:102C5000FF344FF001094FF00009194B53F826706B
:102C600027B91D48BDE8F047FFF7A2BA2846394604
:102C7000224607F09BFCE0B90120B040020601D5D6
:102C80001648EFE7830501D51548EBE7B9F1000FCA
:102C900003D0FFF789FD134804E040EA0800CAF8B2
:102CA00008001148FFF784FA39461048BDE8F0479C
:102CB0000DE60136D1E700BF0C0F002099D40008C3
:102CC0003CC80008ACD4000810DC000813D9000888
:102CD000B0D4000838C80008C5D40008DCD4000807
:102CE000EED4000802D500080CD50008E1DB00088E
:102CF0002DE9F04389B0044607F050FCC6B2002E1F
:102D00006CD18B48FFF754FA8A4C2069002105F0FA
:102D10006BF840BB013688483146FFF7D8FD206983
:102D200004A901F0C5FA01468448FFF7D0FD6069A7
:102D300004A901F0BDFA01468048FFF7C8FDA0696B
:102D400004A901F0B5FA01467C48FFF7C0FDE0692F
:102D500004A901F0ADFA01467948FFF7B8FD0C2E41
:102D600004F11004D1D10025764C2F462B464FF0AC
:102D70000008B04504F1100415DA184654F8101C88
:102D800004F096FD54F80C1C8146284604F090FD92
:102D900054F8081C0546384604F08AFD08F101087D
:102DA0004B460746E5E76848019302950397FFF70E
:102DB000FFF9002401ABE058644920F0004005F021
:102DC0003BF8634B634A0434002814BF104618468E
:102DD000FFF7EEF90C2CEDD15F4891E020465F49FA
:102DE000052207F0E3FB38B9524B002203441030B0
:102DF000C0281A61F8D197E020465949042207F00B
:102E0000D5FB06462046002E40D1202107F0B9FB15
:102E1000002800F08980451C284607F0BFFB344697
:102E20008046504B53F824600EB94F4868E028465E
:102E300031465FFA88F207F0B9FB671C20BB3D4BB7
:102E40000021C2181030C02811619C46F7D1474BB1
:102E5000002403EBC702D2F804E09846BEF1000F4D
:102E600004D143483146FFF732FD55E018F83730BA
:102E70009C42F6DA23010CEB0305103573440FCBAB
:102E8000013485E80F00F1E73C46CAE707F0DBFBB9
:102E9000461E0B2E074643DC2046202107F071FB1F
:102EA000054640B1451C2846FFF760FB214B3F011A
:102EB000D851012400E004462846202107F061FB98
:102EC000054640B1451C2846FFF750FB194B01341D
:102ED00003EB061358612846202107F052FB0546F4
:102EE00040B1451C2846FFF741FB124B013403EB70
:102EF000061398612846202107F043FB18B91D48A6
:102F0000FFF756F910E00130FFF730FB094B032CB7
:102F100003EB0616F061F2D11748FFF7E9FE03E074
:102F200016480C21FFF7D3FC09B0BDE8F08300BFC1
:102F30001DD500080C0F002048D500084ED500080C
:102F4000E1DB0008200F002052D500080AD7233CFF
:102F500019D5000815D5000810DC000861D5000857
:102F600067D50008E0C700086CD5000898C10008C4
:102F700081D5000891D50008AADC0008CBD500084F
:102F8000F8B5074607F00AFB044638B9194B1A484A
:102F90005A791A4B013A53F8221028E0384618495A
:102FA000224607F003FB60B91648FFF701F9164CFB
:102FB00054F8041F19B11548FFF789FCF8E71448C5
:102FC00005E000250D4B53F8256026B91148BDE8F2
:102FD000F840FFF7EDB838463146224607F0E6FAEA
:102FE00001350028EED1034B0B485D713146BDE839
:102FF000F8406CE40C0F0020F3D50008E0C700088F
:1030000013D9000807D60008DCC70008ACD40008B4
:1030100010DC00086CD500081AD6000870B504460C
:1030200007F0BCFA08B91E482EE020461D4907F0FB
:103030002FFB00242646254678B12CB1012C06D161
:1030400007F001FB064602E007F0FDFA05461549C8
:103050000020013407F01CFBEEE70B2D04D9BDE87E
:10306000704011480C2132E4012C07DC0F4B29463B
:1030700033F915200E48BDE8704028E4A6F57A73B0
:10308000B3F57A7F03D90B48BDE870401FE40A48C6
:1030900029463246FFF71BFC044B23F8156070BD30
:1030A0002CD6000879DC000866D60008D20400207F
:1030B0008CD60008A4D60008C6D6000838B5054648
:1030C00007F06CFAC0B270B90446134B04F1200249
:1030D0001B682146114853F822200134FFF7F7FB03
:1030E000152CF2D138BD284607F0ADFA1428044655
:1030F0000BDC2021284607F044FA07F0A4FA064B1F
:1031000020341B6843F8240038BD05481521BDE86C
:103110003840FFF7DCBB00BF1C020020DFD60008F0
:10312000EBD600082DE9FF4180460F461C480021E0
:10313000142207F0F2F9002673B2002B28DC0C22CF
:103140005A43184C02F10C032244127A23440025FE
:10315000E8B20135CAB91D7AD1B2013295B9401A27
:10316000002801DC0136E7E701AD94E8070085E8B7
:10317000070093E8070084E8070095E8070083E864
:103180000700EFE7691E0D40E6E7511E0A40DFE742
:10319000034A4046394604B0BDE8F041FEF7FABDA7
:1031A00010090020100000200E4B1A784F2A16D16B
:1031B0005A88B2F5986F12D11A79BE2A0FD193F8B6
:1031C000BD240020EF2A0CD113F8012B5040064AF1
:1031D0009342F9D1D0F1010038BF002070470020A0
:1031E0007047704700F80008C0FC00084A4B4F22A7
:1031F0002DE9F3411A704FF498625A80BE221A7179
:10320000EF2283F8BD24002283F8BE2411461E4617
:10321000B35C0132B2F5986F81EA0301F8D13E4BFD
:103220003E4A83F8BE143E4B04275A6002F18832AE
:103230005A600020013F17F0FF075DD0384B342261
:10324000384CDA60C4F309037BB1331903F17843D6
:10325000A3F57843D3F800804FF400500023019386
:1032600001F0BEFA0428E5D11BE04FF4302001F054
:10327000B7FA0428DED12A4D4FF430202B6943F0F1
:1032800002032B616C612B6943F040032B6101F059
:10329000A7FA2A6941F6FD73134004282B61D4D0A4
:1032A000C8E71F4D4FF400502B6943F001032B6119
:1032B0001FFA88F3238001F093FA042812D1A31C8B
:1032C0000193019B4FEA1848A3F800804FF4005087
:1032D00001F086FA2B6941F6FE721A4004282A6131
:1032E00006D0A7E72B6941F6FE721A402A61A1E7D2
:1032F0000D4B04349C42A5D1094B04281A6942F0B5
:1033000080021A6102D1FFF74FFF10B90A20FEF7C1
:1033100097FE02B0BDE8F0810C0F00202301674545
:103320000020024000F80008C0FC000808B504486E
:10333000FEF73EFFFFF75AFFBDE8084000F0A0BCD3
:1033400011D70008094B30B59D68094B05F480552D
:103350001868084B1C6800230DB1828800E0A28821
:1033600005495A520233182BF6D130BD0C0F0020FC
:10337000580A00205C0A0020D204002010B5044640
:103380000748FEF715FF074A00231370064A13602B
:10339000064A1370FFF7D6FF2046BDE81040C5E788
:1033A00018D70008680B0020640B0020F3130020DE
:1033B0002DE9F04F8BB009938A4B0792B3F90220A5
:1033C000B3F90030002AB8BF5242002BB8BF5B42AD
:1033D0009A42B8BF1A46844B03921B88814603F079
:1033E0000302069203F0020203F0010392B2059376
:1033F0000023089219461E46184604931F461A4693
:10340000069C002C41D0022A3FD0764C079F0D5FCE
:103410007C426D00A54203DB3C46A542B8BF2C466A
:10342000724DDDF824A031F905C03AF90150CCEB1A
:10343000040404EB050C99F80750642405FB0CF513
:1034400095FBF4F599F81B406FF004076743BD4204
:1034500005DB04EB8404A542B4BF2F462746644D28
:103460005C59644442F2107C6445A8BF6446DFF8AE
:1034700098C16445B8BF64465C5199F811506C43DB
:1034800024130494069C012C3BD05A4D55486D5E84
:10349000594C85EAE576A6EBE576B6F5206F085E31
:1034A00019F802C053F804801DDC022A15D05026FA
:1034B000464396FBFCFC042695FBF6F5C5EB0C0C8D
:1034C000E0444E4EB8F57A5FA8BF4FF47A58B04545
:1034D000ACBF44F80380E65007E080EAE076A6EB54
:1034E000E076642EE3DD0025E550434C1E597D2433
:1034F00096FBF4F609EB0204A47A6643402496FB9B
:10350000F4F6089CB4B1022A68D0DDF80CA0DDF80E
:1035100010B00AFB00F40AFB06F8CAF5FA7505FBC1
:10352000074405FB0B854FF4FA7C94FBFCF495FBF8
:10353000FCF506E0059C002C50D0022A4ED0049DDC
:103540003C46DFF8B0C04FF0040B31F80CC00FFA66
:103550008CF898FBFBFADFF8B4B012F80BB00BFB59
:103560000AFA6FF04F0B9AFBFBFAA244CDF804A0C5
:10357000DFF89CA0042431F90AB021F80AC0CBEB93
:1035800008080AF1080C98FBF4F80AF114041C5915
:1035900053F80CB00AF1140AA34453F80C40C34486
:1035A00043F80A40164CDDF804A0145D013204FB18
:1035B0000BFB20249BFBF4FBCBEB050B114DDA44FA
:1035C000032A43F80C8021F805A003F1040301F15C
:1035D00002017FF415AF0BB0BDE8F08F354604460D
:1035E000AFE700BF7C030020A603002008030020F3
:1035F000A00A00203C030020A80A002080C1FFFF91
:103600008A030020D40A0020F0D8FFFF84030020A2
:10361000240900202DE9F04F89B00793524B029105
:10362000B3F9043001920393504B06461B8803F014
:10363000010103F002039BB204934D4B0691B3F8D2
:1036400000A04FF6FF714FEA1A13B1FBF3F100230C
:1036500005911D461946022D08D1029FDDF80CC0C8
:103660007C791B340CFB04F4641129E03E4C019A74
:1036700031F9048057424FEA4804BC4203DB174645
:10368000BC42B8BF27463B4CDDF81CC00C5F3F1B5B
:103690003CF901403A19069C7CB9029C277907F154
:1036A0001B0408FB04F4049F24114FB190F811C0CF
:1036B0000CFB02F704EB272402E0C47954432411E5
:1036C0002D4FDFF8C48031F907C004279CFBF7FCBD
:1036D000CCEB040C0AFB0CF496F80AB053F8087013
:1036E000E4120BFB0474254FB4F5001FA8BF4FF480
:1036F0000014BC42B8BF3C46214F10F80590DA597F
:1037000043F8084043F807C0C2EB0C0809FB0CF96A
:10371000DDF814C001350CFB08F807F10C0C183764
:10372000DA5953F80CB04FEAA818934453F80C2018
:10373000C344DA51377D032D07FB0BF74FEA2727E8
:1037400007EBE91707EB64340E4F43F80C80CC53BA
:1037500006F1010601F1020103F104037FF47BAFDE
:1037600009B0BDE8F08F00BF7C030020A603002055
:1037700048030020080300203C0300200000E0FF75
:1037800044090020D40A0020A80A00202DE9F04FA7
:1037900089B00793714B814618880492039104F015
:1037A00037F96F4904F08CF9029002994FF07E507E
:1037B00004F03AFA002406904E462546A046B8F199
:1037C000020F684B0BD10399B3F904004A790A320E
:1037D000504304F021F9644904F026FA35E0049AD4
:1037E0005F5F53429F4203DB13469F42B8BF3B4695
:1037F0005E4AAA5E9B1A079A505F184404F00CF9BF
:103800005B4904F011FA5B4B8346B3F800A01AF051
:10381000010F04D0D9F8441004F052F915E0039BCD
:1038200018791430784304F0F7F84F4904F0FCF9A4
:103830001AF0020F074609D0D9F84810584604F08C
:103840003FF90146384604F033F807464A4BDFF8A3
:103850004CB1585F04F0E0F8484BD96804F030F9F7
:1038600082465146384604F021F8316A074604F092
:1038700027F902990590384604F022F9F16A04F01C
:103880001FF954F80B1004F013F83D49074604F0F3
:10389000B5FA30B938463B4904F0CEFA10B1394F89
:1038A00000E0374F4BF80470DFF8F4B0504654F89E
:1038B0000B1003F0FBFF44F80BA0069904F000F98D
:1038C0000BF10C03E2580BF1180B54F80B10824665
:1038D00010460192009303F0EBFF514603F0E8FF1E
:1038E000019A009B44F80B2044F803A0264904F0F9
:1038F0009BF9B16B04F0E4F82449824604F07EFAA7
:1039000038B95046224904F097FA20B1DFF880A078
:1039100001E0DFF878A00598394603F0C9FF514669
:1039200003F0C4FF07F05EF81A4BB0F57A7FA8BF2A
:103930004FF47A709842B8BF184608F10108164B48
:10394000B8F1030FE85204F1040405F1020506F191
:1039500004067FF434AF09B0BDE8F08F48030020BF
:10396000BD3786357C030020000048420803002054
:1039700000002041A60300203C030020200200207C
:1039800000007AC300007A4300004040000096C364
:103990000000964318FCFFFFD40A0020B40A002060
:1039A00068090020F0B5934C934A23689D8AADB214
:1039B000E9B211F0010F36D0198821F40061090431
:1039C000090C1980198889B241F48061198000219D
:1039D00082F86810894908788949B8B192F8690075
:1039E00018B988480078FF2810D1012082F86900B2
:1039F00085480078022804D1188880B240F400601D
:103A00001880097841F00101198216E1097801F066
:103A1000FE0119827B4B1B78FF2B00F00E81FF23E8
:103A200082F8683009E18F0740D5BFF35F8F764990
:103A30000878C0B2012816D1704D2D789DB192F84A
:103A4000695085B1198821F480610904090C198035
:103A5000BFF35F8F198B198882F86A0089B241F42D
:103A6000007119801DE0188BBFF35F8F0878022862
:103A70000CD16248007848B192F8690030B11988D9
:103A800021F480610904090C1980D0E00978032928
:103A900007D15A49097821B192F86910002940F0FC
:103AA000C680998889B241F48061C5E04E0764D52B
:103AB000012182F86A105149097800293ED092F814
:103AC000691000293AD0504992F8680009784F4DA2
:103AD000022919881FD921F480610904090C198071
:103AE0001F8A2E68C1B2FFB240B23754188880B224
:103AF00040F4007018808B1C82F8683023682868B6
:103B00001D8A013149B2EDB24554998889B241F418
:103B1000806199802CE089B241F4007119801E8A7D
:103B20002D68C1B2F6B240B22E541B8A481C40B276
:103B3000DBB203312B5482F8681019E092F8691057
:103B400011B93349097851B1198889B241F400712A
:103B5000198092F86830013382F8683008E01988DB
:103B600089B241F480711980234B012183F86910D7
:103B700021680B88D805FCD45FE001F0400101F01A
:103B8000FF06214809B32149B3F810C00F6892F825
:103B900068105FFA8CFCCDB26E1C49B2F6B207F821
:103BA00001C082F86860077876B2F11C8F4205D1B7
:103BB000998821F480610904090C99800378B34243
:103BC0003BD1023582F8685037E0290635D592F8A6
:103BD00068104DB26F1C1FD00E4E01313668C9B24D
:103BE000755D82F86810EDB21D82007849B2884296
:103BF00023D11CE0D00A002024090020C30A0020A1
:103C0000C00A0020C10A0020CC0A0020C80A0020F7
:103C1000C20A0020C40A0020144982F868600978AA
:103C2000C9B219821249097809B9017829B9998864
:103C300021F480610904090C99800E4B92F96810F7
:103C400018780D4B421C91420FD1002283F8692055
:103C500093F86A3033B12268938823F440731B04CD
:103C60001B0C9380054B00221A70F0BDC10A002086
:103C7000C30A0020CC0A002024090020CD0A00201D
:103C800010B50948FEF794FA084B1C6823682046D3
:103C90001B69984718B90A20FEF789F9F6E7044A24
:103CA000044BDA6010BD00BF2DD70008800600204D
:103CB0000400FA0500ED00E0F8B50121044600F02B
:103CC00061FB01283B4F01D0002616E04FF6FE7342
:103CD0002382A68D0025B6B22046795DFEF76CFDE5
:103CE000354B142202FB0030C36813B1007C31460F
:103CF00098470235082DEFD1E6E7BD5D95B920461E
:103D0000022100F03FFB012850D14FF6FD732382C2
:103D100029462046FEF750FD274B142202FB0030B7
:103D2000A18E3EE0042D12D12046294600F02AFB48
:103D300001283BD14FF6FB73238229462046FEF72C
:103D40003BFD1D4B142202FB0030218F29E0082D82
:103D500012D12046294600F015FB012826D14FF646
:103D6000F773238229462046FEF726FD124B1422C4
:103D700002FB0030A18F14E00C2D17D1204610213A
:103D800000F000FB012811D14FF6EF732382294682
:103D90002046FEF711FD084B142202FB0030B4F858
:103DA0004010836889B20BB1007C98470236082E18
:103DB000A3D1F8BDB0C70008400500202DE9F041AF
:103DC000067B04460F460068314690461D46FEF7C6
:103DD000F3FC0F2808D8194B142202FB0030C0F85E
:103DE0000880C56006710774237B22680C2B1CD8E1
:103DF000DFE803F0071B1B1B0C1B1B1B111B1B1BF2
:103E0000160093899BB243F002030DE093899BB2A5
:103E100043F0040308E093899BB243F0080303E0F6
:103E200093899BB243F01003938125B193899BB290
:103E300043F001039381BDE8F08100BF40050020FD
:103E4000254B10B55343254A254C12680139B2FB66
:103E5000F3F20388013AA04289B292B29BB212D027
:103E600004F50064A0420ED0B0F1804F0BD0A4F551
:103E70009834A04207D004F58064A04203D004F532
:103E80008064A04202D123F070039BB2154CA04283
:103E900006D004F58064A0421CBF23F440739BB29B
:103EA00003800F4B8185984202850FD003F5006394
:103EB00098420BD003F54063984207D003F5806326
:103EC000984203D003F58063984201D10023038612
:103ED0000123838210BD00BF40420F007800002004
:103EE000002C0140001000402DE9F74F9F4E9B46EB
:103EF00033780C4691465A1C054606F8042B006898
:103F0000224649460C275F43FFF79AFFAB68686873
:103F1000ADF8043018238DF8063001A902238DF87E
:103F20000730FEF77DFC2B7B06EB070A2C680C2B79
:103F300000F2F280DFE813F00D00F000F000F00076
:103F40004D00F000F000F0008200F000F000F00002
:103F5000B600238C864823F001031B041B0C23842A
:103F6000218CA288238B844223F073034FEA0343FE
:103F70004FEA134389B292B243F0700314D000F5B4
:103F80000060844210D000F5406084420CD000F5FF
:103F90008060844208D000F58060844204D021F023
:103FA000020141F0030107E021F00E0122F440720A
:103FB00041F0030142F48072A2802383A4F834B05C
:103FC0002184238B23F008031B041B0C43F00803FC
:103FD00032E0238C664823F010031B041B0C23845F
:103FE000218CA288238B844223F4E6434FEA0343C7
:103FF0004FEA134389B292B243F4E04308D000F58C
:104000000060844204D021F0200141F0300107E03B
:1040100021F0E00122F4406241F0300142F480627C
:10402000A2802383A4F838B02184238B23F4006377
:104030001B041B0C43F4006323836DE0238C4C486A
:1040400023F480731B041B0C2384218CA288A38B74
:10405000844223F073034FEA03434FEA134389B2C8
:1040600092B243F0700308D000F50060844204D09F
:1040700021F4007141F4407107E021F4606122F401
:10408000405241F4407142F48052A280A383A4F8CC
:104090003CB02184A38B23F008031B041B0C43F0CA
:1040A000080338E0B4F820C0314A2CF4805C4FEAB1
:1040B0000C4C4FEA1C4CA4F820C0B4F820C0A388D4
:1040C000B4F81C802CF4005C28F4E6484FEA084859
:1040D0004FEA0C4C4FEA18484FEA1C4C94429BB2F2
:1040E00048F4E0484CF4405C03D002F5006294428E
:1040F00003D123F4804343F48043A380A4F81C80BD
:10410000A4F840B0A4F820C0A38B23F400631B04E0
:104110001B0C43F40063A383AB7B43B1B4F844307E
:104120006FEA43436FEA53439BB2A4F844302388B9
:104130009BB243F0010323802B7B0C2B10D8DFE8CC
:1041400003F0070F0F0F090F0F0F0B0F0F0F0D00CD
:10415000343404E0383402E03C3400E04034F451BC
:104160005046AAF8049003B0BDE8F08F90090020F3
:10417000002C014070B50546441E14F8011F61B1C2
:10418000064E304606F0FDF90028F6D0861B04489E
:10419000631B304480F80E31EFE770BDE8DA0008A9
:1041A0000C0F002070B50022064628491001431864
:1041B000415CB14204D00132062AF6D1002070BD24
:1041C000234D082E05F194040FCB84E80F002B46F5
:1041D00017D007D8012E0DD0022E34D11D4B1B68ED
:1041E0009B680BE0102E27D0202E2CD1194B1B687A
:1041F0001B6903E0174B1B685B6820E0C5F898302B
:104200001DE0154A1268127A042A1CD8DFE802F071
:104210000A0A030A0A00114AC5F89820C5F89C202A
:10422000032206E04FF4E132C5F89820C5F89C203F
:10423000012283F8A12006E0064B1B68DB68C5F865
:104240009C30204670BD064870BD00BF50C20008BB
:1042500090090020B0040020F4000020A086010096
:10426000240A00200F4970B500230C781A46D8B2F2
:10427000844205D00D7B854208BF01200CD100E0AF
:1042800000200C2505FB0010074D084E154495F83D
:1042900028510132755D05720133052B01D0012AC9
:1042A000E5D970BD100000200C0F0020F1DA0008E5
:1042B00030B587B005460C4603A800210C2206F055
:1042C0002CF92846002103F0B7FD20B128462A49E1
:1042D00003F0EEFA03E02846274903F0E7FA2749FE
:1042E00003F0EEFB03F0B2FD054685EAE570A0EBB6
:1042F000E57069460A22FEF71FFA00239D4203700B
:10430000ACBF20232D2368468DF80C3006F046F90B
:10431000012807D130238DF80D308DF80E308DF83F
:104320000F300CE0022805D130238DF80D308DF8C8
:104330000E3004E0032804BF30238DF80D306946A9
:1043400003A806F011F903A806F028F90338C5B24E
:104350002A4603A9204606F04BF900236355204660
:10436000074906F001F903A92046294406F0FCF8A4
:10437000204607B030BD00BF6F12033A00007A44F8
:1043800039D70008038A828911EA030092B203D068
:1043900011420CBF0020012070477C4B70B51B7888
:1043A000012B0CBF0325002599BB048C24F00104CC
:1043B0002404240C0484038B048C9BB223F0F303A9
:1043C00043F0010343EA0515714BA4B2984215D09E
:1043D00003F50063984211D0B0F1804F0ED0A3F5E1
:1043E000983398420AD003F58063984206D003F5CB
:1043F0008063984218BF24F00A0401D124F002041B
:1044000044F00104224305830284038B23F00C0350
:104410003AE004293FD1048C5D4B24F010042404BD
:10442000240C0484018B048C21F440710905090DCE
:1044300041F480719842A4B241EA053512D003F5E7
:10444000006398420ED0B0F1804F0BD0A3F59833A3
:10445000984207D003F58063984203D003F5806348
:10446000984207D124F0200444F0100444EA0212D8
:1044700092B204E024F0A00444F010042243058327
:104480000284038B23F440631B041B0C0383038B04
:104490009BB2038370BD0829018C37D121F4807150
:1044A0000904090C0184838B048C9BB223F0F30371
:1044B00043F0010343EA0515354BA4B2984212D0EC
:1044C00003F5006398420ED0B0F1804F0BD0A3F5F6
:1044D0009833984207D003F58063984203D003F5E0
:1044E0008063984207D124F4007444F4807444EA51
:1044F000022292B204E024F4206444F48074224343
:1045000085830284838B23F00C0338E021F48051EF
:104510000904090C0184838B068C23F440731B056A
:104520001B0D43F4807343EA0535194BB6B298422C
:1045300012D003F5006398420ED0B0F1804F0BD03B
:10454000A3F59833984207D003F58063984203D0CF
:1045500003F58063984207D126F4005646F480564E
:1045600046EA023292B205E047F6FF54344044F482
:104570008054224385830284838B23F440631B048D
:104580001B0C8383838B9BB2838370BD84060020C6
:10459000002C014038B5114C04EB0014A278E368FC
:1045A00042B90122A270A1801868197B0222BDE8DD
:1045B0003840F2E6A288E1806078891A084A89B218
:1045C00002EB40020025A2F8A410A5702181186812
:1045D000197B2A46FFF7E1FEA57238BDD006002000
:1045E000900900201F4B10B55A6802F00C02042AF3
:1045F00003D0082A04D01C4A14E01C4A126811E0B7
:104600005A685968C2F38342C90302F1020201D415
:10461000174906E0596811F4003F1449096818BFAA
:1046200049084A4302605968124AC1F30311545CB5
:104630000168E14041605C68C4F30224145D21FA22
:1046400004F484605C68C4F3C224145DE140C1607A
:104650005B68C3F381331A44137CB1FBF3F101614E
:1046600010BD00BF0010024000127A002800002098
:1046700000093D004C00002070B5447986B004F07C
:104680000403866803F0FF0523B14FF480654FF4FF
:10469000005300E02B4614F0010F14BF0422002247
:1046A000A107046D48BF42F00802218A48BF92B2B8
:1046B00089B221F440510B432382A38901A89BB204
:1046C00023F4B05323F00C031D432A43A281A38A91
:1046D00023F440731B041B0CA382FFF783FF1649CE
:1046E000049A039B8C4208BF1346A289192159439F
:1046F00012B2002AB4BF7600B600B1FBF6F1642313
:10470000B1FBF3F21201100903FB1011A08900B2F2
:10471000002806DAC9003231B1FBF3F303F00703D6
:1047200005E009013231B1FBF3F303F00F031A4343
:1047300092B2228106B070BD0038014041719BE702
:10474000816099E7CB78F0B5DA0648BF8A780988A6
:1047500003F00F0548BF154311F0FF0F1DD004688B
:1047600000220127974007EA0106BE4211D19700B7
:104770004FF00F0C0CFA07FC05FA07F724EA0C04BB
:10478000282B44EA070401D1466102E0482B08BF08
:1047900006610132082AE4D10460FF291FD9446868
:1047A000002202F108060127B74007EA0106BE42CF
:1047B00011D197004FF00F0C0CFA07FC05FA07F720
:1047C00024EA0C04282B44EA070401D1466102E0E4
:1047D000482B08BF06610132082AE2D14460F0BDCF
:1047E00010B50446FDF7DDF8012806D11CB1FDF730
:1047F000D8F8013CF8E7052010BD002C08BF0520C3
:1048000010BD00BF000000002DE9F04F1421012869
:1048100034BF0646012601FB06F3DFF8D4A1DFF81A
:10482000BCB10AEB03025AF803301069CBF8003030
:10483000684B15891E70684BB2F80A80DC6989B034
:104840002043546848EA0507D861022227612046C0
:104850008DF80E1003A90193ADF80C708DF80F20A0
:10486000FDF7DEFF019B4FF008099B46A268154249
:1048700003D10A20FDF790FBF8E70A206561FDF7F8
:104880008BFB25610A20FDF787FBB9F10109EDD10A
:10489000C4F814800A20FDF77FFB65610A20FDF74C
:1048A0007BFB25610A20FDF777FB0222C4F810800C
:1048B00020468DF80F2003A91C228DF80E20ADF89C
:1048C0000C70FDF7ADFF454B454A1C689442DBF880
:1048D000102008D142F40012CBF81020DBF8102091
:1048E00022F4001207E042F48002CBF81020DBF83B
:1048F000102022F48002CBF81020A38803A823F410
:1049000040731B041B0CA38023889BB243F001035C
:104910002380A588FFF766FE25F03F050599314AFB
:104920002D04B1FBF2F22D0C1543ADB2A580238806
:10493000012523F001031B041B0C23802A4B03A831
:10494000B1FBF3F34FF496714A439BB24FF47A7183
:10495000002B92FBF1F208BF0123013292B243F423
:1049600000432284A38323889BB243F00103238066
:10497000238823F4816323F002031B041B0C238090
:104980004FF480432381142303FB06A6737B00248A
:104990008DF80C308DF80D408DF80E408DF80F50CD
:1049A000FDF7C2F8337B9DF80F208DF80C308DF8A1
:1049B0000D401AB103A8FDF7B7F807E0590903F055
:1049C0001F039D40094A203142F8215009B0BDE83B
:1049D000F08F00BF4C0A002000100240D00A0020D7
:1049E0000054004040420F00804F120000E100E000
:1049F000B8C7000808B5054B1A88013292B21A8070
:104A0000034B1878FFF700FF002008BDB404002016
:104A10004C0A002010B54000204CC0B22070204845
:104A2000012401701F49002008701F490C701F49A4
:104A30000B601F490B601F4B1F491A701F4B204A08
:104A40001B680C701070988810F4007F104615D108
:104A50001A88D2050DD447F230521C88A40502D51D
:104A6000013AFAD112E08AB11A8892B242F4807205
:104A70001A809A8892B242F440729A8047F2305378
:104A80000A7812B1013BFBD100E013B9BDE8104038
:104A9000B0E7007880F0010010BD00BFC00A002020
:104AA000C10A0020C20A0020C30A0020C80A002050
:104AB000C40A0020CC0A0020CD0A0020D00A002021
:104AC000CE0A0020244A13B513681446998A89B285
:104AD0000191019911F4706F02D0204A01211170E7
:104AE000019A12F4E06F2AD01A8B9A8822F480621D
:104AF0001204120C9A80019A910520D41A8892050A
:104B00001DD41A88D0050FD51A88D105FCD41A886F
:104B100092B242F400721A801A889205FCD4104BAB
:104B20001878FFF771FE0AE01A8892B242F4007218
:104B30001A809A8822F440721204120C9A80226819
:104B4000938A23F470631B041B0C9382054B002291
:104B50001A7002B010BD00BFD00A0020CE0A00209B
:104B60004C0A0020CD0A00202DE9F84FFEF71CFB6F
:104B700010B90A20FDF764FA894C4FF49862204678
:104B8000884905F0C1FC94F8BC344FF49472022BB0
:104B900084BF002384F8BC3494F8BC34824E02FBFA
:104BA000034303F5A2733360A36842F201021A4083
:104BB0003AB944F208021A401AB9794A43F4005348
:104BC0009360A368DB0703D54FF40050FDF7ECFDBD
:104BD000A3685F0409D50820FDF7E6FD4FF40050F7
:104BE000FDF7E2FD0120FDF7DFFDA3681D0706D5F7
:104BF0004FF40050FDF7D8FD0120FDF7D5FDA36867
:104C000098040ED54FF40040FDF7CEFD4FF4006040
:104C1000FDF7CAFD4FF48030FDF7C6FD4020FDF7DB
:104C2000C3FDA368590603D54FF48030FDF7BCFDE2
:104C30005E4B5F4D1D60FFF715FB5E4B05F11A02E1
:104C400001201A60FFF7AEFA01460120FEF76AFA6A
:104C5000002840D00220FFF7A5FA01460220FEF707
:104C600061FA002837D01020FFF79CFA0146102087
:104C7000FEF758FAA3681A0600D560B30820FFF7BC
:104C800091FA01460820FEF74DFAA3681B0700D5EC
:104C900008B30420FFF786FA01460420FEF742FA23
:104CA000A3685F0503D400231A46194609E00028CB
:104CB000F9D110E079B90121C00708D40C33182BC1
:104CC0000BD03D481844007A8507F5D5F2E701324C
:104CD000D2B2022AF2D901F075FD3568002395F8A9
:104CE000516095F8500003FB03F11939714301F647
:104CF000C4115943414340F6C41291FBF2F12F4ACB
:104D000022F813100133072BEDD195F8523095F8A6
:104D100053E0B4F8D070B4F8D2C0C3F1640B03EB25
:104D2000830858425FFA8BFB4FEA4808CEF16409CA
:104D3000C7EB0C0C80B2002286B231B2002904DC31
:104D4000002E14BF1E46012600E05E4601FB01FA5C
:104D500076430AFB0EFA9AFBF6F64E444E434FF0AA
:104D60000A0A96FBFAF6464436B206FB0CF64FF4F6
:104D70007A7196FBF1F612493E4456520232504483
:104D8000182A80B2D8D10F4A0F4B1A602A780F4BDD
:104D9000012A03D0022A1FD00D4A1EE00D4A1CE052
:104DA0000C0F002000F800081C020020F400002076
:104DB0001A100020B0040020100000206E03002014
:104DC0008E03002000100020380200207000002018
:104DD000B133000815360008394A3A4E1A6005F515
:104DE0008E737360384B00229A80384B384A05F531
:104DF0009271136005F1DC02B260A3F12202F2604D
:104E0000A3F128022C3332617361324A163BB3613D
:104E100005F593731160F361B4F8F00002F0F8FD4A
:104E20007062B4F8F20002F0F3FD95F8603006F11C
:104E3000200286F8203095F87C30B06286F8213068
:104E400094F82331B5F8D80086F82C30224B1A603C
:104E50002B1D336305F16C037363204B05F168026E
:104E60001A6002F0D9FD01461D4802F0DDFE02F095
:104E700043FA0FA3D3E9002302F092FA02F0C2FC36
:104E8000184B1860686E02F037FA0BA3D3E90023C1
:104E900002F086FA0B4602461349002002F0AAFBF4
:104EA00002F0B0FC114B1860BDE8F88FAFF3008042
:104EB0003B597E90A9E78140182D4454FB210940BD
:104EC0008D3700084C0A00206408002004100020E0
:104ED000A4020020F8040020D8020020340300209F
:104EE00000006144EC0400200000E03F24030020A7
:104EF00008B5FEF77BF9FFF737FEBDE808400F2045
:104F000014210122FDF75DB810B50446204605F0D6
:104F100045FB10F0FF0F07D10B4B0C4893F8BC1466
:104F2000BDE81040FDF7D3BC204605F08CFB0228FD
:104F300008D8054B064C83F8BC04FEF757F9FFF779
:104F400013FEE3E710BD00BF0C0F00203BD70008A5
:104F5000AADC00082DE9F04F6F4985B0044605F042
:104F6000E5FA6E49002820460CBF0126032605F00D
:104F7000DDFA002808BF0226F20740F1B280684837
:104F8000FDF7A5FC002001F093F9664F6648FDF798
:104F90009EFC6648FDF79BFC7A79654B654803EB00
:104FA0008203596AFDF793FC3869002102F01CFF67
:104FB00000285CD13C460546D4F8108000214046CC
:104FC00002F012FF00284ED101355B482946D4F883
:104FD00014B0D4F818A0D4F81C90FDF778FC404623
:104FE000002102F00BFF10B15448FDF770FC694638
:104FF0004046FFF75DF901465148FDF768FC584609
:10500000002102F0FBFE10B14C48FDF760FC694640
:105010005846FFF74DF901464948FDF758FC504600
:10502000002102F0EBFE10B14448FDF750FC694648
:105030005046FFF73DF901464148FDF748FC484618
:10504000002102F0DBFE10B13C48FDF740FC694650
:105050004846FFF72DF901463A48FDF738FC0C2D7C
:1050600004F11004A8D13848691CFDF730FC37481A
:10507000FDF72DFC364CD7F8088054F8041F19B101
:105080003448FDF724FCF8E70C46334B53F8245022
:1050900055B10123A34013EA080F03D02F48294636
:1050A000FDF715FC0134F0E72D48FDF710FC29460B
:1050B0007B1893F80E3104AA13442A4A8A5C013102
:1050C000082903F8102CF3D10023274869468DF8EE
:1050D0000830FDF7FCFB2548FDF7F9FB402001F007
:1050E0000FFDB30714D52248FDF7F1FB2148FDF76A
:1050F000EEFB2148FFF708FF2048FDF7E8FB1E48BC
:10510000FDF7DCFF1948FDF7E2FB802001F0F8FC19
:1051100005B0BDE8F08F00BF48D700084FD70008A2
:1051200057D700080C0F002065D7000877D7000874
:10513000B8C7000883D700088ED7000879DC0008BC
:105140008FDB0008E1DB000896D70008A8D700082D
:1051500038C80008B8D700083CC80008C6D70008FF
:10516000D3D70008E8DA0008DFD7000810DC000811
:10517000E8D70008FBD70008AADC000809D8000817
:1051800013B5062204466B463B216820FFF742FC1C
:105190009DF800209DF8013043EA022323809DF80A
:1051A00002209DF8033043EA022363809DF8042027
:1051B0009DF8053043EA0223A38002B010BD13B569
:1051C000062204466B4643216820FFF723FC9DF826
:1051D00000209DF8013043EA022323809DF802203D
:1051E0009DF8033043EA022363809DF804209DF874
:1051F000053043EA0223A38002B010BD2DE9F74F2A
:10520000A04AA1491368A14D03F59C4320330B60CC
:10521000AB68174613F4807F04D09D4B1B681B6856
:105220001B699847AB6842F201041C405CB9994E77
:10523000337873B1964B1B681B681B68984700F066
:105240000DFF347005E0944B1A7801321A7000F0AB
:1052500005FFAB68D80404D5904B1B780BB9FDF75C
:1052600042F98F4B3C681B681E7C86B18D4A013E1B
:1052700032F91600A0F57A70B0F57A7FA8BF4FF426
:105280007A7020EAE07002F0C7FB874934E0AB682F
:1052900019043AD5804A5368E31A002B35DB04F52C
:1052A0009C4320335360814B5979814B33F8110073
:1052B000137A80B2013303F00F031372D71802F090
:1052C000ABFB7C4902F0B0FC02F0E6FD334678729D
:1052D0003046794A9A5C01331044102B80B2F8D1E1
:1052E00000B290FBF3F000B26428A8BF642020EA6B
:1052F000E07002F091FB714902F096FC704902F0F7
:10530000DFFB02F0C9FD6F4B1880AB68DA0510D5E2
:105310006D4B9C426D4C08D923681B681B6A9847EB
:1053200018B923681B685B6A984723681B685B6928
:105330009847AA685B4F12F4805F544BB5F8DC10B5
:10534000B7F9062007D0B3F81831581A824207DDA2
:1053500019448A4202E0B3F81A319A42C0F26582D7
:1053600001225B480023D0F800A095F8219195F820
:105370002211B5F81A61B5F81CC11C468046F85ECA
:10538000A408B042C4BF64F07F04E4B202336045B5
:10539000B8BF44F04004082BF1D13F4E737EA342C6
:1053A00004D1B37EF92B03D8013300E00023B37698
:1053B000DAF880307476A3B1384B1B783BB182B9F0
:1053C000444B1B78DB070CD5FCF71CFE09E0414B76
:1053D0001B78580705D511B1FDF785F801E0002AC3
:1053E000FAD0B37E2C49142B40F09580394B19F13B
:1053F00000091B7818BF4FF0010903F0040303F004
:10540000FF0293B1DAF880301BB95F2C01D1FDF7B0
:105410006AF8B9F1000F7ED0DAF88030002B7AD12B
:105420007D2C78D1FDF75FF875E0572C0BD12A4B16
:105430004FF47A721A80294B1B6813F008036AD163
:10544000274A138067E0AB685B0712D55A2C10D14E
:10545000244B187818B11A700122234B4FE0CA7EF2
:10546000224B82F00102CA760AB1022247E00322EF
:1054700045E05D2C00F0AA815B2C00F0A9815E2C38
:105480003FD1A7E1E8130020EC0100200C0F002021
:10549000E8010020F0000020840A0020EC03002036
:1054A000F40000204A03002000007A44C0030020DA
:1054B000D0030020CDCC23428D0A00200000C8423A
:1054C00000C07F44CE040020404B4C0070080020F8
:1054D0001C020020F4130020F0130020F40100202F
:1054E00018030020CD020020CF020020CE020020B1
:1054F000A72C40F02B819C4B1A7842F004021A70C2
:1055000009E0DAF88030002B40F018816F2C40F071
:105510000F81FCF777FDD5F808C01CF0040F2FD0E1
:10552000F27E924B8AB1924A127856070DD5914A73
:10553000B7F90610B2F81A21914206DD1A7822B99D
:105540008D49322008808D49CA761B7C53B18C4B23
:105550001A782AB98B4A127812B9874A32211180F7
:1055600001220CE0874B1A7852B1814A127802F07E
:10557000040202F0FF011AB91970834B01221A705C
:10558000D8F80070814B002293F8018080371046D4
:1055900011461346434501DB00233BE0082BFBD0BB
:1055A0002BB19C0703D1043A1030D2B2C0B2784C70
:1055B00040F2A46904EB4304268954B21C44A6F2C9
:1055C000155A04EB440436B2BAF5C77FE4B204F1CD
:1055D000010B8CBF4FF0000A4FF0010A4E450AFA4A
:1055E0000BFAD4BF4FF000094FF0010904F1020B90
:1055F00009FA0BF94AEA090940F2135A5645CCBF99
:105600000026012606FA04F449EA04048440013322
:105610002143BFE757F82320544E11420CBF00220C
:1056200001229A550133152BF4D17378594F5A4CF6
:105630001BB13B6898070BD416E01CF4807F13D095
:10564000564B1B681B689B6898470028F1D10BE0FC
:10565000228812F001030DD1484942F00102CB61CA
:105660000B624D490A8006E0238823F00103238062
:10567000012300E00023B2788AB183B1238823F0AC
:10568000010203F0020392B29BB222805BB93B4954
:1056900042F00202CB610B623F4B1A8003E0238889
:1056A00023F00203238023883D4A13F0030F4FF4B5
:1056B000804114BF516111613A6812F00A0F22D083
:1056C00032794AB159070AD443F004032380354B99
:1056D0001A88354B1A8002E023F004032380737983
:1056E0003BB123885A0608D42B4A43F04003138069
:1056F00003E0238823F040032380B3791BB1294BB7
:105700001A882A4B1A80F37A1BB1238843F48073DA
:1057100002E0238823F4807323806B79082B02D066
:105720000E2B40F08E80238823F04003238088E0F6
:10573000B9F1000F02D07E2C3FF4EBAE972C7FF432
:10574000D7AE1B4B4FF4C8721A80E4E60023BB2C83
:10575000019301D1022303E0B72C2BD14FF6FE7346
:10576000ADF8063045E000BF02020020EC03002047
:10577000F41300200C0F0020B4020020840A002043
:10578000CC020020CD020020CF020020CC0400205B
:105790004A030020F4010020A60300207008002026
:1057A0000010014018030020D0040020A8030020AE
:1057B000A0020020BE2C01D1022304E0BD2C7FF406
:1057C000AAAE4FF6FE73ADF8043012E0012202E0FB
:1057D000022200E00322D4B2631E85F8BC34FDF738
:1057E00005FDFFF7C1F9022028212246FCF7E9FB5D
:1057F00091E6D8F80030BDF80410B3F85C200A44F4
:10580000A3F85C20BDF80610B3F85E200A44A3F8A4
:105810005E20FDF7EBFCFFF7A7F90F201421012212
:10582000FCF7CFFB0023B37675E6074B002200217F
:10583000DA611A625A629A62DA6219635963996389
:105840008FE503B0BDE8F08F840A002013B5224B2A
:10585000400002ACC0B283F83C0004F8012D83F88C
:105860003D100122002183F83E2083F83F1083F889
:10587000482083F84920DA6C83F84A1091881C6428
:1058800089055C6415D41188CC050DD447F23051DC
:105890001088800502D50139FAD113E091B1118841
:1058A00089B241F480711180918889B241F44071CC
:1058B000918047F2305293F8491011B1013AFAD170
:1058C00000E012B9FFF796F804E0034B93F84A00A2
:1058D00080F0010002B010BD840A002007B54FF42B
:1058E0000053ADF8043002238DF8073004238DF8FF
:1058F00006301C4B1C4A1B68934201D11B4803E035
:105900001B4A934203D11B4801A9FCF789FF6B2175
:1059100080226820FFF79AFF0520FCF748FB192139
:1059200000226820FFF792FF6B2103226820FFF717
:105930008DFF372102226820FFF788FF0E4B1A21C6
:105940001A786820FFF782FF1B2118226820FFF7D2
:105950007DFF1C2110226820FFF778FF03B05DF85F
:1059600004FB00BF2800002000127A00000C014058
:10597000001BB700001001403D00002037B5062293
:10598000044603216B461E20FFF744F89DF80130C2
:105990009DF80000154D43EA002000B202F03CF8EB
:1059A000296802F08DF802F051FA9DF8033020804A
:1059B0009DF8020043EA002000B202F02DF8A96829
:1059C00002F07EF802F042FA9DF80530A0809DF8C2
:1059D000040043EA002000B202F01EF8696802F0F9
:1059E0006FF802F033FA608003B030BD4000002051
:1059F00007B52320FCF7DBFA6820752101220DF1A1
:105A00000703FFF707F828B19DF80700B0F1680316
:105A10005842584103B05DF804FB00BF2DE9F04F38
:105A2000AE4E85B03778032F14D9AD4BAD48B3F9DE
:105A30000410B0F904200029B8BF49426FF0630395
:105A40005B1A9A4204DB01F164039342A8BF134638
:105A500083801FE0012F1DD8A34BA44C1B78013B72
:105A6000142B00F2DF81DFE813F09100DD01DD018E
:105A700068009F00DD01DD012F01DD01DD01DD0199
:105A8000DD01DD01BD00DD01DD01DD01DD01DD0147
:105A90009F01B601924B9649B3F806A0914B096855
:105AA000B3F80280B3F80090B3F904B0914C0291BE
:105AB0000025BD4204F11004CED20FFA8AF001F0A5
:105AC000ABFF54F8101C01F0FBFF03460FFA88F0FF
:105AD000019301F0A1FF54F8081C01F0F1FF019BB4
:105AE0000146184601F0E4FE03460FFA89F00193DF
:105AF00001F092FF54F80C1C01F0E2FF019B0146FB
:105B0000184601F0D5FE029A034692F9000001936F
:105B100040420BFB00F001F07FFF54F8041C01F041
:105B2000CFFF019B0146184601F0C2FE02F08EF93C
:105B3000714B23F815000135BBE702210420FCF767
:105B400067FB684D0121AF8878431FFA80F8042075
:105B5000FCF75EFB6D8800FB05801FFA80F80420CF
:105B6000FCF764FB4044208102210520FCF750FB38
:105B70007843012187B20520FCF74AFB00FB057042
:105B800087B20520FCF752FB38440BE005200121C9
:105B9000FCF73EFB534B9D88684385B20520FCF71C
:105BA00045FB284460813DE1544B00201D68FCF713
:105BB0003DFBDFF8608195F90630B8F90220322705
:105BC000534393FBF7F3184420800120FCF72EFB8E
:105BD00095F90E30B8F90020534393FBF7F738449A
:105BE00060801FE1464B1B7813F0040F454B02D138
:105BF0001B689B880BE01968394A0B88B2F90620AC
:105C000049889A4203DB9142B4BF0B461346E381B5
:105C1000E289394B394F1A803B4B1B681D7845B3DD
:105C20000220FCF703FB3A68B2F91030518A98421F
:105C300003DB0BB29842B8BF034634490968488970
:105C4000C3EB000E274B0FFA8EFED9880FFA81FCAA
:105C5000F44501DA0D4401E001DD4D1BDD8092F9D0
:105C60001620B3F906305343642293FBF2F3184431
:105C7000A080274B1B88D9050CD5194B1A88D7F85B
:105C80000090E28022819A88184F62815B88032508
:105C9000A38101E0134BF1E709EBC50393F906304B
:105CA000B7F90680284608FB03F8642398FBF3F84D
:105CB000A7F80680FCF7BAFA01354044072DF880B2
:105CC00007F10207E8D1ADE00D4B1B7813F0040F8C
:105CD0000C4B21D11B689B882AE000BFCC1300200D
:105CE0007C030020D40A0020F4040020600000207F
:105CF000F8040020A0070020CE130020540A002042
:105D0000F41300205C0A0020600A0020640A0020CE
:105D1000A6030020080300201968AD4A0B88B2F9D9
:105D2000062049889A4203DB9142B4BF0B461346D2
:105D3000E381E289A74BA84D1A80A84B03201B885A
:105D40000121DA0503D5FCF763FAA14F02E0FCF765
:105D50005FFAA34FB7F80280022100FB08F01FFA98
:105D600080F90320FCF754FA3F88012100FB0790DB
:105D7000E8800420FCF74CFA00FB08F002211FFA2F
:105D800080F80420FCF744FA00FB078028810320F8
:105D9000FCF74CFAE3881844E0800420FCF746FA4C
:105DA0002389184420813DE001210420FCF730FACA
:105DB0008B4D6F88784387B204202781FCF736FA31
:105DC0003844208101210520FCF722FA2D88684300
:105DD00085B26581E2E6824B0325B3F804909846CC
:105DE00028460221FCF714FA00FB09F0012187B2D2
:105DF0002846FCF70DFAC5F106035B0838F81330A6
:105E000000FB037087B224F815702846FCF70EFAE1
:105E1000384424F815000135072DE1D16C4BDA88A0
:105E20006C4B1A806F4DDFF8E491AB6813F0200FD4
:105E300033D00020FCF7FAF9208080460120FCF7DF
:105E4000F5F9694B644FDB79608033B3674B1B68AE
:105E50001B7813F0020F664B23D0D9F800C0B3F9BA
:105E600000109CF90E209CF906C0B3F902304A4399
:105E7000CCF1000C03FB0CF3322192FBF1F26FF03A
:105E8000310C92B293FBFCFC9444E04493FBF1F19F
:105E9000A7F800800A4410447880D9F80010002345
:105EA00019E0D9F80010B3F902C091F90620B3F94E
:105EB00000300CFB02FC32229CFBF2FCE044A7F811
:105EC000008091F90E104B4393FBF2F2E3E7E252AC
:105ED0000233102B0CD0E05E31F9232001EB830755
:105EE00090427F88F3DB3AB28242A8BF0246EEE7D7
:105EF0003E4B1B681B785B0704D43649347808880E
:105F000001231BE03B4B00241F780423043FFFB216
:105F10005FFA87F84FFA88F2D4420BD4364A03F17D
:105F20000109381932F813105FFA89F9C0B2FCF789
:105F30005DFC4B460134042CECD1DEE7A34208D2D1
:105F400031F9132000B28242A8BF104680B201335B
:105F5000F4E72A4B4FEA44081A68AB6803F480550B
:105F60000395254D03F01009254BB5F90660254D25
:105F70001B782F68244D03F00403DBB2D5F800C072
:105F800002930023434563D0B2F802A004B2544503
:105F900005DD104CC0EB0A0A1D5B55441D53039DE3
:105FA0000C4C002D34D07D8931F903A0AE42CBBF1B
:105FB000BCF802509588B2F802B0BCF800B0AA450F
:105FC00003DBDA45B4BF55465D46E55239E000BF14
:105FD0007C030020CE13002060000020A6030020D8
:105FE000D40A00200C0F0020EC030020680A0020D7
:105FF00008030020870600204A0300205C0A0020D6
:10600000F4130020640A0020580A0020540A0020DB
:1060100031F903A01588B2F802B0AA4503DBDA45CE
:10602000B4BF55465D46E55204EB030ABC89A6425F
:1060300007DAB9F1000F01D1148800E09488AAF8BA
:106040000040029C14B9044C1C5BCC52023399E70B
:1060500005B0BDE8F08F00BFD20400203F4A2DE913
:10606000F84F916840F201130B4040F201118B424E
:1060700093460AD13A4B1A7A93F809905A72B9EBBF
:10608000020918BF4FF0010901E04FF001094FF07C
:106090000008344B5FFA88F41B78A3425CD9324B7A
:1060A000324E1B68324F23B93B685B8926F81430A7
:1060B0004FE03A68072C94BF12F804A0A246294882
:1060C00051469847DBF808300546DB0509D5B9F19C
:1060D000000F06D0274B50461B6829461B68DB691A
:1060E0009847A5F2EE2240F2DC5392B29A4288BF62
:1060F0003B68DBF8082088BF5D8942F2010313404A
:106100002BB31D4B1978164B01F0030202EB8402EE
:1061100093F86A0003EB420255811A4620B903291D
:1061200015D9012183F86A1002EBC40399895D89AE
:1061300002EB44020D44D9891B8A0D441D44ADB2C3
:10614000A2F86C5004232DB295FBF3F5ADB226F8FE
:10615000145008F101089CE7BDE8F88F0C0F0020EF
:10616000D40A0020CC0400207C0800204A03002030
:10617000F4000020E8010020840A002013B5012269
:1061800004464FF6FF710068FDF75AFE236801A828
:106190001A8892B242F001021A80637B8DF80430B3
:1061A00001238DF805308DF806308DF80730FBF7A8
:1061B000BBFC02B010BD30B51249134A0C78134B2A
:1061C0009CB1D3F8844015680444A54218D31268E2
:1061D0000020C3F884200E4A0870117809B10139F3
:1061E0001170012283F8882030BDD3F88400146830
:1061F000C830844204D3126801200870C3F8842098
:1062000030BD00BF09040020080F0020D40A002080
:10621000CE02002037B5214D8DF8073095F8893032
:106220008DF8062002AA8DF804008DF805101A4496
:1062300012F8042C443AD2B20F2A09D81849022B7A
:1062400031F8124008D8A4B12046FFF7B4FF10E09F
:10625000022B4FF0C804F7D9124B1A68D5F88430D6
:10626000121B934205D20D4A002382F889300E4A50
:10627000137095F88830012B00D064B995F88930F7
:10628000022B03D8054A013382F88930074A0023DC
:1062900085F88830137003B030BD00BFD40A0020E9
:1062A00048C90008080F0020CE0200200904002081
:1062B000024B03481968034AFCF709BB7C00002025
:1062C000FADA000824DB0008234B70B519684FF494
:1062D0007A73B1FBF3F1214B21481A78214B224DFF
:1062E0001B78FCF7F4FA214B21481968214B2E68E2
:1062F000B1FBF3F1FCF7EBFA00241F4BE2B253F8C9
:10630000221049B1012303FA02F2324202D01B48A3
:10631000FCF7DDFA0134F0E72A6892070DD5184A38
:106320001848127803EB8203196AFCF7D0FA164B6F
:10633000197A11B11548FCF7CAFA1548FBF738FF6E
:10634000BDE87040134B14481A88144B92B2198858
:106350004FF49863FCF7BBBA080F0020B10300208C
:106360002CDB000874000020F401002078000020DD
:106370006ADB000840420F0068C90008ACD400087E
:10638000F513002088DB00088C02002092DB000857
:1063900010DC0008B404002096DB0008480300204D
:1063A00010B50748FBF704FF0024064B0648E21827
:1063B000E15852680C34FCF78AFAC02CF5D110BDB4
:1063C000C8DB000888C80008DEDB00082DE9F041C2
:1063D000002407462546114B3946E65804EB0308CE
:1063E000304604F017F958B10D483146FCF76FFA02
:1063F00040460021FCF746FB0A48FCF768FA0135E5
:10640000143440F6D4039C42E5D125B90648BDE8D2
:10641000F041FBF7CDBEBDE8F08100BFD0C9000858
:10642000CEDC000810DC0008E6DB00082DE9F74FA1
:10643000044604F0B3F8054620B1012819D12378A9
:106440002A2B16D15248FBF7B3FE0024514B524879
:10645000E618E158FCF73BFA30462946FCF712FBF8
:106460004E48FBF7A5FE143440F6D4039C42EDD110
:106470008AE020463D2104F084F800287FD00346BE
:1064800013F8012C202A01D1013BF9E7451C2846CD
:10649000C4EB030A04F0D7F883462846FCF766F8F5
:1064A0000026054614237343DFF8E89053F809707B
:1064B00003EB0908384604F071F803461A462046F3
:1064C0003946019304F072F8019B00284ED15FFA1F
:1064D0008AF29A424AD1D8F80C0001F09DFA01469E
:1064E000284601F09FFC00283ED0D8F8100001F0AB
:1064F00093FA0146284601F08BFC002834D098F826
:1065000004309C064FF0140303FB0696327958BF03
:106510005D4610062946B36806D521484FF49474A9
:1065200090F8BC0404FB003302F03F02042A0BD0B5
:1065300004D8013A012A0CD819700AE0102A05D0B3
:10654000202A05D0082A04D1198002E0196000E051
:106550001D6039461348FCF7BAF93046002103B0F4
:10656000BDE8F04FFCF78EBA0F4803E00136712EFC
:1065700098D10E4803B0BDE8F04FFBF719BE204696
:1065800003B0BDE8F04F21E703B0BDE8F08F00BFD6
:10659000FEDB0008D0C90008CEDC000810DC0008D3
:1065A0000C0F002013DC00081EDC0008E6DB0008EE
:1065B0002DE9F047744B86B01A789A46DFF8DC91E3
:1065C000BAB901238AF80030704BD9F80020596815
:1065D000914204D019690C33914218BF0023022163
:1065E00059726B4B6B481A60FBF7E2FD6A48FBF788
:1065F000DFFDD9F8000003685B689847002800F0C9
:10660000C080664B624C186803689B6898470928ED
:10661000014601D03F2850D14FF000086668604F16
:1066200045462EB15F483968324603F0BFFF10B9C6
:10663000B84605B93D465C4B0C379F42F1D3D5B106
:10664000D5F800E0D8F800C0636851481EF8037020
:106650001CF80310B9420ED15A1C41B92D2B06D893
:1066600042600344202702441F72117203E0234456
:106670001F726260E8E763680BB1454512D04B4872
:10668000FBF796FD454509D855F80C0BFBF790FD37
:10669000D9F800000921FBF7F1FCF3E73E48FBF7CE
:1066A00087FD002663689E42A3D23E4BD9F80000C6
:1066B000995DFBF7E3FC0136F4E7636833B904281E
:1066C0003BD104F10800FCF759FE5AE00C2801D137
:1066D000374889E70A2901D00D2949D13548FBF708
:1066E00067FD6368E21800231372227A232A17D009
:1066F0000493314B2B4E009303A8294910220C23FD
:10670000039603F0A4FF054638B1006803F046FF86
:106710000130AB683044984702E02848FBF748FD59
:1067200020480021302203F0F8FE002363609AF82D
:106730000030002B7FF45AAF23E00C28C8D07F290B
:1067400003D156E72F2B3FF654AFA1F12002D2B26E
:106750005E2A3FF64EAF13B920293FF44AAF5A1CC8
:106760006260D9F800001C442172FBF787FC40E707
:106770007F29E7D1013B6360002223441A7210484D
:1067800035E706B0BDE8F087F313002010000020C5
:10679000600B00203EDC000876DC0008800600204C
:1067A00088C80008680B002048C900087BDC000886
:1067B00080DC000810DC0008891900088BDC000868
:1067C000A7DC000810B500231249DAB2585C27286C
:1067D000084603D00133092BF6D11A460E4B83F835
:1067E00028210022845CD1B2102C03D00132092A66
:1067F000F8D111464FF4E132C3F82C21C3F830210F
:10680000C3F83421C3F83821522283F8291183F8C0
:106810003C2110BDF1DA00080C0F00202DE9F74FE4
:10682000A24AA34C106851686B4603C34FF49862A8
:106830000021DFF8A492204603F06FFE04F5A27356
:10684000C9F800304F23237003236371A3604FF412
:106850001673A4F8F030FA23A4F8F2302A23A4F82F
:10686000EE304FF4FA73A4F8F630202384F8F430B5
:106870006E2384F804312B2384F80531212384F816
:1068800006314FF4C873A4F8083140F24C43A4F821
:106890001A3140F26C73A4F81C31192384F82331A7
:1068A00040F27E43A4F8D03040F23A73A4F8D230DC
:1068B0004FF47A73A4F8D43040F27E53A4F8D63063
:1068C00040F2EA53A4F8D83040F2B45301273226FC
:1068D00040F2DC5BA4F8DA304FF47A53A4F8DC60C1
:1068E000A4F8DE30A4F8E06084F8EC70A4F818B1E5
:1068F00084F8227184F82571FFF764FF40F6AC53E9
:10690000A381D9F8003000251E21A573D97399738E
:106910000B211972142117225972197550211A76F8
:106920005A769977552264219A71D9772D220820B9
:1069300078211A74D8745A775973DA75DFF89CE1A4
:106940005C4A5D490E204FF0280898724FF00A0A01
:106950005A20DE71D872C3F824E01D7083F80480D9
:1069600083F805809D765D74DD769D741D7783F8D0
:1069700015A083F80C8083F821701A63D963196419
:106980004FF08241D9624FF07C5199634B495A6371
:106990001A674B4A59644B49C3F828E083F8500002
:1069A000DFF83CE141205A67474A996483F8510077
:1069B00059660420152183F8526083F86000C3F8FB
:1069C0004CE083F8545083F8555083F85650A3F8A0
:1069D00058B083F85350A3F85C50A3F85E50A3F866
:1069E0005A5083F8688083F8698083F86C109A673E
:1069F00083F87C703548FDF7BDFBD9F800604FF493
:106A00004873A6F8D830C82386F81D314FF4966332
:106A1000A6F81E3140F2D933A6F8203140F64303E0
:106A2000A6F8223186F8D45086F8D55086F8D6805C
:106A300086F8D77086F8DA5086F81CA133464FF4F2
:106A40007F72A3F8DC204FF4FA62A3F8DE2040F254
:106A5000DC52A3F8E0201DF80520013583F8E22080
:106A6000082D4FF0FF0283F8E32003F10803E6D17D
:106A7000012386F8243186F8253186F82631002353
:106A8000E21810330021C02B1161F9D131464FF4C7
:106A900094720F4803F038FD0E4831464FF494725B
:106AA00003B0BDE8F04F03F02FBD00BFB0C9000830
:106AB0000C0F00209A99193F8FC2753DCDCC4C3DEB
:106AC000F6287C3F0000A0403D0A773FABDC000881
:106AD00078110020A01200201C020020000020409D
:106AE0000000404008B50548FBF762FBFFF796FE43
:106AF000FCF77CFBBDE80840FDF7C2B8B4DC000839
:106B000070B5064600240B4BE5182A7916420AD0C8
:106B1000E1580948FBF7DBFE28460021FBF7B2FFEE
:106B20000648FBF745FB143440F6D4039C42EAD1F7
:106B300070BD00BFD0C90008CADC000810DC000826
:106B40002DE9F0411E46964B8CB098428846174678
:106B500053D1944C944BA2602360944B20656361A5
:106B600003F58073A3614FF48073E3602361904B5E
:106B7000B507A364E36403F5484303F154032363B7
:106B8000A3F11403D3F8D42F636342F48042C3F813
:106B9000D42FD3F8D02F42F00102C3F8D02F4FF0FA
:106BA00002038DF803304FF40073ADF800304FF05E
:106BB00018038DF8023003D57E486946FBF730FE96
:106BC0004FF48063ADF80030F4074FF048038DF8C0
:106BD000023003D577486946FBF722FE0E238DF875
:106BE000043001A801238DF805308DF806308DF8AA
:106BF00007306C4CFAF798FF4DE06F4B984240F02D
:106C0000CA806E4C684BA26023608023E3604023FF
:106C100023616B4B206563618033A361694BB007CF
:106C2000A364E36403F5E53303F5FE73DA6942F424
:106C30000032DA615A6942F001025A614FF00203F0
:106C40008DF803304FF00403ADF800304FF0180317
:106C50008DF8023003D557486946FBF7E1FD08235C
:106C6000ADF80030F1074FF048038DF8023003D53E
:106C700050486946FBF7D4FD26238DF804300222E4
:106C8000012301A88DF805308DF806208DF8073016
:106C9000FAF74AFF494C0025012384F84430256265
:106CA000E561A5626562C4F82C806671A760A57174
:106CB0002046FDF7E1FCE36CF20701934FF48053AB
:106CC0000A934FF080030295039504950595079567
:106CD000089509950B95069324D5206BD0B1E368F0
:106CE00004932023099363690293FAF7A6FE01A98E
:106CF000206BFAF784FE236B1A6842F001021A60D7
:106D0000226D918A89B241F0400191825B689BB209
:106D1000236407E0236D4FF6DF721A80DA6842F0D1
:106D20002002DA60A36C002501934FF480530A938C
:106D300080230693B307029503950495059507955F
:106D4000089509950B951ED5606BB8B1236904931E
:106D500010230393FAF771FE606B01A9FAF74FFE57
:106D6000636B1A6842F002021A605D605D60236D19
:106D70009A8A92B242F080029A8204E0236DDA6825
:106D800042F08002DA60236D20469A8992B242F482
:106D900000529A8100E000200CB0BDE8F08100BFF5
:106DA00000380140B40E0020B8C90008980B00203C
:106DB000043801400008014000440040600E0020FB
:106DC000980D0020044400402DE9F04F87B099460B
:106DD0000746884615469DF840B0FDF7E3F902AE38
:106DE0000446034600F1100E18685968324603C283
:106DF000083373451646F7D1237B0BB903950495E9
:106E0000384602A9FCF78EF9044608B9002031E0A3
:106E10004368586828B1384602A92246FAF7BAFFF3
:106E2000F2E7A36894F800A01E781EB9CDF800B070
:106E3000124804E0012E1DD11148CDF800B04B4698
:106E400041462A46FFF77CFE03460028DED00D4A65
:106E5000067102EB8A02C2F8C002626850600A48FA
:106E600042689A4204D002690C309A4218BF00204E
:106E70004772184607B0BDE8F08F00BF00380140E8
:106E800000440040980B0020100000200148FCF74F
:106E900013BF00BF000800400148FCF70DBF00BF52
:106EA000000400404FF08040FCF706BF0148FCF7AB
:106EB00003BF00BF002C014038B5194C236D1D885D
:106EC000ADB2AA0612D5E26A1AB1988880B290478C
:106ED0000CE09B88E2696169DBB28B54E269E3688C
:106EE0000132B2FBF3F103FB1123E3612B0616D54C
:106EF000A26A616A0A4B8A420CD09869196D805C5B
:106F00000132C0B288801969B2FBF1F001FB102296
:106F10009A6238BD1B6DDA6822F08002DA6038BDF3
:106F2000600E00200D4BD3F8A4201188090613D55C
:106F3000D96F986F81420BD0D86E405C0131C0B2DE
:106F400090805A6EB1FBF2F002FB1011D9677047C6
:106F5000D36823F08003D360704700BF600E002029
:106F60000B480C4B4FF400525A60D0F888204FF673
:106F7000FE7311680B401360826FC36F9A4202D098
:106F80005430FAF723BD012380F89830704700BFD2
:106F9000600E002000000240FDF794BDFDF792BD99
:106FA000FCF700BDFCF7FEBC0F4B1A6842F0010273
:106FB0001A6059680D4A0A405A601A6822F08472B1
:106FC00022F480321A601A6822F480221A605A6809
:106FD00022F4FE025A604FF41F029A60044B4FF0F5
:106FE00000629A60704700BF001002400000FFF886
:106FF00000ED00E0024B1A6801321A60704700BFD2
:10700000080F002008B5084BB3F8D80093F8C42443
:107010000023D9B2914204D2044921F8130001336C
:10702000F7E7FBF7D9F8FEE7080F0020CE130020A2
:1070300081F0004102E000BF83F0004330B54FEA29
:1070400041044FEA430594EA050F08BF90EA020F96
:107050001FBF54EA000C55EA020C7FEA645C7FEA29
:10706000655C00F0E2804FEA5454D4EB5555B8BF4C
:107070006D420CDD2C4480EA020281EA030382EABD
:10708000000083EA010180EA020281EA0303362D4F
:1070900088BF30BD11F0004F4FEA01314FF4801C22
:1070A0004CEA113102D0404261EB410113F0004F34
:1070B0004FEA03334CEA133302D0524263EB4303EB
:1070C00094EA050F00F0A780A4F10104D5F1200E89
:1070D0000DDB02FA0EFC22FA05F2801841F10001E4
:1070E00003FA0EF2801843FA05F359410EE0A5F1B8
:1070F00020050EF1200E012A03FA0EFC28BF4CF0E9
:10710000020C43FA05F3C01851EBE37101F000459E
:1071100007D54FF0000EDCF1000C7EEB00006EEBAB
:107120000101B1F5801F1BD3B1F5001F0CD3490835
:107130005FEA30004FEA3C0C04F101044FEA44528C
:1071400012F5800F80F09A80BCF1004F08BF5FEA13
:10715000500C50F1000041EB045141EA050130BDF3
:107160005FEA4C0C404141EB010111F4801FA4F196
:107170000104E9D191F0000F04BF01460020B1FAEB
:1071800081F308BF2033A3F10B03B3F120020CDA23
:107190000C3208DD02F1140CC2F10C0201FA0CF001
:1071A00021FA02F10CE002F11402D8BFC2F1200C66
:1071B00001FA02F120FA0CFCDCBF41EA0C0190401C
:1071C000E41AA2BF01EB0451294330BD6FEA040465
:1071D0001F3C1CDA0C340EDC04F11404C4F1200250
:1071E00020FA04F001FA02F340EA030021FA04F362
:1071F00045EA030130BDC4F10C04C4F1200220FAB9
:1072000002F001FA04F340EA0300294630BD21FAF6
:1072100004F0294630BD94F0000F83F4801306BFBC
:1072200081F480110134013D4EE77FEA645C18BFB0
:107230007FEA655C29D094EA050F08BF90EA020F47
:1072400005D054EA000C04BF1946104630BD91EA3F
:10725000030F1EBF0021002030BD5FEA545C05D142
:107260004000494128BF41F0004130BD14F5800481
:107270003CBF01F5801130BD01F0004545F0FE41F5
:1072800041F470014FF0000030BD7FEA645C1ABF2A
:10729000194610467FEA655C1CBF0B46024650EA61
:1072A000013406BF52EA033591EA030F41F400218D
:1072B00030BD00BF90F0000F04BF0021704730B513
:1072C0004FF4806404F132044FF000054FF00001E8
:1072D00050E700BF90F0000F04BF0021704730B5A9
:1072E0004FF4806404F1320410F0004548BF40427E
:1072F0004FF000013EE700BF42004FEAE2014FEAD3
:1073000031014FEA02701FBF12F07F4393F07F4FAD
:1073100081F06051704792F0000F14BF93F07F4FDF
:10732000704730B54FF4607401F0004521F0004122
:1073300020E700BF50EA010208BF704730B54FF0A8
:1073400000050AE050EA010208BF704730B511F0AD
:10735000004502D5404261EB41014FF4806404F1E5
:1073600032045FEA915C3FF4DCAE4FF003025FEA67
:10737000DC0C18BF03325FEADC0C18BF033202EBEF
:10738000DC02C2F1200300FA03FC20FA02F001FA49
:1073900003FE40EA0E0021FA02F11444C1E600BFE8
:1073A00070B54FF0FF0C4CF4E06C1CEA11541DBF9B
:1073B0001CEA135594EA0C0F95EA0C0F00F0DEF866
:1073C0002C4481EA030621EA4C5123EA4C5350EA4B
:1073D000013518BF52EA033541F4801143F480139C
:1073E00038D0A0FB02CE4FF00005E1FB02E506F02D
:1073F0000042E0FB03E54FF00006E1FB03569CF082
:10740000000F18BF4EF0010EA4F1FF04B6F5007F87
:1074100064F5407404D25FEA4E0E6D4146EB0606F9
:1074200042EAC62141EA55514FEAC52040EA5E5082
:107430004FEACE2EB4F1FD0C88BFBCF5E06F1ED82C
:10744000BEF1004F08BF5FEA500E50F1000041EB63
:10745000045170BD06F0004646EA010140EA020010
:1074600081EA0301B4EB5C04C2BFD4EB0C0541EA32
:10747000045170BD41F480114FF0000E013C00F347
:10748000AB8014F1360FDEBF002001F0004170BD6B
:10749000C4F10004203C35DA0C341BDC04F1140484
:1074A000C4F1200500FA05F320FA04F001FA05F210
:1074B00040EA020001F0004221F0004110EBD370DD
:1074C00021FA04F642EB06015EEA430E08BF20EA09
:1074D000D37070BDC4F10C04C4F1200500FA04F3AC
:1074E00020FA05F001FA04F240EA020001F000413E
:1074F00010EBD37041F100015EEA430E08BF20EAB1
:10750000D37070BDC4F1200500FA05F24EEA020EF8
:1075100020FA04F301FA05F243EA020321FA04F027
:1075200001F0004121FA04F220EA020000EBD370DE
:107530005EEA430E08BF20EAD37070BD94F0000FDE
:107540000FD101F00046400041EB010111F4801F12
:1075500008BF013CF7D041EA060195F0000F18BFC3
:10756000704703F00046520043EB030313F4801FFF
:1075700008BF013DF7D043EA0603704794EA0C0FB9
:107580000CEA135518BF95EA0C0F0CD050EA4106CF
:1075900018BF52EA4306D1D181EA030101F000414C
:1075A0004FF0000070BD50EA410606BF1046194674
:1075B00052EA430619D094EA0C0F02D150EA013680
:1075C00013D195EA0C0F05D152EA03361CBF1046C1
:1075D00019460AD181EA030101F0004141F0FE4160
:1075E00041F470014FF0000070BD41F0FE4141F4E4
:1075F000780170BD70B54FF0FF0C4CF4E06C1CEAE4
:1076000011541DBF1CEA135594EA0C0F95EA0C0F98
:1076100000F0A7F8A4EB050481EA030E52EA033553
:107620004FEA013100F088804FEA03334FF0805574
:1076300045EA131343EA12634FEA022245EA1115A1
:1076400045EA10654FEA00260EF000419D4208BF52
:10765000964244F1FD0404F5407402D25B084FEAFF
:107660003202B61A65EB03055B084FEA32024FF4AB
:1076700080104FF4002CB6EB020E75EB030E22BF08
:10768000B61A754640EA0C005B084FEA3202B6EBC8
:10769000020E75EB030E22BFB61A754640EA5C0077
:1076A0005B084FEA3202B6EB020E75EB030E22BF07
:1076B000B61A754640EA9C005B084FEA3202B6EB08
:1076C000020E75EB030E22BFB61A754640EADC00C7
:1076D00055EA060E18D04FEA051545EA16754FEA29
:1076E00006164FEAC30343EA52734FEAC2025FEA47
:1076F0001C1CC0D111F4801F0BD141EA00014FF0D6
:1077000000004FF0004CB6E711F4801F04BF0143A6
:107710000020B4F1FD0C88BFBCF5E06F3FF6AFAEC2
:10772000B5EB030C04BFB6EB020C5FEA500C50F152
:10773000000041EB045170BD0EF0004E4EEA1131D5
:1077400014EB5C04C2BFD4EB0C0541EA045170BDDC
:1077500041F480114FF0000E013C90E645EA060E20
:107760008DE60CEA135594EA0C0F08BF95EA0C0F4E
:107770003FF43BAF94EA0C0F0AD150EA01347FF496
:1077800034AF95EA0C0F7FF425AF104619462CE76D
:1077900095EA0C0F06D152EA03353FF4FDAE1046D0
:1077A000194622E750EA410618BF52EA43067FF421
:1077B000C5AE50EA41047FF40DAF52EA43057FF4B1
:1077C000EBAE12E74A0011D212F5001211D20DD51C
:1077D0006FF47873B3EB62520ED44FEAC12343F0D7
:1077E000004343EA505323FA02F070474FF0000081
:1077F000704750EA013002D14FF0FF3070474FF030
:10780000000070474FEA4102B2F1E04324BFB3F5F4
:10781000001CDCF1FE5C0DD901F0004C4FEAC00207
:107820004CEA5070B2F1004F40EB830008BF20F0EB
:107830000100704711F0804F21D113F13872BCBFA5
:1078400001F00040704741F480114FEA5252C2F1FA
:107850001802C2F1200C10FA0CF320FA02F018BF43
:1078600040F001004FEAC1234FEAD32303FA0CFC96
:1078700040EA0C0023FA02F34FEA4303CCE77FEA25
:10788000625307D150EA01331EBF4FF0FE4040F46F
:107890004000704701F0004040F0FE4040F400001E
:1078A000704700BF80F0004002E000BF81F000415F
:1078B00042001FBF5FEA410392EA030F7FEA226C96
:1078C0007FEA236C6AD04FEA1262D2EB1363C1BF26
:1078D000D218414048404140B8BF5B42192B88BF95
:1078E000704710F0004F40F4000020F07F4018BFB8
:1078F000404211F0004F41F4000121F07F4118BFD8
:10790000494292EA030F3FD0A2F1010241FA03FC7F
:1079100010EB0C00C3F1200301FA03F100F0004367
:1079200002D5494260EB4000B0F5000F13D3B0F12F
:10793000807F06D340084FEA310102F10102FE2A9E
:1079400051D2B1F1004F40EBC25008BF20F001000E
:1079500040EA03007047490040EB000010F4000FBC
:10796000A2F10102EDD1B0FA80FCACF1080CB2EB4F
:107970000C0200FA0CF0AABF00EBC25052421843AE
:10798000BCBFD0401843704792F0000F81F4000153
:1079900006BF80F400000132013BB5E74FEA410326
:1079A0007FEA226C18BF7FEA236C21D092EA030F92
:1079B00004D092F0000F08BF0846704790EA010F0C
:1079C0001CBF0020704712F07F4F04D1400028BF39
:1079D00040F00040704712F100723CBF00F500001B
:1079E000704700F0004343F0FE4040F40000704751
:1079F0007FEA226216BF08467FEA236301464202FD
:107A000006BF5FEA412390EA010F40F4800070470F
:107A10004FF0000304E000BF10F0004348BF4042B5
:107A20005FEA000C08BF704743F0964301464FF0F1
:107A300000001CE050EA010208BF70474FF000034D
:107A40000AE000BF50EA010208BF704711F000438E
:107A500002D5404261EB41015FEA010C02BF84465E
:107A60000146002043F0B64308BFA3F18053A3F5BD
:107A70000003BCFA8CF2083AA3EBC25310DB01FA04
:107A800002FC634400FA02FCC2F12002BCF1004F88
:107A900020FA02F243EB020008BF20F00100704719
:107AA00002F1200201FA02FCC2F1200250EA4C006D
:107AB00021FA02F243EB020008BF20EADC707047B3
:107AC0004FF0FF0C1CEAD0521EBF1CEAD15392EAC1
:107AD0000C0F93EA0C0F6FD01A4480EA010C40029D
:107AE00018BF5FEA41211ED04FF0006343EA5010F7
:107AF00043EA5111A0FB01310CF00040B1F5000F39
:107B00003EBF490041EAD3715B0040EA010062F1E7
:107B10007F02FD2A1DD8B3F1004F40EBC25008BFD1
:107B200020F00100704790F0000F0CF0004C08BFEF
:107B300049024CEA502040EA51207F3AC2BFD2F1BC
:107B4000FF0340EAC250704740F400004FF00003CA
:107B5000013A5DDC12F1190FDCBF00F00040704704
:107B6000C2F10002410021FA02F1C2F1200200FA42
:107B700002FC5FEA310040F1000053EA4C0308BF09
:107B800020EADC70704792F0000F00F0004C02BF5A
:107B9000400010F4000F013AF9D040EA0C0093F0D5
:107BA000000F01F0004C02BF490011F4000F013B2F
:107BB000F9D041EA0C018FE70CEAD15392EA0C0F9D
:107BC00018BF93EA0C0F0AD030F0004C18BF31F008
:107BD000004CD8D180EA010000F00040704790F0DE
:107BE000000F17BF90F0004F084691F0000F91F082
:107BF000004F14D092EA0C0F01D142020FD193EA48
:107C00000C0F03D14B0218BF084608D180EA0100CF
:107C100000F0004040F0FE4040F40000704740F0AB
:107C2000FE4040F4400070474FF0FF0C1CEAD05279
:107C30001EBF1CEAD15392EA0C0F93EA0C0F69D0D5
:107C4000A2EB030280EA010C49024FEA402037D040
:107C50004FF0805343EA111143EA10130CF0004037
:107C60008B4238BF5B0042F17D024FF4000C8B4227
:107C700024BF5B1A40EA0C00B3EB510F24BFA3EB07
:107C8000510340EA5C00B3EB910F24BFA3EB9103D7
:107C900040EA9C00B3EBD10F24BFA3EBD10340EA31
:107CA000DC001B0118BF5FEA1C1CE0D1FD2A3FF677
:107CB00050AF8B4240EBC25008BF20F0010070472C
:107CC0000CF0004C4CEA50207F32C2BFD2F1FF03CF
:107CD00040EAC250704740F400004FF00003013A00
:107CE00037E792F0000F00F0004C02BF400010F4A4
:107CF000000F013AF9D040EA0C0093F0000F01F0B8
:107D0000004C02BF490011F4000F013BF9D041EAD9
:107D10000C0195E70CEAD15392EA0C0F08D142020C
:107D20007FF47DAF93EA0C0F7FF470AF084676E7DF
:107D300093EA0C0F04D14B023FF44CAF08466EE7B8
:107D400030F0004C18BF31F0004CCAD130F0004286
:107D50007FF45CAF31F000437FF43CAF5FE700BFDE
:107D60004FF0FF3C06E000BF4FF0010C02E000BF07
:107D70004FF0010C4DF804CD4FEA40024FEA4103A9
:107D80007FEA226C18BF7FEA236C11D001B052EA5F
:107D9000530C18BF90EA010F58BFB2EB030088BF25
:107DA000C81738BF6FEAE17018BF40F00100704794
:107DB0007FEA226C02D15FEA402C05D17FEA236C76
:107DC000E4D15FEA412CE1D05DF8040B704700BFBD
:107DD000844608466146FFE70FB5FFF7C9FF002854
:107DE00048BF10F1000F0FBD4DF808EDFFF7F4FF8D
:107DF0000CBF012000205DF808FB00BF4DF808ED26
:107E0000FFF7EAFF34BF012000205DF808FB00BF48
:107E10004DF808EDFFF7E0FF94BF012000205DF86A
:107E200008FB00BF4DF808EDFFF7D2FF94BF01201B
:107E300000205DF808FB00BF4DF808EDFFF7C8FF14
:107E400034BF012000205DF808FB00BF4FEA40026C
:107E5000B2F1FE4F0FD34FF09E03B3EB12620DD978
:107E60004FEA002343F0004310F0004F23FA02F0E2
:107E700018BF404270474FF00000704712F1610F89
:107E800001D1420205D110F0004008BF6FF0004060
:107E900070474FF00000704742000ED2B2F1FE4F23
:107EA0000BD34FF09E03B3EB126209D44FEA0023C9
:107EB00043F0004323FA02F070474FF00000704790
:107EC00012F1610F01D1420202D14FF0FF30704731
:107ED0004FF00000704700BF73B96AB9002908BFAE
:107EE0000028BCBF00204FF00041C4BF6FF000412C
:107EF0004FF0FF3000F03CB882B0EC462DE9005066
:107F000000F006F8DDF804E002B00CBC704700BFDA
:107F10002DE9704F089E14461D468046894600F0A4
:107F200029F804FB01F3A4FB00AB00FB05329344EA
:107F3000B8EB0A0869EB0B09C6E90089BDE8708F48
:107F40002DE9704F089E14461D468046894600F074
:107F500061F900FB05F5A0FB04AB04FB0154A3444D
:107F6000B8EB0A0869EB0B09C6E90089BDE8708F18
:107F7000704700BF00292DE9F00FC0F2A180002456
:107F8000002BC0F29880154606460F46002B3FD1C5
:107F90008A4258D9B2FA82F34BB1C3F1200201FAF6
:107FA00003F720FA02F29D4000FA03F61743290C6A
:107FB000B7FBF1F201FB1277A8B200FB02F34FEA24
:107FC000164C4CEA0747BB4209D97F1902F1FF3C26
:107FD00080F00581BB4240F20281023A2F44FF1A31
:107FE000B7FBF1F301FB137100FB03F0B6B246EAF5
:107FF0000141884208D9491903F1FF3780F0F18027
:10800000884240F2EE80023B43EA0242002303E052
:108010008B420AD900231A461046194614B1404231
:1080200061EB4101BDE8F00F7047B3FA83F8B8F196
:10803000000F40F088808B4202D3824200F2E2803F
:1080400000230122E8E712B90123B3FBF2F5B5FAE8
:1080500085F2002A3AD17F1B280C1FFA85FC0123E8
:10806000B7FBF0F100FB11770CFB01F24FEA164869
:1080700048EA0747BA4207D97F1901F1FF3802D20F
:10808000BA4200F2C4804146BF1AB7FBF0F200FBCF
:1080900012700CFB02FCB6B246EA0040844507D9D8
:1080A000401902F1FF3702D2844500F2AE803A4611
:1080B00042EA0142B0E7E443524263EB430362E722
:1080C000404261EB41014FF0FF3459E79540C2F166
:1080D000200927FA09F126FA09F99740280CB1FB83
:1080E000F0F800FB18111FFA85FC0CFB08F349EAB5
:1080F00007094FEA194747EA01418B4206FA02F69F
:1081000008D9491908F1FF327AD28B4278D9A8F1FF
:1081100002082944C91AB1FBF0F300FB13170CFB4A
:1081200003F21FFA89F949EA0747BA4207D97F19CA
:1081300003F1FF3160D2BA425ED9023B2F44BF1A2D
:1081400043EA08438CE7C8F1200225FA02F103FA5A
:1081500008FC27FA02F320FA02F207FA08F741EACC
:108160000C0C4FEA1C49B3FBF9F109FB11331FFA60
:108170008CFA0AFB01FB17433A0C42EA03439B4586
:1081800005FA08F008D913EB0C0301F1FF3235D2E0
:108190009B4533D902396344CBEB0303B3FBF9F2BC
:1081A00009FB12330AFB02FABFB247EA0347BA459A
:1081B00008D917EB0C0702F1FF331BD2BA4519D9C6
:1081C000023A674442EA0145A5FB0001CAEB0707F2
:1081D0008F424FF000030AD305D02A461CE76246BF
:1081E000FDE63B4610E706FA08F68642F5D26A1E1F
:1081F000002311E71A46E5E70B46A0E71146CBE757
:10820000904687E74346424606E7023A50E702397E
:108210002F4439E72DE9F00F144605460E46002B92
:1082200043D18A4253D9B2FA82F757B1C7F1200637
:1082300020FA06F601FA07F302FA07F400FA07F546
:108240001E43210CB6FBF1F201FB1266A0B200FB4B
:1082500002F32F0C47EA0646B34209D9361902F158
:10826000FF3780F0FD80B34240F2FA80023A2644A4
:10827000F61AB6FBF1F301FB136100FB03F0ADB29C
:1082800045EA0141884208D9091903F1FF3680F017
:10829000E980884240F2E680023B43EA0242002342
:1082A00010461946BDE8F00F70478B424CD8B3FA20
:1082B00083F6002E4FD18B4202D3824200F2DD8042
:1082C000BDE8F00F0023012210461946704712B98D
:1082D0000124B4FBF2F4B4FA84F2002A40F0828064
:1082E000091B260CA7B20123B1FBF6F006FB101107
:1082F00007FB00F24FEA154C4CEA01418A4207D9CC
:10830000091900F1FF3C02D28A4200F2C88060469F
:10831000891AB1FBF6F206FB121107FB02F7ADB2A8
:1083200045EA0145AF4208D92C1902F1FF3180F02E
:108330009B80A74240F29880023A42EA00421046EF
:108340001946BDE8F00F704700231A46104619463B
:10835000BDE8F00F7047C6F1200522FA05F703FAD1
:1083600006F421FA05F301FA06FB20FA05F53C4371
:108370004FEA1448B3FBF8FC08FB1C331FFA84F9DE
:1083800009FB0CFA45EA0B0B4FEA1B4545EA034390
:108390009A4502FA06F204D91B190CF1FF356FD386
:1083A000AC46CAEB0303B3FBF8F508FB153309FB36
:1083B00005F91FFA8BFB4BEA0347B94504D93F196E
:1083C00005F1FF3362D31D4645EA0C4CACFB02239A
:1083D000C9EB07079F424FF000054AD346D06246DB
:1083E0002B465DE79440C2F1200921FA09FC914037
:1083F00020FA09F9260CBCFBF6F806FB18CCA7B24C
:1084000007FB08F349EA01094FEA194141EA0C4C1C
:10841000634500FA02F509D91CEB040C08F1FF32A0
:108420003BD2634539D9A8F10208A444C3EB0C0C34
:10843000BCFBF6F306FB13C107FB03F21FFA89F935
:1084400049EA01418A4207D9091903F1FF3022D2D2
:108450008A4220D9023B2144891A43EA084343E770
:108460003A4605E7334618E70A4666E7B0409042C9
:10847000B5D20CF1FF32002312E7334632460FE744
:108480009A458DD9ACF1020C23448AE7B9459AD9B3
:10849000023D274498E70346DEE79046C6E70238E8
:1084A000214435E71C481D49026800608A4200F0FB
:1084B0001D80002100F004B8194B5B584350043173
:1084C0001848194B42189A42FFF4F6AF174A00F0C9
:1084D00003B8002342F8043B154B9A42FFF4F9AF6E
:1084E000FEF762FD00F038F8FFF7FEBF114E1248AC
:1084F00030601248016821F0706101604102016042
:108500000F4C182020600F490F4808600F48D0F822
:1085100000D0406800470000F04F0020EFBEADDE05
:1085200010E8000800000020EC000020F00000200F
:108530000814002018100240090000000400014047
:10854000140C0140000C01404434434400F0FF1F70
:10855000FFF7FEBF000000002DE9804891B0F7F75B
:10856000D7FD834E834CD6F80880002318F0080FFF
:108570002370374600F0CA8063681B7A042B00F230
:10858000C380DFE803F00303056D9400237ABCE0A9
:10859000627A784B002A00F0B78000225A7293F872
:1085A0002020100700F1B080D97A9A7A01F00700F4
:1085B00042EA00225A621A7B02F03F00400140EA80
:1085C000D1019962597B890041EA92119A7B02F0AC
:1085D000010041EA8021D962D97B01F00F00C0017E
:1085E00040EA52021A631A7C02F07F00000140EA5E
:1085F00011115963597C490041EAD212997C01F06A
:10860000030042EA40229A63DA7C02F01F008001F4
:1086100040EA9101D963197DC90041EA5212997D5E
:108620001A645A7D01F0070042EA00225A64DA7D9A
:1086300002F03F00400140EAD1019964197E8900AF
:1086400041EA92115A7E02F0010041EA8021D96488
:10865000997E01F00F01C90141EA52021A6551E009
:1086600094F85420434B002A4ED0002283F8542023
:1086700093F85620012A47D193F87A20102A84BF14
:10868000102283F87A2094F87A103B4A0023D8B25B
:10869000884202F1020235D212F8010C12F8025C93
:1086A00040EA0525354840F823500133EFE794F8B8
:1086B000BC20304B42B3002283F8BC2093F8BD208D
:1086C000A82A21D193F8D050F5B92A4901EB4503E6
:1086D00093F8C00093F8C13003EB0020FEF7EAFDE9
:1086E0001FA3D3E90023FEF785FF1FA3D3E90023CF
:1086F000FEF7A2FCFFF766F8214B43F82500013591
:10870000082DE2D1012300E00023237018F4804FEC
:1087100008D094F8F43023B1164B002283F8F420EB
:1087200001232370237843B118F4807F05D0114BC7
:10873000D3F8F8301B681B689847DFF84880227828
:10874000D8F8003032B90B4AD2F8FC209A1AD2433A
:10875000D20F00E00122BAB1FCF750FDB3E000BF38
:108760009A999999999919400000000000707740F2
:108770000C0F0020F0000020480100206C010020B8
:10878000C4010020E8130020D4F800A1A64D0AF18E
:108790000101C4F80011BAF1000F40F09080D5F843
:1087A0000421110740F18F80D5F808219A1A002A78
:1087B000C0F2898003F5C33905F5867009F1A00977
:1087C000C5F80891FDF7DAF8984B05F58670014673
:1087D0001A78F9F7CFF995F8120105F5867110F0BE
:1087E000040F17D0C5F814915346FA180025A2F8C3
:1087F000FE508D4ACD5A02F58C7E23F80E5002F5BC
:108800008F7E23F80E500233062BEED120F00400A9
:1088100082F8120194F82421834BA2B1B3F80C0121
:10882000B6F8FE20821AA3F80C21B3F80E01B6F8B0
:108830000021821AA3F80E21B3F81001B6F8022124
:10884000821AA3F81021D4F81431774A002B3AD0B9
:108850007748C3EB0909814502F58C7502F58F70E5
:1088600019D8744BDA6882F40052DA600023CA5ACD
:1088700035F903E017B2BE45C4BFDFF8CCE123F8F9
:108880000E2030F903E0BE45BCBF6B4FDA53023314
:10889000062BECD117E00023C2F8143135F903E0C0
:1088A000C15EFA1871444FF0020E734491FBFEF161
:1088B000062BA2F8FE10F1D1FCF71AFB03E0022907
:1088C000C8BFC5F80021F9F799FAB389C8F80000C4
:1088D0002BB1D4F82821821A002AFFF642AE524F5B
:1088E000184496F80580D4F83431C4F8280107F507
:1088F000A070D4F82C51CDF81080984707F5A070DF
:10890000014694F84621F9F735F94C4B1B88002BAA
:1089100000F0B980D7F848314FF000081B7807F510
:10892000A67903934746454A1288B2F57A7F0292A8
:10893000434A04D1002142F80810C9F810104149F7
:10894000C85F52F80810014442F80810FFF764F8B5
:10895000D9F8102083460132012AC9F8102007D126
:108960000022C9F80400C9F80000C9F808202CE06A
:10897000D9F800C061468DE80410FEF797FF009A11
:1089800082461046FFF748F801465046FFF74CF97B
:10899000DDF804C001466046FEF78AFF0246114634
:1089A000C9F8040058460092FEF780FF0146504681
:1089B000FFF786F8D9F80810FEF77AFF009AC9F891
:1089C0000C00C9F80020C9F808001E49029B0022CB
:1089D00001F1540B012B7A5227F80B20DFF85CA031
:1089E00044D1D9F81000012808DD0138FFF714F848
:1089F0000146D9F80C00FFF717F900E0002002F05B
:108A0000BFF8039B02460BB318460092FFF704F829
:108A1000009A01461046FFF70FFAB8B14FF47A7387
:108A2000AAF800302FE000BFF0000020F213002071
:108A30007FC3C901001001400E020020F013002086
:108A4000780200203002002008020020B54A4FF4CE
:108A50007A7158F802200A2002F5FA7292FBF1F2BC
:108A60002BF807200F210122F9F7ABFA0237062F66
:108A700008F1040809F114097FF455AF029F07F1CA
:108A8000FF39AAF800900023A74F07F5A07207F559
:108A9000CA71985A595A411A99520233062BF3D186
:108AA000D7F8043113F0020300F02083D7F8A03187
:108AB00007F5D470984707F5D470014697F8AE21B2
:108AC000F9F758F8B7F8B03107F5D478002B45D04E
:108AD0000022D7F8B4011346934F38F902C0B7F813
:108AE000B01107F5DC7EB1F5C87F04BF00214EF858
:108AF00003105EF803108C4F61444EF803100433EA
:108B000000210C2B28F80210815202F10202E3D15D
:108B1000B7F8B031012B1CD1D7F8B8314FF4C87277
:108B2000C83393FBF2F30380D7F8BC31C83393FB0F
:108B3000F2F34380D7F8C031C83393FBF2F27B4B9A
:108B40001B88D21A8280A5F85C10A5F85E10FCF78D
:108B5000CFF9B4F8B031013BA4F8B031B3685A078B
:108B600079D5B4F8C421704B322A13D1D3F8B4218B
:108B70001188A3F8C61151889288A3F8C811A3F8E8
:108B8000CA21B5F85C20A3F8CC21B5F85E20A3F883
:108B9000CE2101E0002A3CD00021D4F8B4610A467D
:108BA000614838F901E0B0F8C43100F5E877322BBC
:108BB00004BF0023BB50B8585B4B7044B85004321C
:108BC00000200C2A28F80100705201F10201E7D1BF
:108BD000B3F8C421012A17D183F8DD21022283F8DA
:108BE000DE21B3F8C62183F8DC013280B3F8C82156
:108BF0007280B3F8CA21B280B3F8CC21B3F8CE3179
:108C0000A5F85C20A5F85E30B4F8C431013BA4F8A7
:108C1000C43194F8DF21444BEAB1D3F8D061D3F8E2
:108C2000B4113220002296FBF0F683F8DF210E808B
:108C3000D3F8D46196FBF0F64E80D3F8D83193FB8D
:108C4000F0F03A4B1B88C01A8880A5F85C20A5F884
:108C50005E20FCF74DF9D4F8B431B4F8A8111A88A5
:108C600000268A1AA4F8A821B4F8AA115A88B14695
:108C70008A1AA4F8AA219B88B4F8AC21D31AA4F8C4
:108C8000AC31F9F7BBF8D4F8E0310546C31A184601
:108C90000293FEF7BDFED4F8E4110390FEF710FF37
:108CA000D4F8E881C4F8E05198F800A00590354662
:108CB0001F4F785FFEF7B0FE0599FEF701FF07A989
:108CC0008851BAF1000F35D05046FEF7A5FE014697
:108CD0004FF07E50FEF7A8FF0246114607F1AC0B9D
:108CE0004FF07E500092FEF7E1FD56F80B10FEF7B4
:108CF000E7FE07F168018446485FCDF804C0FEF73F
:108D00008BFE009AB8371146FEF7DAFEDDF804C094
:108D100001466046FEF7CCFD4BF80600FFF796F8DB
:108D200078530CE078020020F000002000000020C2
:108D30003002002007F1B8026837E95BA952BA4F48
:108D40000436EA5F0235062D02FB0299B0D1B74D19
:108D50004FF0640A2A880AFB09F3524393FBF2FAA4
:108D6000AAF1490A07F1080007A91FFA8AFAF9F7D8
:108D700079FABAF13B0FD8F8046010D9B4F90C02B3
:108D8000FEF74AFED4F8086201463046FFF754F871
:108D9000A74F94F8123168B343F008032CE04FF06A
:108DA0007E513046FEF784FD01464FF07E50FEF7BF
:108DB0003BFF4FF0000B82469E4B304653F81B1092
:108DC0000193FEF77DFE024637F90B000092FEF795
:108DD00023FE009A01461046FEF76AFD5146FEF753
:108DE0006FFE019B43F81B000BF1020BBBF1060F5A
:108DF000E2D1C3E723F008033146D4F8040287F830
:108E0000123101F0BBFE0746C4F81002D4F800028C
:108E1000D4F808B200F10046D4F804020146FEF787
:108E20004FFE594682465846FEF74AFE01465046D6
:108E3000FEF73EFD01F0A4FE0146304601F09EFE25
:108E40000646C4F814023846FEF756FA72A3D3E970
:108E50000023FEF7A5FAFEF7D5FC01F0C3FDA4F848
:108E600018023046FEF748FA6BA3D3E90023FEF759
:108E700097FAFEF7C7FC01F0B5FDD4F80431A4F869
:108E80001A021B0739D56C4807A9F9F7EBF9D8F88E
:108E900008904FF07E514846FEF70AFD01464FF01C
:108EA0007E50FEF7C1FE4FF0000B8246604D4846F3
:108EB00005F5077353F81B100193FEF701FE05F546
:108EC0008671024631F90B000092FEF7A5FD009A6B
:108ED00001461046FEF7ECFC5146FEF7F1FD019B02
:108EE00043F81B000BF1020BBBF1060FDED1184655
:108EF000F9F770FAA5F8280241E0DFF830A107A9D8
:108F00000AF10400F9F7AEF96868D5F808B001462F
:108F1000FEF7D6FDD5F80C90594605465846FEF7A3
:108F2000CFFD01462846FEF7C3FC494605464846A4
:108F3000FEF7C6FD01462846FEF7BAFC01F020FE0A
:108F400000210546FEF750FFA0B9DAF804002946D3
:108F5000FEF76AFE2946CAF80400DAF80800FEF7B0
:108F600063FE2946CAF80800DAF80C00FEF75CFE3A
:108F7000CAF80C003148F9F72DFAA4F82802304954
:108F80000398FEF79DFD07F10047814606F1004674
:108F9000B4F928020A970B96FEF73EFD00F1004057
:108FA000FEF7AAF91EA3D3E90023FEF7F9F9FEF7AD
:108FB00029FC0C90B4F9F801FEF72EFD0D90B4F9E0
:108FC000FA01FEF729FD0E90B4F9FC01FEF724FD2D
:108FD0000AA90F900DA8F9F745F998F80130144D3A
:108FE000012B31D1174B1B7858070ED4D5F82C32F2
:108FF000402093FBF0F0181AFEF70EFD0F99FEF7D4
:1090000057FCFEF723FFC5F82C02094BD3F82C02BE
:10901000402390FBF3F019E03B597E90A9E7814093
:10902000399D52A246DF913FE80200200000002057
:10903000F0000020F00200200C03002004000020BB
:10904000BD378635F4130020A84B1888FEF7E4FCE2
:1090500001460F98FEF72AFCD4F834120F904846C8
:10906000FEF726FC01464846FEF7DEFDD4F83052F6
:10907000064629460F98FEF719FC01463046FEF7D2
:109080001FFD01462846FEF713FC0646C4F83002D1
:109090000D98D4F8387201F0A5FCD4F84452297820
:1090A000F9F712FA3844C4F838020E98D4F83C7232
:1090B00001F098FC2978F9F707FA3844C4F83C0223
:1090C0003046D4F8407201F08DFC6978F9F7FCF96C
:1090D000874B38441A68029FC4F840023A441A6029
:1090E000D4F848320133C4F8483205E0A7F8A83173
:1090F000A7F8AA31A7F8AC317E4D049FB5F84031EE
:10910000012FA5F84C32B5F842312E46A5F84E3263
:109110000ED1B5F95222B5F9443103EB42030322D3
:1091200093FBF2F39BB2A5F85032A5F8523203E05C
:10913000B5F84431A5F85032F8F760FE6E4BD5F81B
:109140002C211860D5F85432B5F96042C31A9BB28D
:109150000293A5F85832B2F85830C5F854029C4230
:109160000FDBB4F5FA6F92F8567007DAE11A4F4345
:10917000A3F5FA6397FBF3F7643703E0C7F16407DD
:1091800000E064275D4B0020B3F8189193F9EC30B0
:1091900015465B429BB204930146594B40F2E63EB2
:1091A000C35E0393C9EB030303F2F31CF44503D836
:1091B000002BB8BF5B4201E04FF4FA730229DFF8DD
:1091C00034E133D092F8D4C0BCF1000F04D0634531
:1091D000CCBFCCEB030300234FF0640C93FBFCF8F3
:1091E0000EEB480A6FF0630B0BFB083BBAF87EA24C
:1091F0000EEB480EBEF980820FFA8AFECEEB080E07
:109200000EFB0BFE9EFBFCFEF24492F854E0DFF8EE
:10921000FC8003FB0EFE3B4B20F808A09EFBF3F303
:1092200063449BB27B4393FBFCFC1CE092F8D5C0EB
:10923000BCF1000F04D06345CCBFCCEB030300238B
:10924000DDF8108003FB08FCAEF890C292F855E000
:1092500083EAE37CACEBE37C0CFB0EFC294B9CFB30
:10926000F3FC0CF1640C02EB010E9EF80480264B1B
:109270000CFB08F84FF0640E98FBFEF801F8038031
:1092800095F80EA003F103080CFB0AFA9AFBFEFA0C
:1092900001F808A095F818A003F106080CFB0AFCD9
:1092A0009CFBFEFCDDF80CE001F808C0CE45A3F500
:1092B000257807DA08F5237330F803E0CEF1000EC5
:1092C00020F803E00131032900F1020005F1010556
:1092D0007FF463AF094DB5F81A319C4218DBB4F541
:1092E000FA6FA8BF4FF4FA6413E000BF000000203B
:1092F000EC130020F0000020E81300200C0F0020E9
:109300004A0300200CFEFFFF840300207C030020A2
:109310001C46E41A4FF47A725443C3F5FA63B4FB63
:10932000F3F3642093FBF0F208EB42016FF0630467
:1093300004FB0233B1F89E1208EB4202B2F9A042DC
:109340000AB2A21A534393FBF0F0B8F8B6320144C4
:10935000A8F892125906A04F43D5B7F8B832B7F81B
:109360002802C01A00B2FDF7B5FF99A3D3E9002384
:10937000FEF716F8FEF746FA044601F0FDFA8146BC
:10938000204601F06DFB0446B7F98E02FEF744FB60
:109390008246B7F98C02FEF73FFB49468346FEF74B
:1093A0008FFB2146034650460193FEF789FB019B44
:1093B00001461846FEF77AFAFEF748FD4946A7F837
:1093C0008C025046FEF77CFB214681465846FEF74C
:1093D00077FB01464846FEF76BFAFEF737FDA7F824
:1093E0008E02AA6840F602031340002B66D098F85C
:1093F000C032D8F8BC7202980133DBB206210744B0
:10940000B3FBF1F088F8C03201FB103313F0FF0911
:10941000714CC8F8BC7251D1920712D5F8F762FCB2
:1094200094F8C122B4F8C232934207D3D4F8C432BC
:109430009B7893428CBF0023012300E04B4688F8C1
:10944000C832AB681B0536D598F8DD32D8F8CC1297
:1094500008EB4303B3F8E002082391FBF3F280B278
:109460008A1A024492FBF3F39BB240F6E44159435B
:10947000D8F8C43240F6FF70B1FBF0F1D888C8F8D4
:10948000CC22091A4FF47A7251439B8891FBF3F175
:109490004F43524B97FBF2F2C8F8E812D3E90001B0
:1094A000801841EBE271C3E900014D4A0023FEF749
:1094B00013FDC8F8F8020023C8F8BC3298F8082356
:1094C000454B98F8C87202B1012283F81123AB68AA
:1094D000444C13F4807F2CD0D8F8143320781B68C8
:1094E000C0F380005B683C4D984758B1012385F874
:1094F0001833D5F814331B68DB68984710B1022382
:1095000085F81833D8F814331B689B68984730B136
:1095100023785D0703D4304B022283F81823D8F850
:1095200014331B689B69984718B12B4B002283F8B2
:10953000182398F81823284B022A02D14C204E21D8
:1095400014E0012A06D153204D214C220B46FCF792
:1095500061FE1FE093F81123012A04D15320014634
:1095600002464D23F3E727B153204D210A464423F9
:10957000EDE7B3F8B622100603D553204D2102467D
:10958000E4E793F8DE211AB13220FCF714FE01E083
:1095900083F819732378590704D5134B4FF40052FD
:1095A0005A6171E098F8FC221AB90E4A43F001039F
:1095B0001370B8F8B03123B1074BD3F804319A07D0
:1095C00016D40A4B1B88003318BF012311E000BFDB
:1095D000399D52A246DF913FF0000020E0030020B9
:1095E000407E0500F413002000100140F01300201D
:1095F000012343B1C64BDA6882F40052DA60237863
:1096000023F00103237098F812311B0703D4237849
:1096100023F00103237098F810331BB1237823F053
:10962000010323702378BB4A13F0010F0AD00023F3
:10963000C8F81C3303F180434FF4005103F588331D
:1096400019610EE0D8F81C13136851B9B24903F53B
:10965000F42303F59073C1F81C33AD4B4FF4005164
:109660005961D8F81C33126873B1D21A002A0BDB87
:10967000A74A03F5F423D16803F5907381F40051F0
:10968000D160A54AC2F81C33A44B1B781BB1FCF770
:109690008FFF00F087BCA24F97F84A30012B05D00E
:1096A000A0494C378F42F7D100F07CBC9A4B3A6806
:1096B000C3F8B873C3F8BC23974CD4F8BC03254651
:1096C00003685B6898470028EAD0D4F8BC030368B5
:1096D0009B689847D4F8B83393F84820F2B9B0F1B2
:1096E000240EDEF1000252EB0E0283F84820002A1D
:1096F000E2D18D4B1B785D07DED4232802D1FCF725
:1097000057FFD9E7D4F8C0331B7D8342D4D1874AB1
:10971000874B1A60874A884BDA60CDE7012A05D16A
:109720004D2814BF0022022200F024BC022A05D1D9
:109730003C2814BF0022032200F01CBC032A0BD1DA
:1097400040284FF0000200F215841A71DA71587146
:109750009871042200F00EBC042A07D19A7983F88C
:10976000490050409871052200F004BC052AA3D19D
:1097700059791A799142997906D941409971511CC8
:1097800019711344187297E7814240F0EF8393F800
:109790004930702B00F0888275D8682B00F01D824C
:1097A00027D8652B00F0FD8018D8642B40F0FF848B
:1097B0000720624CF8F796FCE620F8F764FC607925
:1097C000F8F761FC0020F8F75EFC94F824015C4B8C
:1097D0005C4A00280CBF10461846ADE3662B00F02B
:1097E0008881672B40F0E3841020F8F77BFC00248D
:1097F000B6E16D2B00F0118213D8692B00F0F981CE
:109800006C2B40F0D4840620F8F76CFCB4F91802F5
:10981000F8F76BFCB4F91A02F8F767FCB4F9280200
:109820007AE36E2B00F000826F2B40F0C08407209B
:10983000F8F758FCD4F82C3193F85000F8F723FCD3
:10984000D4F82C3193F85100F8F71DFCD4F82C31E2
:1098500093F85400F8F717FCD4F82C3193F855001E
:10986000F8F711FCD4F82C3193F85600F8F70BFCFC
:10987000D4F82C3193F85200F8F705FCD4F82C31C9
:1098800093F85300F9E1772B00F0118367D8732B1D
:1098900000F0288358D8712B00F09E82722B40F084
:1098A0008684264D1620F8F71DFC0020F8F71DFCD5
:1098B000B5F9D000F8F719FCB5F9D200F8F715FCA6
:1098C000B5F9D400F8F711FCD4F82C31B3F91E0126
:1098D000F8F70BFC0020F8F708FC0020F8F72AFC4A
:1098E000D4F82C31B3F95A000A2390FBF3F0F8F7BF
:1098F000FCFB95F80401F8F7C6FB95F80601F8F7AC
:10990000C2FB95F80501F8F7BEFB0020B5E100BFEA
:1099100000100140E8130020F0000020F3130020A5
:1099200010040020A8040020F4130020EFBEADDED8
:10993000F04F00200400FA0500ED00E00C0F0020BD
:109940003C00008034000080742B00F07682752B80
:1099500040F02D842F20F8F7C5FBC94C34E2A02B32
:1099600000F0DD820AD8782B00F002817B2B40F0DA
:109970001E840820F8F7B6FB002422E1F02B00F04B
:10998000BE82FE2B40F013840820F8F7ABFB0020CA
:10999000F8F7ABFB0020F8F7A8FB0020F8F7A5FBD1
:1099A000ABE20B20F8F79EFBB4F95802F8F79DFBE9
:1099B000B4F8C40300B2F8F798FBD4F80431C3F349
:1099C000C000C3F38002800040EA4200C3F34002BB
:1099D0001043C3F3401240EAC20003F010031843DF
:1099E000F8F783FBB4F8B63294F802B303F0080A30
:1099F00094F803934AEA8B1A94F804434AEAC91983
:109A000049EA04299F4C13F0010F94F808A30CBFF6
:109A10004FF0000C4FF0020C49EA0A3994F809A300
:109A200013F0020F49EA4A3994F80BA30CBF4FF028
:109A3000000E4FF0040E49EACA3994F80CA313F053
:109A4000040F49EA0A4994F80DA30CBF002510251C
:109A500049EA4A4994F80EA313F0400F49EA8A49AB
:109A600094F80FA30CBF0020202049EACA4994F8BB
:109A700010A313F0100F49EA0A59DFF828A20CBF0F
:109A800000214FF400719AF800A013F0200FCAF3E0
:109A9000800A49EA0A0949EA0C0C4CEA0E0E4EEA21
:109AA000050545EA00000CBF00224FF48062014327
:109AB00013F4807F0CBF00234FF400630A4300209F
:109AC00094F8C6E31343044674450CD26E4A01254C
:109AD000A25C05FA02F21A4218BFA54004F1010483
:109AE00018BF2843F0E7F8F725FB684B93F8BC0450
:109AF000C3E01220F8F7F6FA654B1B88B3F5806FC8
:109B000021D90025634BE85E082390FBF3F0023572
:109B1000F8F7EBFA062DF5D1B4F94C02F8F7E5FAAF
:109B2000B4F94E02F8F7E1FAB4F95002F8F7DDFAA9
:109B3000B4F90C01F8F7D9FAB4F90E01F8F7D5FA2F
:109B4000B4F91001E8E1B4F9F801F8F7CEFAB4F984
:109B5000FA01F8F7CAFAB4F9FC01F8F7C6FADBE73C
:109B60004D4B185D0134F8F78EFA102CF8D1F7E15F
:109B70003820F8F7B7FA4FF00009D5F82C3109F181
:109B80001B04E4002344B3F90400F8F7AEFAD5F857
:109B90002C3109F101092344B3F90600F8F7A5FABD
:109BA000D5F82C312344B3F90800F8F79EFAD5F81C
:109BB0002C311C44A07AF8F766FAB9F1080FDCD111
:109BC000CEE1D5F82C3103EBC40393F8E300013464
:109BD000F8F759FA082CF4D1C2E11020F8F782FA0C
:109BE00000242E4B185D0134F8F74DFA102CF8D1F3
:109BF000B6E194F8DC030024400000F0FE00F8F722
:109C000071FA95F8DC339C4280F0AA81244B33F939
:109C10001400F8F76AFA0134F3E70620F8F762FA5D
:109C20000020F8F787FA68E10720F8F75BFA94F864
:109C3000C102F8F728FAD4F8F8024FF6FF75A842E7
:109C4000A8BF284620EAE07000B2F8F74EFAB4F94F
:109C5000DE03F8F74AFADFF82C900C4BD9F8E8024B
:109C600093F80C310028B8BF40420BB10A23584387
:109C7000A842A8BF284600B24EE1F8F704FA6FE107
:109C80004FC00008F0000020B70400200C0F002097
:109C900000000020E802002060000020CE13002019
:109CA0004A030020F41300201E20F8F71BFAD4F812
:109CB0002C3100241B78022B70D1D6F82C31AF49FF
:109CC00003EB8403586AFDF7FBFE00F08BFEFA28D5
:109CD000A8BFFA2020EAE070C0B2F8F7D4F9D6F8AD
:109CE0002C31A74903EB8403186BFDF7E9FE00F064
:109CF00079FEFA28A8BFFA2020EAE070C0B2F8F78F
:109D0000C2F9D6F82C319F4903EB8403D86BFDF7D9
:109D1000D7FE00F067FE6428A8BF642020EAE07048
:109D2000C0B20134F8F7AFF9032CC6D1072CD5F82F
:109D30002C311FD1986C9149FDF7C2FE00F052FE04
:109D4000FA28A8BFFA2020EAE070C0B2F8F79BF921
:109D5000D5F82C318949D86CFDF7B2FE00F042FEEF
:109D6000FA28A8BFFA2020EAE070C0B2F8F78BF911
:109D700000200DE023441879F8F785F9D5F82C3147
:109D80002344987BF8F77FF9D5F82C312344187ECB
:109D90000134F8F778F90A2CC8D1E1E0D5F82C3174
:109DA00023441879F8F76FF9D5F82C312344987BC0
:109DB000F8F769F9D5F82C312344187E0134F8F707
:109DC00062F90A2CEAD1CBE014F8010F002800F068
:109DD000C780F8F758F9F7E794F8C6030024800025
:109DE00000F0FC00F8F77EF995F8C623664B944224
:109DF0000DD2D3F82C2103F2C733E35C01342033B6
:109E000052F82300C0F30B00F8F76FF9ECE70024D9
:109E100095F8C6235C4B944280F0A280D3F82C21A5
:109E200003F2C733E35C013402EB8303B3F882002F
:109E3000C0F30B00F8F759F9EAE74FF0000A0124E4
:109E40004FF0000995F8C633994528DA4F4B19F8B9
:109E5000030000234E4903EB0108595C814204D002
:109E60000C33B3F5847FF5D116E0D8F8040000F088
:109E700095FB03460CB9A34601E082440CE09B45E8
:109E80000ADAD8F8041011F80B0001930BF1010B5A
:109E9000F8F7F9F8019BF2E709F10109D2E7002C84
:109EA0005ED05FFA8AF0F8F71DF90024C8E794F84D
:109EB000C603F8F717F9002495F8C6339C424FD231
:109EC000324BE05C0023324A99189A5C824204D0FB
:109ED0000C33B3F5847FF6D102E0087AF8F7D3F8B3
:109EE0000134E9E70820F8F7FDF80124E0B2013475
:109EF000F8F7C9F8092CF9D132E000200CE0042071
:109F0000F8F7F0F8D4F82C31B3F95E00F8F7EDF873
:109F1000D4F82C31B3F95C00F8F7E7F820E00C2016
:109F2000F8F7E0F81B4B1868F8F704F91A4B1868B3
:109F3000F8F700F9194B1868F8F7FCF810E000F290
:109F40007B82D22B40F0CB82154B1B7803F00403AD
:109F500003F0FF04002B00F037820020F8F7C2F86E
:109F6000094BD3F8B8339879F8F78DF8064B0022EF
:109F7000D3F8B83383F84820FFF79EBB0000204198
:109F80000000C84200007A44F0000020B70400201E
:109F900080C00008E8F7FF1FECF7FF1FF0F7FF1F76
:109FA000F41300209C4CD4F8383113B104F2FA3089
:109FB0009847D4F80431984A13F0080F974F38D0D7
:109FC000B2F8901201F145039BB28A2B2DD8B2F85A
:109FD000B6325E0729D5B2F82802B2F8E03394F819
:109FE0001251C21A92B293B218B2B330BCBF02F58A
:109FF000B4739BB21AB2B32AC4BFA3F5B4739BB2B5
:10A000002D0797F8EC00844A13D540B240424343F1
:10A01000D2F82C011BB2007B43436FF01D0093FB71
:10A02000F0F31944A2F8901203E0B4F82832A4F82F
:10A03000E033D4F82C61784D96F8DA90B9F1000F3E
:10A0400055D0B5F8B6329A0751D0D5F80002D5F8F8
:10A0500004320146D5F80882B5F892A20193FDF7C3
:10A060002FFD019B834619461846FDF729FD014641
:10A070005846FDF71DFC414683464046FDF720FD4E
:10A0800001465846FDF714FC00F07AFD01464046B3
:10A09000FDF7CAFD62498046FDF7BAFE18BB40468F
:10A0A00000F01CFDD5F8FC13FDF70AFD00F09AFC4A
:10A0B000B0F5617FA8BF4FF46170FDF70BF954A3B1
:10A0C000D3E90023FDF796FAFDF79CFB00F0C8FCEE
:10A0D00005464846FDF7A0FC2946FDF7F1FC00F0D7
:10A0E00081FC80B200E000205044A4F892024D4B65
:10A0F000301D1D6806F1500106F15C03B7F8F6202B
:10A10000A847FBF78BFCD4F80034002B4BD0424B14
:10A1100093F80434013B142B40D8DFE803F00B3FE5
:10A120003F27423F3F1F3F3F3F3F3F2F3F3F3F3F84
:10A130003F272F00D4F808345B782BB13A4B00202E
:10A140005989F8F753FB2EE0384B1B7803F00403D2
:10A1500003F0FF00002BF1D10146F2E7324C002062
:10A16000E188F8F743FB01202189EAE72E4C002023
:10A170002189F8F73BFB01206189E2E72A4C0020A6
:10A18000E188F8F733FB01202189F8F72FFB022043
:10A190006189F8F72BFB0320A189D2E7BB689B06F6
:10A1A00001D5F8F72FFBF8F717F8FEF7DAB9D02B3F
:10A1B0000BD11E4B1B7858073FF5CFAEFCF72EFB9B
:10A1C000F9F714F8FAF7D0FCC7E600F2F280CC2BCE
:10A1D0002ED1D4F82C41F7F7C9FD84F85000F7F7D9
:10A1E000C5FD84F85100F7F7C1FD84F85400F7F776
:10A1F000BDFD84F85500F7F7B9FD84F85600F7F770
:10A20000B5FD84F85200F7F7B1FD84F85300A4E6D9
:10A21000A2EB0FE5DD169640F00000200C0F0020A9
:10A220008FC2753C7000002060000020F4130020F5
:10A2300075D8CA2B60D1D4F82C412378022B4BD18E
:10A24000A1460024F7F792FDFDF7E2FBA649FDF7D2
:10A25000EBFCC9F82400F7F789FDFDF7D9FBA3490A
:10A26000FDF7E2FCC9F83000F7F780FDFDF7D0FB01
:10A270009F49FDF7D9FC0134032CC9F83C0009F1D2
:10A280000409DFD1072CD5F82C9114D1F7F76EFD16
:10A29000FDF7BEFB9449FDF7C7FCC9F84800F7F786
:10A2A00065FDFDF7B5FB9049FDF7BEFCC9F84C0014
:10A2B000F7F75CFD0CE0F7F759FDA14489F80400BD
:10A2C000F7F754FD89F80E00F7F750FD89F81800EC
:10A2D00001340A2CD6D140E6013C0025F7F746FDB3
:10A2E00001342071F7F742FDA073F7F73FFD013508
:10A2F0000A2D2076F2D130E600F2C480C82B40F05F
:10A30000EE800024F7F73CFD7A4B03F25A221053FB
:10A310000234102CF6D1012283F8F4201DE6CE2B56
:10A320000BD1754B1B785A073FF517AE94F81231D5
:10A3300043F0040384F812310FE630D9F7F720FD1B
:10A34000F7F71EFD6D4DA5F8D000F7F719FDA5F83C
:10A35000D200F7F715FDD4F82C41A5F8D400F7F793
:10A360000FFDA4F81E01F7F70BFDF7F709FDF7F74E
:10A3700007FDF7F705FD00EB80004000A4F85A0048
:10A38000F7F7F4FC85F80401F7F7F0FC85F806010F
:10A39000F7F7ECFC85F80501F7F7E8FCDDE5564B2F
:10A3A0001B7859073FF5D9AD4FF4C873A4F8B03105
:10A3B000D3E5D52B33D012D8D32B7FF4C0ADF7F72C
:10A3C000DFFCA4F8E003C8E5F7F7D0FC4B4B02280C
:10A3D00083F8BC047FF6F4AE83F8BC44F0E6EF2BC0
:10A3E0000AD1D4F82C41F7F7CBFCA4F85E00F7F7BC
:10A3F000C7FCA4F85C00B0E5FA2B05D13E4B1B78F6
:10A400005B077FF5DDAE6AE0D62B68D10024F7F755
:10A41000B7FC3B4B18530234102CF8D19DE50024B7
:10A42000D5F82C91F7F7A2FC09EBC4030134082CF2
:10A4300083F8E300F4D190E54FF00009D5F82C4102
:10A44000F7F79EFC04EBC904A4F8DC00F7F798FCCE
:10A45000A4F8DE00F7F794FCA0F57A7307289BB206
:10A4600098BF84F8E300B3F57A7F98BFA4F8E000C2
:10A47000F7F77CFC09F10109B9F1080F84F8E20053
:10A48000DCD16AE5002495F8C6931A4B4C450FD2EF
:10A49000D3F82C9103F2C73314F803A0F7F770FC3C
:10A4A0000AF1200AC0F30B0049F82A000134EAE758
:10A4B00000244C453FF451AD124B14F803A0D5F8DD
:10A4C0002C31013403EB8A0ADAF880B0F7F758FC34
:10A4D000C0F30B004BEA0040CAF88000E9E7012016
:10A4E0000021F7F7E1FD3BE5000020410000C842F4
:10A4F00000007A44F0000020F41300200C0F00202C
:10A50000D2040020B704002010B50023934203D0EA
:10A51000CC5CC4540133F9E710BD024403469342B6
:10A5200002D003F8011BFAE7704700000D4B70B52D
:10A530001D680022845C2B195B7803F00303012B58
:10A540008B5C08BF2034EE18767806F00306012EE7
:10A5500008BF2033E41A02D10132002BEAD1204691
:10A5600070BD00BF8000002010B50446224613785D
:10A570000134002BFAD1CC5CD4540133002CFAD135
:10A5800010BDC9B2024610F8013B1BB18B42F9D194
:10A59000104670470029FBD018467047034613F851
:10A5A000012B002AFBD1181A013870470F4BF0B568
:10A5B0001E680023934215D0C55C7419647804F0BA
:10A5C0000304012CCC5C08BF203537197F7807F0D5
:10A5D0000307012F08BF20342D1B04D10133002CA9
:10A5E000E8D100E000252846F0BD00BF8000002033
:10A5F00010B5034632B111F8014B013A03F8014B93
:10A60000002CF7D11A44934203D0002103F8011B18
:10A61000F9E710BD30B503780BB1044604E00B78C0
:10A62000002B18BF002030BD22461078013438B10D
:10A630000023C85C28B1D55C8542F5D10133F8E729
:10A6400030BD104630BD00210A2200F001B92DE9CD
:10A65000F04E82468B461F46144612B90020BDE8D4
:10A66000F08E002BFAD00026A642F7D2A5196D086D
:10A6700007FB05B950464946089B9847002802DB6E
:10A6800003D06E1C25462C46EEE74846BDE8F08E0A
:10A69000174B2DE9F0411D680646AC6D0F46FCB91D
:10A6A000502000F0E3F8A8658460AB6D046044605E
:10A6B0001C61DC60AB6D9C615C61AB6DDC629C62BB
:10A6C000AB6D5C631C63AB6DDC639C63AB6D5C6406
:10A6D0001C64AB6DDC649C64AB6D1C77AB6D5C6221
:10A6E00030463946AA6D0123BDE8F04100F002B8BA
:10A6F000E4000020F0B508B9106828B3044614F847
:10A70000015B0F4617F8016B3EB1B542FAD10BB1B0
:10A710002046F3E714600370F0BD4DB9156028467C
:10A72000F0BD17F8016BAE4207D0002EF9D11C46E0
:10A73000234613F8015B0F46F3E715B100212170A2
:10A7400000E02B461360F0BDF0BD000084463F489A
:10A750002DE9F04FD0F800800E46344614F8015B26
:10A7600008EB0500407800F0080000F0FF0708B192
:10A770002646F2E72D2D03D1B41C7578012703E09E
:10A780002B2D04BF7578B41C33F010000DD1302D83
:10A7900008D1207800F0DF00582851D165781023C7
:10A7A000023402E0002B08BF0A23002F0CBF6FF019
:10A7B000004A4FF0004ABAFBF3F903FB19AA00263E
:10A7C000304608EB050B9BF801B01BF0040F01D0DD
:10A7D000303D0BE01BF0030B1BD0BBF1010F14BF8E
:10A7E0004FF0570B4FF0370BCBEB05059D4210DABE
:10A7F000B6F1FF3F0AD0484506D801D1554503DCE4
:10A8000003FB0050012601E04FF0FF3614F8015B16
:10A81000D7E7731C0CD1002F4FF022030CBF6FF051
:10A8200000404FF00040CCF800302AB9BDE8F08F6E
:10A8300007B1404242B106B1611E1160BDE8F08F20
:10A84000002B08BF0823B0E7BDE8F08F8000002090
:10A8500030B51346044A05460C4610682946224680
:10A86000BDE83040FFF772BFE4000020024B014614
:10A87000186800F003B800BFE400002070B5CD1CDC
:10A8800025F0030508350C2D38BF0C25002D064694
:10A890003FDB8D423DD3214B1C6818462146A1B1B8
:10A8A0000B685B1B0ED40B2B03D90B60CC18CD505F
:10A8B0001FE08C4202D1626802601AE04B6863605C
:10A8C0000C4616E00C464968E9E7154C23681BB9AD
:10A8D000304600F027F820602946304600F022F884
:10A8E000431C014615D0C41C24F0030484420AD141
:10A8F000256004F10B00231D20F00700C31A0BD0C4
:10A900005A42E25070BD3046611A00F00BF8013037
:10A91000EED10C233360002070BD00BFFC1300207B
:10A92000F813002038B5064C00230546084623607E
:10A9300000F008F8431C02D1236803B12B6038BD36
:10A9400004140020094A136863B118446946884218
:10A9500002D8106018467047054B0C221A604FF061
:10A96000FF307047034B1360EFE700BF0014002077
:10A97000041400200814002000B5194A20F00043F8
:10A98000934283B0014617DDB3F1FF4F04DBFCF7C0
:10A990008DFF03B05DF804FB694600F037FB00F063
:10A9A0000302012A0098019911D0022A0AD09AB113
:10A9B000012201F0EFF8ECE7002100F0EFFC03B01A
:10A9C0005DF804FB00F0EAFC00F10040E1E701F073
:10A9D000E1F800F10040DCE700F0E0FCD9E700BF5F
:10A9E000D80F493F30B5C0F3C754A4F17F031E2BE5
:10A9F00083B0014620DC581C1BDB162B4FEAD175B7
:10AA000009DDC1F3160040F40000963CA04005B1FA
:10AA1000404203B030BD114B53F825402046FCF7AF
:10AA200047FF019001982146FCF740FF20F00043CA
:10AA300033B9002003B030BDFDF708FA03B030BDD4
:10AA4000C0F31604C0F3C75044F40004C0F19600EC
:10AA500024FA00F0002DDCD0DAE700BFFCE30008A8
:10AA600000B51D4A20F00043934283B0014618DD33
:10AA7000B3F1FF4F04DBFCF719FF03B05DF804FBF3
:10AA8000694600F0C3FA00F00300012818D002283C
:10AA90000ED0D0B10098019900F080FC00F1004088
:10AAA000EBE70021002201F075F803B05DF804FB2C
:10AAB00000980199012201F06DF800F10040DCE7F7
:10AAC0000098019900F06AFCD7E7009801990122EB
:10AAD00001F060F8D1E700BFD80F493F70B58AB0E8
:10AAE000054600F09BF8224C064694F900300133ED
:10AAF00003D0284601F02CFA10B930460AB070BDD8
:10AB0000284601F0DBF94FF07E51FDF795F900285A
:10AB1000F3D018490122002328460092089301919E
:10AB2000FCF7EAFB02460B461348CDE90423CDE9C6
:10AB3000022301F0A7F894F90030CDE90601022BB9
:10AB40000BD0684601F09CF838B1089B53B9DDE999
:10AB50000601FCF757FE0AB070BD01F073FA21231D
:10AB60000360F2E701F06EFA089B0360EFE700BFB5
:10AB7000E800002004E400080CE4000800F0B6B986
:10AB800070B58AB0054600F0B5FB224C064694F934
:10AB90000030013308D0284601F0DAF920B1284608
:10ABA0000021FDF72BF910B930460AB070BD1A49E3
:10ABB000012200232846019100920893FCF79CFB98
:10ABC0002478CDE90401CDE902017CB900220023FB
:10ABD000CDE90623684601F053F888B1089BA3B974
:10ABE000DDE90601FCF70EFE0AB070BD0020002171
:10ABF00002460B46FCF7FEFC022CCDE90601E9D12A
:10AC000001F020FA21230360E8E701F01BFA089B1A
:10AC10000360E5E7E800002010E40008F8B520F044
:10AC20000043B3F17E5F044610D008DCB3F17C5FD3
:10AC300011DAB3F10C5F00F384809D48F8BD014642
:10AC4000FCF734FE0146FCF7EFFFF8BD002840F3A7
:10AC5000CD800020F8BD0028C0F2CA8001464FF028
:10AC60007E50FCF723FE4FF07C51FCF729FF044691
:10AC700000F040FB8F4906462046FCF721FF8E4935
:10AC8000FCF716FE2146FCF71BFF8C49FCF70EFE75
:10AC90002146FCF715FF8A49FCF70AFE2146FCF71E
:10ACA0000FFF8849FCF702FE2146FCF709FF8649A1
:10ACB000FCF7FEFD2146FCF703FF844905462046CC
:10ACC000FCF7FEFE8249FCF7F1FD2146FCF7F8FE99
:10ACD0008049FCF7EDFD2146FCF7F2FE7E49FCF7CA
:10ACE000E5FD2146FCF7ECFE4FF07E51FCF7E0FD60
:10ACF00001462846FCF798FF3146FCF7E1FE26F4B2
:10AD00007F6525F00F05074629462846FCF7D8FE43
:10AD100001462046FCF7CAFD294604463046FCF7AA
:10AD2000C7FD01462046FCF77FFF01463846FCF789
:10AD3000BFFD01462846FCF7BBFD0146FCF7B8FD08
:10AD4000F8BD0146FCF7BCFE5A490546FCF7B8FEC3
:10AD50005949FCF7ADFD2946FCF7B2FE5749FCF70F
:10AD6000A5FD2946FCF7ACFE5549FCF7A1FD294697
:10AD7000FCF7A6FE5349FCF799FD2946FCF7A0FE17
:10AD80005149FCF795FD2946FCF79AFE4F490646C6
:10AD90002846FCF795FE4E49FCF788FD2946FCF74E
:10ADA0008FFE4C49FCF784FD2946FCF789FE4A4991
:10ADB000FCF77CFD2946FCF783FE4FF07E51FCF743
:10ADC00077FD01463046FCF72FFF01462046FCF791
:10ADD00077FE01464148FCF769FD01462046FCF735
:10ADE00065FD01463E48FCF761FDF8BD3D48F8BDF4
:10ADF0004FF07E51FCF75CFD4FF07C51FCF760FE9C
:10AE00002C490446FCF75CFE2B49FCF751FD21461A
:10AE1000FCF756FE2949FCF749FD2146FCF750FE98
:10AE20002749FCF745FD2146FCF74AFE2549FCF77A
:10AE30003DFD2146FCF744FE2349FCF739FD214640
:10AE4000FCF73EFE0646204600F054FA1F49054630
:10AE50002046FCF735FE1E49FCF728FD2146FCF78D
:10AE60002FFE1C49FCF724FD2146FCF729FE1A4958
:10AE7000FCF71CFD2146FCF723FE4FF07E51FCF74A
:10AE800017FD01463046FCF7CFFE2946FCF718FEB9
:10AE90001249FCF70BFD01462846FCF709FD014667
:10AEA000FCF706FD01461048FCF700FDF8BD00BFA9
:10AEB000DB0FC93F08EF1138047F4F3A4611243D9C
:10AEC000A80A4E3E90B0A63EABAA2A3E2EC69D3D95
:10AED0006133303F2D57014039D119406821A233E9
:10AEE000DA0FC93FDB0F4940DA0F494021F0004239
:10AEF000B2F1FF4FF8B5044614DC20F00045B5F17F
:10AF0000FF4F06460EDCB1F17E5F3AD08F1707F097
:10AF1000020747EAD07755B9022F2FD0032F2FD140
:10AF20003148F8BD08462146FCF7C2FCF8BDFAB12D
:10AF3000B2F1FF4F29D0B5F1FF4F19D0AA1AD2159F
:10AF40003C2A19DC002938DB2046FCF76DFE00F0B6
:10AF5000B5FF00F09DFE012F2CD0022F22D0002F34
:10AF60002FD02249FCF7A4FC2149FCF79FFCF8BD37
:10AF7000002E15DB1F48F8BD1E48ECE71C48F8BD45
:10AF8000F8BDBDE8F84000F083BEB5F1FF4F19D021
:10AF9000022FF3D0032FC3D0012F1BD00020F8BD08
:10AFA0001548F8BD1149FCF783FC01461048FCF731
:10AFB0007DFCF8BD00F10040F8BD3C32C4DA002051
:10AFC000C9E7F8BD022F0CD0032F08D0012F04D001
:10AFD0000A48F8BD4FF00040F8BD0948F8BD0948DF
:10AFE000F8BD0948F8BD00BFDB0F49C02EBDBB331B
:10AFF000DB0F4940DB0FC93FDB0FC9BFDB0F493F08
:10B00000DB0F49BFE4CB16C0E4CB16402DE9F04F6F
:10B01000AB4A20F00044944289B006460D4664DDF8
:10B02000A84A94421CDC0028A74940F3EC80FCF7B6
:10B030003DFCA64B24F00F049C42064664D0A44974
:10B04000FCF734FC014628603046FCF72FFCA04991
:10B05000FCF72CFC01236860184609B0BDE8F08FAE
:10B060009C4A944262DDB4F1FF4F46DAE715863F11
:10B07000A4EBC7542046FCF7E9FEFCF7CDFC0346E1
:10B08000014620460593FCF711FC4FF08741FCF781
:10B0900017FD8046FCF7DAFEFCF7BEFC01460446CD
:10B0A00040460694FCF702FC4FF08741FCF708FD90
:10B0B00000210790FCF798FE002800F0C58020468C
:10B0C0000021FCF791FE002814BF012302238248CF
:10B0D0000221019000913A4605A8294600F022FA83
:10B0E000002EC0F2A780034603E000222860002360
:10B0F0004A60184609B0BDE8F08F0146FCF7D6FB60
:10B10000002368602860F4E77449FCF7CFFB7449BA
:10B110000446FCF7CBFB014628602046FCF7C6FB43
:10B120006F49FCF7C3FB01236860E2E700F0C6FE4D
:10B130006C490746FCF7C4FC4FF07C51FCF7B8FBA8
:10B14000FCF784FE8246FCF767FC5F498346FCF708
:10B15000B7FC01463846FCF7A9FB5D4980465846D6
:10B16000FCF7AEFCBAF11F0F81464946404618DC99
:10B170005D4B0AF1FF3253F8223024F0FF029A426D
:10B180000FD0FCF793FB07462F6039464046FCF78B
:10B190008DFB4946FCF78AFB002E686056DB534660
:10B1A000A7E7FCF783FBE315C0F3C7529A1A082AF6
:10B1B0000746E9DD494958460393FCF781FC0746F9
:10B1C00039464046FCF772FB044621464046FCF7F0
:10B1D0006DFB3946FCF76AFB414907465846FCF7C8
:10B1E0006FFC3946FCF762FB814649462046FCF776
:10B1F0005DFB039BC0F3C7529B1A192B074641DC2A
:10B200002860A046C1E7FCF753FB304B24F00F0445
:10B210009C42064623D02E49FCF74AFB0146286093
:10B220003046FCF743FB2A49FCF742FB4FF0FF3363
:10B2300068605EE795E80C0003F1004102F100420E
:10B2400043422A60696054E7032340E707F100475F
:10B2500000F100402F606860CAF1000349E71F4910
:10B26000FCF726FB1E490446FCF722FB014628603A
:10B270002046FCF71BFB1A49FCF71AFB4FF0FF3383
:10B28000686036E719495846FCF71AFC0746394604
:10B290002046FCF70BFB804641462046FCF706FBA8
:10B2A0003946FCF703FB124904465846FCF708FCF4
:10B2B0002146FCF7FBFA81464946404661E700BF5C
:10B2C000D80F493FE3CB1640800FC93FD00FC93F8D
:10B2D00043443537800F494398E40008004435372C
:10B2E00008A3852E84F9223F18E4000800A3852EC8
:10B2F00032318D2420F00042B2F1FF4FF8B5044600
:10B3000003462DD25AB300283DDBB2F5000F4FEAB9
:10B31000E0502CD37F38C3F31603C20743F4000375
:10B3200048BF5B00002740105B003E4619244FF0E9
:10B330008072B5189D4202DC5B1BAE181744013CBD
:10B340004FEA43034FEA5202F3D113B107F001036E
:10B350001F447F1007F17C5707EBC050F8BDF8BDC4
:10B360000146FCF7ADFB2146FCF7A2FAF8BD14F448
:10B3700000020FD15B00190202F10102FAD5C2F1FD
:10B3800001021044C6E70146FCF790FA0146FCF7BB
:10B390004BFCF8BD01221044BCE700BF2DE9F84387
:10B3A00020F00046B6F1485F05460F4649DAFCF743
:10B3B0004DFD002800F09D8029462846FCF780FBC3
:10B3C0004E490446FCF77CFB4D49FCF771FA2146D7
:10B3D000FCF776FB4B49FCF769FA2146FCF770FB5A
:10B3E0004949FCF765FA2146FCF76AFB4749FCF737
:10B3F0005DFA2146FCF764FB4549FCF759FA214602
:10B40000FCF75EFB804620464FF07C51FCF758FB72
:10B41000414606462046FCF753FB3946044628467B
:10B42000FCF74EFB01462046FCF740FA0146304649
:10B43000FCF73CFA01464FF07E50FCF737FABDE8C6
:10B44000F8830146FCF73CFB2C490446FCF738FB2B
:10B450002B49FCF72DFA2146FCF732FB2949FCF772
:10B4600025FA2146FCF72CFB2749FCF721FA214657
:10B47000FCF726FB2549FCF719FA2146FCF720FBCF
:10B480002349FCF715FA2146FCF71AFB214B8046AD
:10B490009E42B8DD204B9E4227DC06F17F463146B6
:10B4A0004FF07E50FCF702FA814620464FF07C5167
:10B4B000FCF706FB3146FCF7F9F941460646204603
:10B4C000FCF7FEFA394604462846FCF7F9FA01462D
:10B4D0002046FCF7EBF901463046FCF7E7F9014658
:10B4E0004846FCF7E3F9BDE8F883DFF834900B4EEB
:10B4F000DBE74FF07E50BDE8F88300BF4ED747AD85
:10B50000F6740F317CF29334010DD037610BB63AEB
:10B51000ABAA2A3D9999993E0000483F0000903E11
:10B520000000383F2DE9F04FDFB00B93013B029351
:10B53000D31E48BF131DB84C06466898DB1054F85C
:10B54000204023EAE3730C93DB4302EBC30308942C
:10B550000693089C029B0C9A1D190991C3EB0207E4
:10B560001DD4699C3D4404EB870901354FF0000868
:10B5700022AC0AE059F80800FCF74EFA0137AF4256
:10B5800044F8080008F1040809D0002FF2DA013766
:10B590000020AF4244F8080008F10408F5D1089AE9
:10B5A000002AC0F2DF82089A0B9B02F101089C007E
:10B5B00022AF4FEA880827440025029A002AC0F2E9
:10B5C000F28105EB070B4FF000094FF0000A56F827
:10B5D00009005BF8041DFCF773FA01465046FCF7BE
:10B5E00067F909F10409A1458246F0D14AA840F85B
:10B5F00005A004354545E0D1089A0EAB03EB820364
:10B600000D9391464FEA89030793079A5EAB134463
:10B61000B9F1000F53F850AC23DD0DF134084AAFF7
:10B62000174490440DAD4FF06E515046FCF748FA68
:10B63000FCF70CFCFCF7F0F94FF087418346FCF770
:10B640003FFA01465046FCF731F9FCF7FFFB59463B
:10B6500045F8040F57F8040DFCF72AF945458246D2
:10B66000E1D15046069900F08DFC4FF07851054627
:10B67000FCF726FA00F026FC4FF08241FCF720FA96
:10B6800001462846FCF712F90546FCF7DFFB824627
:10B69000FCF7C2F901462846FCF708F9069A8046ED
:10B6A000002A40F3678109F1FF310EA850F82130DC
:10B6B000C2F1080043FA00F202FA00F01B1A0698E1
:10B6C0009244C0F1070743FA07F70EA840F821306B
:10B6D000002F32DDB9F1000F0AF1010A40F3758144
:10B6E0000EAB079A19461144002507E0C2F5807099
:10B6F00012B143F8040C01258B420BD053F8042BF4
:10B70000002DF3D0C2F1FF028B4243F8042C4FF01E
:10B710000105F3D1069B002B0DDD012B00F03281DA
:10B72000022B08D109F1FF330EA951F8232002F0B2
:10B730003F0241F82320022F70D040460021FCF741
:10B7400053FB002800F08380089A09F1FF35AA42D4
:10B750000DDC079A0EAB0D981344002253F8041D1C
:10B76000834242EA0102F9D1002A40F0E481089BB9
:10B770000EA85A1E50F82230002B40F0F18100EB49
:10B780008202012352F8041D01330029FAD04B44F0
:10B7900099450A933DDADDF82CA022AACA44DDF8C7
:10B7A000308002EB8A02C844C9EB0309131D0392DF
:10B7B0000593699A079B4FEA89094AAF02EB88080B
:10B7C000CDF810901F44002558F8040FFCF724F919
:10B7D000029B039A002B50514FF0000B13DBDDF856
:10B7E00014A04FF00009AA4456F809005AF8041DA5
:10B7F000FCF766F901465846FCF75AF809F10409C6
:10B80000A1458346F0D1049A0435954247F804BF18
:10B81000DAD1DDF82890F5E6B0E7000841464FF0B0
:10B820007E50FCF743F88046002D86D006994FF0F5
:10B830007E5000F0A7FB01464046FCF737F88046F3
:10B8400040460021FCF7D0FA00287FF47DAF069B2C
:10B8500040465942CDF808A000F094FB4FF08741D4
:10B860000446FCF7DFFA002800F07F814FF06E51AC
:10B870002046FCF725F9FCF7E9FAFCF7CDF84FF084
:10B8800087410546FCF71CF901462046FCF70EF8F7
:10B89000FCF7DCFA0EAB43F829002846FCF7D6FA91
:10B8A000069C09F1010508340EA9069441F825000B
:10B8B00006994FF07E5000F065FB002D04464FDBEB
:10B8C0006E1C4FEA8508C6EB867A0DF138094AAB43
:10B8D000C1444FEA8A0A98444FF0000B59F80B0014
:10B8E000FCF79AF82146FCF7EBF84FF06E5148F858
:10B8F0000B002046FCF7E4F8ABF1040BD3450446FB
:10B90000ECD1DFF88C92DDF820A00024B34603953B
:10B910000497BAF1000FB8BF002515DB00263746A3
:10B92000002501E0A7420FDC58F8061059F8060080
:10B93000FCF7C6F801462846FBF7BAFF0137BA45BF
:10B94000054606F10406EDDA5EA800EB8403013437
:10B95000A345A8F1040843F8A05CDAD1039D049F35
:10B96000689C032C00F29880DFE814F0CB009C0068
:10B970009C00310010D109F1FF330EA951F823705A
:10B980003F12A5E609F1FF330EA850F8232002F07C
:10B990007F0240F82320CEE64FF07C51FCF742FABC
:10B9A00058B90746C9E64FF0000A4AA840F805A072
:10B9B000043545457FF401AE1EE6B9F1000F4FF0A6
:10B9C00002070AF1010A3FF78BAE0025A2E6002D1F
:10B9D00040F3DC804FEA850B5EAB36AE05F1FF3AF3
:10B9E0005B4406EB8A0A53F8A08C54465B4635AAA2
:10B9F000BB462F4600E0C84654F804594146284645
:10BA000001920093FBF754FF814649462846FBF715
:10BA10004DFF4146FBF74CFF019AC4F80490944255
:10BA2000A060009BE7D13D46012D5F469B4640F359
:10BA3000AD805EAB9B445BF8A04C00E044465AF8F6
:10BA4000049921464846FBF733FF80464146484665
:10BA5000FBF72CFF2146FBF72BFF5645CAF8048065
:10BA6000CAF80800EAD16C1C06EB840400200836F2
:10BA700054F8041DFBF71CFFB442F9D1002F7ED00F
:10BA8000369A379B099C00F1004002F1004203F115
:10BA90000043A06022606360029A02F007005FB07A
:10BAA000BDE8F08F002DB8BF00200ADB36AE6C1C5D
:10BAB000002006EB840454F8041DFBF7F9FEB442A1
:10BAC000F9D1002F35D000F10043099C01462360D5
:10BAD0003698FBF7EBFE002D08DD36AC04EB850550
:10BAE00054F8041FFBF7E4FEAC42F9D10FB100F1AA
:10BAF0000040099A5060029A02F007005FB0BDE86A
:10BB0000F08F002D39DB6C1C36AE002006EB840470
:10BB100054F8041DFBF7CCFEB442F9D10FB100F18B
:10BB20000040099A1060029A02F007005FB0BDE879
:10BB3000F08F0346C9E7069A0EAC54F82530083A50
:10BB4000CDF808A00692002B7FF4B2AE04EB85037B
:10BB500053F8041D013D083A0029F9D00692A7E6E2
:10BB6000012314E60B9B9C0046E52046FCF76EF98A
:10BB70000EAA4D4642F829009AE60020CEE7099C1D
:10BB8000369A379BA0602260636085E7002075E7E6
:10BB9000BCE700082DE9F84320F00043B3F1485F0B
:10BBA00004460F46904603DAFCF750F9002857D0B8
:10BBB00021462046FBF784FF21460546FBF780FF20
:10BBC000294906462846FBF77BFF2849FBF76EFE0E
:10BBD0002946FBF775FF2649FBF76AFE2946FBF766
:10BBE0006FFF2449FBF762FE2946FBF769FF2249F4
:10BBF000FBF75EFE8146B8F1000F22D038464FF0C9
:10BC00007C51FBF75DFF494680463046FBF758FF05
:10BC100001464046FBF74AFE2946FBF751FF3946ED
:10BC2000FBF744FE154905463046FBF749FF014640
:10BC30002846FBF73DFE01462046FBF737FEBDE8F0
:10BC4000F88349462846FBF73BFF0C49FBF72EFEDD
:10BC50003146FBF735FF2146FBF72AFEBDE8F883A6
:10BC60002046BDE8F88300BFD3C92E2F342FD7322A
:10BC70001BEF3836010D50398988083CABAA2A3EA3
:10BC80000020704700200149704700BF0000F87F86
:10BC90002DE9F04120F00045B5F1A14F04460646DC
:10BCA00008DBB5F1FF4F6FDC002840F3A0806F4840
:10BCB000BDE8F0816E4B9D4277DCB5F1445F68DBF7
:10BCC0004FF0FF3721462046FBF7FAFE014680463B
:10BCD000FBF7F6FE67490546FBF7F2FE6649FBF700
:10BCE000E7FD2946FBF7ECFE6449FBF7E1FD294639
:10BCF000FBF7E6FE6249FBF7DBFD2946FBF7E0FEBA
:10BD00006049FBF7D5FD2946FBF7DAFE5E49FBF7F4
:10BD1000CFFD4146FBF7D4FE5C4980462846FBF741
:10BD2000CFFE5B49FBF7C2FD2946FBF7C9FE594927
:10BD3000FBF7BCFD2946FBF7C3FE5749FBF7B6FDF1
:10BD40002946FBF7BDFE5549FBF7B0FD2946FBF739
:10BD5000B7FE7B1C014640464CD0FBF7A9FD2146AF
:10BD6000FBF7AEFE4E4B4F4D53F82710FBF79EFDF1
:10BD70002146FBF79BFD014655F82700FBF796FD92
:10BD8000002E30DBBDE8F0810146FBF791FDBDE8F8
:10BD9000F0814549FBF78CFD4FF07E51FCF74CF8E4
:10BDA00000288DD02046BDE8F08100F087F83F4B99
:10BDB00004469D4229DCA3F5D0039D4244DC0146A4
:10BDC000FBF776FD4FF07E51FBF770FD4FF08041A1
:10BDD00005462046FBF76CFD01462846FBF724FF8D
:10BDE000002704466EE700F10040BDE8F0813048CE
:10BDF000BDE8F081FBF75CFD2146FBF761FE0146E3
:10BE00002046FBF753FDBDE8F0812A4B9D4214DC30
:10BE10004FF07F51FBF74AFD4FF07F51054620461A
:10BE2000FBF74EFE4FF07E51FBF742FD01462846E0
:10BE3000FBF7FAFE0227044644E701461E48FBF7DB
:10BE4000F3FE032704463DE74FF07E51FBF72EFD3E
:10BE50004FF07E5105462046FBF72AFD0146284655
:10BE6000FBF7E2FE012704462CE700BFDB0FC93FCA
:10BE7000FFFFDF3ED769853C59DA4B3D356B883D86
:10BE80006E2EBA3D2549123EABAAAA3E21A215BD8F
:10BE90006BF16E3D95879D3D388EE33DCDCC4C3E9C
:10BEA000E8E70008F8E70008CAF24971FFFF973F8A
:10BEB000DB0FC9BFFFFF1B40000080BF20F0004028
:10BEC000704700BF2DE9F04120F00047FD0D7F3D98
:10BED000162D064613DC002D80461BDB194F2F4123
:10BEE000074214D01849FBF7E3FC0021FBF7A4FF3D
:10BEF00068B1002E1BDB28EA0700BDE8F081B7F12E
:10BF0000FF4F04D30146FBF7D3FCBDE8F081304678
:10BF1000BDE8F0810C49FBF7CBFC0021FBF78CFF5F
:10BF20000028F4D0002E08DB0020BDE8F0814FF49B
:10BF3000000343FA05F5A844DDE7002FE7D00348E6
:10BF4000BDE8F081FFFF7F00CAF24971000080BFA9
:10BF500030F0004001D102207047A0F50003B3F19A
:10BF6000FE4F01D204207047054B421E9A4201D871
:10BF700003207047B0F1FF4358425841704700BF5B
:10BF8000FEFF7F0038B530F00044024603460D4600
:10BF900014D0B4F1FF4F0DD2B4F5000F0FD3E40D60
:10BFA0002C44FE2C2EDC002C1DDD23F0FF4343EA45
:10BFB000C45038BD0146FBF77BFC38BD38BD4FF09F
:10BFC0009841FBF77DFD194B02469D4207DBC0F30C
:10BFD000C7540346193CE3E7154800F02DF814490F
:10BFE000FBF76EFD38BD14F1160F13DA4CF2503327
:10BFF0009D421146F0DD0F4800F01EF80D49FBF799
:10C000005FFD38BD11460B4800F016F80949FBF7F3
:10C0100057FD38BD04F1190023F0FF4343EAC05037
:10C020004FF04C51FBF74CFD38BD00BFB03CFFFF5B
:10C030006042A20DCAF2497101F0004120F00040B7
:10C0400008437047014B1868704700BFE4000020A8
:10C05000524F4C4C3B50495443483B5941573B414C
:10C060004C543B506F733B506F73523B4E61765252
:10C070003B4C4556454C3B4D41473B56454C3B00A0
:10C0800000000000A4D20008000000000100000031
:10C09000A9D200080100000002000000B0D2000890
:10C0A0000200000003000000B9D2000803000000F5
:10C0B00004000000BFD200080500000005000000D9
:10C0C000C4D200080600000006000000CED200081E
:10C0D0000700000007000000D7D200080800000099
:10C0E00008000000E0D2000809000000090000007C
:10C0F000E9D200080A0000000A000000F3D200089C
:10C100000B0000000B000000FDD200080C00000036
:10C110000C00000007D300080D0000000D00000017
:10C120000FD300080E0000000E00000017D3000817
:10C130000F0000000F0000001FD3000810000000D7
:10C140001000000028D300081100000011000000BA
:10C150002FD30008120000001200000039D300089D
:10C16000130000001300000041D300081400000079
:10C17000140000004CD3000815000000150000005A
:10C1800000000000FF00000000100140002010022D
:10C1900000100140004010020000000000000000FC
:10C1A0000301000050C700080400000010C7000889
:10C1B00004000000D0C6000802010000B0C600085C
:10C1C00000010000000000000600000050C600084A
:10C1D00006000000F0C5000801010000000000009A
:10C1E00004000000B0C500080600000050C50008AB
:10C1F00008000000D0C400080800000050C4000877
:10C2000008000000D0C30008010100000000000089
:10C21000000100000000000000010000000000001C
:10C220000400000090C300080600000030C30008AE
:10C2300000010000000000000201000010C300081F
:10C2400001010000000000000000000000000000EC
:10C25000020000008025000000C201000000000074
:10C26000100000008025000000C201000100000055
:10C27000200000008025000000C201000000000036
:10C28000010000008025000000C201000000000045
:10C29000080000008025000000C20100000300002B
:10C2A0000400000080250000004B0000000000009A
:10C2B000F8C20008ECC20008EAC20008E8C20008A0
:10C2C000A91700086517000841170008191700088A
:10C2D00009170008FD24000895170008B11600088A
:10C2E000891700087B170008FF00FF000001060304
:10C2F0000D0307030C03FF00000201020202030208
:10C300000802090206030D0307030C03FF000000E7
:10C310000000803F0000000000000000000080BF1F
:10C320000000803F00000000000000000000803F8F
:10C330000000803F000080BF0000803F000080BF01
:10C340000000803F000080BF000080BF0000803FF1
:10C350000000803F0000803F0000803F0000803FE1
:10C360000000803F0000803F000080BF000080BFD1
:10C370000000803F000000000000000000000000FE
:10C380000000803F000000000000000000000000EE
:10C390000000803F000000000000803F0000803F60
:10C3A0000000803F000080BF000080BF0000000050
:10C3B0000000803F000000000000803F000080BFC0
:10C3C0000000803F0000803F000080BF0000008030
:10C3D0000000803F0000803F000000BF0000803F61
:10C3E0000000803F000000BF000080BF0000803FD1
:10C3F0000000803F000080BF0000003F0000803F41
:10C400000000803F0000003F0000803F0000803FB0
:10C410000000803F0000003F000080BF000080BFA0
:10C420000000803F000080BF000000BF000080BF10
:10C430000000803F000000BF0000803F000080BF80
:10C440000000803F0000803F0000003F000080BFF0
:10C450000000803FF704353FF70435BF0000803F00
:10C460000000803FF70435BFF70435BF0000803F70
:10C470000000803FF70435BFF704353F0000803FE0
:10C480000000803FF704353FF704353F0000803F50
:10C490000000803F00000000000080BF000080BF5F
:10C4A0000000803F000080BF00000000000080BF4F
:10C4B0000000803F000000000000803F000080BFBF
:10C4C0000000803F0000803F00000000000080BFAF
:10C4D0000000803F000080BF0000803F000080BF60
:10C4E0000000803F000080BF000080BF0000803F50
:10C4F0000000803F0000803F0000803F0000803F40
:10C500000000803F0000803F000080BF000080BF2F
:10C510000000803F000080BF0000803F0000803F9F
:10C520000000803F000080BF000080BF000080BF8F
:10C530000000803F0000803F0000803F000080BF7F
:10C540000000803F0000803F000080BF0000803F6F
:10C550000000803F000000BFD0B35D3F0000803F7F
:10C560000000803F000000BFD0B35DBF0000803FEF
:10C570000000803F0000003FD0B35D3F000080BF5F
:10C580000000803F0000003FD0B35DBF000080BFCF
:10C590000000803F000080BF00000000000080BF5E
:10C5A0000000803F0000803F000000000000803F4E
:10C5B0000000803F000000000000803F000080BFBE
:10C5C0000000803F000080BF000080BF000000002E
:10C5D0000000803F000000000000803F0000803F1E
:10C5E0000000803F0000803F000080BF000000008E
:10C5F0000000803FD0B35DBF0000003F0000803FDF
:10C600000000803FD0B35DBF000000BF000080BFCE
:10C610000000803FD0B35D3F0000003F0000803F3E
:10C620000000803FD0B35D3F000000BF000080BF2E
:10C630000000803F00000000000080BF0000803F3D
:10C640000000803F000000000000803F000080BF2D
:10C650000000803F00000000A8AAAA3F0000803F21
:10C660000000803F000080BFB0AA2ABF000080BF4A
:10C670000000803F0000803FB0AA2ABF000080BFBA
:10C680000000803F00000000A8AAAA3F000080BF71
:10C690000000803F000080BFB0AA2ABF0000803F9A
:10C6A0000000803F0000803FB0AA2ABF0000803F0A
:10C6B0000000803F0000803F0000000000000000FC
:10C6C0000000803F000080BF00000000000000006C
:10C6D0000000803F000080BF0000803F000080BF5E
:10C6E0000000803F000080BF000080BF0000803F4E
:10C6F0000000803F0000803F0000803F0000803F3E
:10C700000000803F0000803F000080BF000080BF2D
:10C710000000803F000000000000803F000080BF5C
:10C720000000803F000080BF000000000000803F4C
:10C730000000803F0000803F000000000000803FBC
:10C740000000803F00000000000080BF000080BFAC
:10C750000000803F00000000A8AAAA3F00000000DF
:10C760000000803F000080BFB0AA2ABF0000000088
:10C770000000803F0000803FB0AA2ABF00000000F8
:10C78000000000008025000000C20100020000003F
:10C79000010000008025000000C20100030000002D
:10C7A000002C014000000040000400400008004050
:10C7B0000000040008000C0000540040000C014080
:10C7C000400080001F2000000000200000580040B2
:10C7D000000C01400004000821220000000040007D
:10C7E0003ADA00083EDA000844DA00084ADA0008BB
:10C7F0004DDA000854DA000857DA00085CDA00085D
:10C8000068DA00086BDA000871DA000878DA0008E4
:10C8100082DA00088CDA000895DA0008A3DA00084A
:10C82000AFDA0008B6DA0008BCDA0008C9DA000896
:10C83000D4DA0008E1DA00080000000092D900080C
:10C8400099D900089ED90008AFD90008B9D90008C5
:10C85000C4D90008CFD90008DAD90008DED9000809
:10C86000E7D90008EDD90008F7D9000805DA000873
:10C8700008DA000818DA00081FDA000828DA0008C9
:10C8800032DA00080000000013D8000817D80008AA
:10C89000BD3000083ED8000843D80008F12C00083D
:10C8A000C1DC000857D80008E56A000874D8000801
:10C8B00079D80008554F0008A8D80008AADC00085D
:10C8C0007D330008ADD80008B5D80008E52B000876
:10C8D000C9D80008CDD80008CD630008E0D800080A
:10C8E000AADC0008A1630008E5D80008E9D8000820
:10C8F000412B000851D8000805D90008812F0008F5
:10C9000018D900081ED900081D3000084FD70008AC
:10C9100039D90008094F000848D900084DD9000846
:10C920002D33000863D500085DD900082D64000888
:10C930008BD900087FD90008C9620008EADE000828
:10C94000AADC0008B16200089001C800C800C80055
:10C95000C800C800C800C800C80064000000C800C3
:10C96000C800C800C800320010DD000815DD00084E
:10C9700019DD000822DD0008E7D90008DAD900082F
:10C980001EDD000800000000AADC0008D4DC00085E
:10C99000DCDC0008E4DC0008ECDC0008F3DC000868
:10C9A000FEDC000806DD00080BDD000800000000CA
:10C9B0001E1E64646464646499280008E717000814
:10C9C000B517000841470008031800083D47000854
:10C9D0002CDD000844000000180F002000000000BB
:10C9E0002823000035DD0008410000001A0F002058
:10C9F000000000000100000043DD000844000000CA
:10CA000024100020B0040000A40600004ADD000845
:10CA1000440000002610002000000000D0070000A5
:10CA200054DD000844000000281000200000000031
:10CA3000D00700005EDD0008420000002A10002040
:10CA400000000000120000006BDD00084200000042
:10CA50002C100020000000000100000080DD000814
:10CA600044000000DC0F002000000000D0070000A0
:10CA70008DDD000844000000DE0F002000000000F3
:10CA8000D00700009ADD000844000000E00F0020FD
:10CA900000000000D0070000A6DD000844000000F0
:10CAA000E20F002000000000D0070000B6DD000803
:10CAB00044000000E40F002000000000D007000048
:10CAC000C7DD000844000000E60F00200000000061
:10CAD000D0070000D2DD000844000000E80F00206D
:10CAE00000000000D0070000E7DD0008440000005F
:10CAF000EA0F002032000000007D0000F6DD000893
:10CB000044000000EC0F002032000000F2010000A1
:10CB100005DE0008410000002D100020000000008C
:10CB20000100000012DE0008410000002E1000206D
:10CB3000000000000100000025DE000841000000A8
:10CB40002F10002000000000B400000031DE0008BB
:10CB500041000000301000200000000064000000D0
:10CB60003DDE00084200000031100020FFFFFFFF03
:10CB70000100000053DE00084100000034100020D6
:10CB800000000000080000006ADE0008410000000C
:10CB900035100020000000000800000081DE0008C1
:10CBA0004100000048100020300000007E0000001E
:10CBB00092DE00085000000038100020B004000091
:10CBC00000C201009FDE0008500000003C10002061
:10CBD000B004000000C20100ACDE0008410000000B
:10CBE000221000200000000003000000BEDE00084C
:10CBF000410000004C100020000000000200000076
:10CC0000D1DE0008410000004D10002000000000AF
:10CC100001000000E2DE0008410000004E1000208C
:10CC20000000000001000000F2DE000841000000EA
:10CC3000101000200A000000C8000000FDDE0008FF
:10CC400041000000111000200A0000003200000026
:10CC500013DF000841000000121000200A0000004D
:10CC60003200000029DF00084400000014100020FA
:10CC700001000000102700003DDF00084400000014
:10CC800016100020000000007206000052DF0008AD
:10CC9000410000001810002000000000010000000A
:10CCA00070DF000841000000EE0F002000000000CF
:10CCB000080000007BDF000841000000EF0F0020AB
:10CCC000000000000800000085DF000841000000AF
:10CCD000F00F002000000000080000008FDF0008B7
:10CCE00048000000F20F00204CFFFFFF6801000029
:10CCF000A0DF000848000000F40F00204CFFFFFFF9
:10CD000068010000B2DF000848000000F60F0020B4
:10CD10004CFFFFFF68010000C2DF00084400000074
:10CD2000021000206400000084030000D8DF000827
:10CD300044000000FA0F0020000000000001000085
:10CD4000E1DF0008410000000010002000000000AA
:10CD500080000000F1DF000844000000FC0F00200C
:10CD600064000000E803000002E000084400000046
:10CD7000FE0F002064000000E803000014E000083B
:10CD8000810000002611002001000000FA000000D0
:10CD900026E00008810000002711002000000000AC
:10CDA000010000003BE00008810000002A11002083
:10CDB000000000009600000055E00008840000001C
:10CDC0002811002001000000840300001DE000087D
:10CDD000810000002411002000000000200000005D
:10CDE0006FE0000881000000251100200000000015
:10CDF000640000007CE0000842000000F80F002002
:10CE0000FFFFFFFF0100000092E000088200000029
:10CE100074110020FFFFFFFF01000000A0E00008E8
:10CE200082000000751100200000000001000000D9
:10CE3000B2E0000881000000A01000200000000007
:10CE4000FA000000BAE0000881000000A1100020F4
:10CE50000000000064000000C2E000088100000043
:10CE6000A21000200000000064000000CAE00008DA
:10CE700081000000A31000200000000064000000FA
:10CE8000D3E0000881000000A41000200000000092
:10CE900064000000E3E0000881000000A51000200D
:10CEA0000000000064000000ECE0000881000000C9
:10CEB000A61000200000000064000000F5E000085B
:10CEC00084000000A8100020E8030000D007000044
:10CED00004E10008810000006C1100200000000047
:10CEE000C800000013E10008810000006D1100205F
:10CEF00000000000C800000026E1000884000000D7
:10CF00006E110020E8030000D007000038E100089F
:10CF1000840000007011002064000000D0070000B1
:10CF20004AE1000884000000721100206400000043
:10CF3000B80B00005CE100088100000076110020C1
:10CF400000000000FF00000069E10008410000004F
:10CF5000F90F0020000000000500000076E1000845
:10CF600081000000B010002000000000FA00000066
:10CF700085E1000881000000B810002000000000DA
:10CF80006400000094E1000881000000B910002056
:10CF90000000000064000000A2E10008A000000002
:10CFA000B41000200100000014000000B2E10008ED
:10CFB00081000000CC1000200000000001000000F3
:10CFC000C1E1000888000000AE100020D4FEFFFF81
:10CFD0002C010000D0E1000888000000AC10002007
:10CFE000D4FEFFFF2C010000DEE1000881000000FC
:10CFF000BC1000200000000030000000ECE1000840
:10D00000A0000000C010002000000000010000008F
:10D01000FBE10008A0000000C41000200000000098
:10D020000100000007E20008A0000000C810002076
:10D03000000000000100000013E20008880000006A
:10D04000AA100020B0B9FFFF5046000023E20008FC
:10D0500081000000501000200000000002000000CD
:10D0600032E200088100000055100020000000009E
:10D07000C80000003AE20008810000005F100020B4
:10D0800000000000C8000000AADF000881000000C6
:10D090006910002000000000C800000042E2000803
:10D0A000810000005410002000000000C8000000B3
:10D0B00049E20008810000005E100020000000002E
:10D0C000C800000099DF00088100000068100020FF
:10D0D00000000000C800000050E2000881000000CD
:10D0E0005610002000000000C800000056E20008B2
:10D0F000810000006010002000000000C800000057
:10D10000BCDF0008810000006A1000200000000061
:10D11000C80000005CE20008A000000078100020B9
:10D12000000000006400000065E20008A0000000AC
:10D130008410002000000000640000006EE200087F
:10D14000A00000009010002000000000640000001B
:10D1500077E20008A000000074100020000000002A
:10D16000640000007FE20008A000000080100020A2
:10D17000000000006400000087E20008A00000003A
:10D180008C10002000000000640000008FE2000806
:10D19000A00000007C1000200000000064000000DF
:10D1A00096E20008A00000008810002000000000A7
:10D1B000640000009DE20008A00000009410002020
:10D1C0000000000064000000A4E20008A0000000CD
:10D1D0009C100020000000000A000000B2E20008DD
:10D1E000A000000098100020000000000A000000CD
:10D1F000BEE200088100000057100020000000007F
:10D20000C8000000C4E20008810000006110002096
:10D2100000000000C8000000CAE200088100000011
:10D220006B10002000000000C8000000D0E20008E1
:10D23000810000005B10002000000000C80000001A
:10D24000D8E2000881000000651000200000000006
:10D25000C8000000E0E20008810000006F1000201C
:10D2600000000000C8000000E8E2000881000000A3
:10D270005D10002000000000C8000000EEE2000881
:10D28000810000006710002000000000C8000000BE
:10D29000F4E200088100000071100020000000008E
:10D2A000C800000041524D3B00414E474C453B00F9
:10D2B000484F52495A4F4E3B004241524F3B004D5E
:10D2C00041473B0048454144465245453B0048459F
:10D2D000414441444A3B0043414D535441423B0089
:10D2E00043414D545249473B0047505320484F4D0E
:10D2F000453B0047505320484F4C443B005041535E
:10D3000053544852553B004245455045523B004C12
:10D3100045444D41583B004C45444C4F573B004C15
:10D320004C49474854533B0043414C49423B00471A
:10D330004F5645524E4F523B004F53442053573B9C
:10D340000054454C454D455452593B004155544FAE
:10D3500054554E453B0000000000004000080140CD
:10D3600001000000001C00280000004000080140EF
:10D3700002000000041C00280000004000080140DA
:10D3800004000000081C00280000004000080140C4
:10D39000080000000C1C00280004004000080140A8
:10D3A00040000000001D002800040040000801406B
:10D3B00080000000041D002800040040000C014013
:10D3C00001000000081D002800040040000C01407E
:10D3D000020000000C1D0028002C01400008014044
:10D3E00000010000001B0128002C01400008014042
:10D3F000000800000C1B012800080040000C014040
:10D4000040000000001E002800080040000C014001
:10D4100080000000041E002800080040000C0140AD
:10D4200000010000081E002800080040000C014018
:10D43000000200000C1E00283031323334353637FC
:10D4400038394142434445464748494A4B4C4D4E82
:10D450004F505152535455565758595A002025642D
:10D46000202564004D75737420626520616E7920FB
:10D470006F72646572206F662041455452313233B9
:10D48000340D0A0043757272656E7420617373699E
:10D49000676E6D656E743A2000456E61626C6564FE
:10D4A0002066656174757265733A200025732000EB
:10D4B000417661696C61626C652066656174757244
:10D4C00065733A2000496E76616C69642066656117
:10D4D00074757265206E616D650D0A0047505320AA
:10D4E000756E617661696C61626C650D0A00534FFF
:10D4F0004E415220756E617661696C61626C650D9A
:10D500000A0044697361626C65642000456E616263
:10D510006C656420004E4709004F4B09004375734A
:10D52000746F6D206D697865723A200D0A4D6F74C5
:10D530006F720954687209526F6C6C095069746398
:10D5400068095961770D0A002325643A090025739B
:10D55000090053616E69747920636865636B3A09E9
:10D56000007265736574006C6F616400496E76616A
:10D570006C6964206D6978657220747970650D0A34
:10D58000004C6F61646564202573206D69780D0A15
:10D590000057726F6E67206E756D626572206F66E0
:10D5A00020617267756D656E74732C206E6565649D
:10D5B00073206964782074687220726F6C6C2070BC
:10D5C00069746368207961770D0A004D6F746F721A
:10D5D000206E756D626572206D75737420626520B2
:10D5E0006265747765656E203120616E6420256404
:10D5F0000D0A0043757272656E74206D69786572EC
:10D600003A2025730D0A00417661696C61626C6590
:10D61000206D69786572733A20004D6978657220D3
:10D6200073657420746F2025730D0A00557361674C
:10D63000653A0D0A6D6F746F7220696E64657820AB
:10D640005B76616C75655D202D2073686F77205B5C
:10D650006F72207365745D206D6F746F72207661D8
:10D660006C75650D0A004E6F2073756368206D6FD1
:10D67000746F722C207573652061206E756D626504
:10D6800072205B302C2025645D0D0A004D6F746F95
:10D6900072202564206973207365742061742025CD
:10D6A000640D0A00496E76616C6964206D6F746F59
:10D6B000722076616C75652C20313030302E2E3220
:10D6C0003030300D0A0053657474696E67206D6FD9
:10D6D000746F7220256420746F2025640D0A006128
:10D6E00075782025752025750D0A00496E76616CC8
:10D6F0006964204665617475726520696E64657839
:10D700003A206D757374206265203C2025750D0AE2
:10D7100000536176696E67000D0A4C656176696E2B
:10D720006720434C49206D6F64650D0A000D0A5255
:10D7300065626F6F74696E67002E0070726F666944
:10D740006C652025640D0A006D617374657200704C
:10D75000726F66696C65000D0A23207665727369C5
:10D760006F6E0D0A000D0A232064756D70206D61C7
:10D77000737465720D0A000D0A23206D6978657255
:10D780000D0A006D697865722025730D0A00636DBE
:10D79000697820256400636D697820256420302035
:10D7A00030203020300D0A000D0A0D0A2320666556
:10D7B00061747572650D0A00666561747572652025
:10D7C0002D25730D0A0066656174757265202573D9
:10D7D0000D0A000D0A0D0A23206D61700D0A006DFF
:10D7E00061702025730D0A000D0A232064756D7089
:10D7F0002070726F66696C650D0A000D0A23207037
:10D80000726F66696C650D0A000D0A2320617578D8
:10D810000D0A0061757800666561747572655F6EEA
:10D82000616D6520617578666C6167206F7220623A
:10D830006C616E6B20666F72206C69737400636D2F
:10D8400069780064657369676E20637573746F6DC2
:10D85000206D6978657200726573657420746F203D
:10D8600064656661756C747320616E6420726562B4
:10D870006F6F740064756D70007072696E742063F0
:10D880006F6E666967757261626C6520736574742A
:10D89000696E677320696E206120706173746162C4
:10D8A0006C6520666F726D006578697400666561ED
:10D8B00074757265006C697374206F72202D7661C7
:10D8C0006C206F722076616C006765740067657408
:10D8D000207661726961626C652076616C756500A5
:10D8E00068656C70006D6170006D617070696E6765
:10D8F000206F66207263206368616E6E656C206FB6
:10D9000072646572006D69786572206E616D652064
:10D910006F72206C697374006D6F746F720067654D
:10D92000742F736574206D6F746F72206F757470CF
:10D9300075742076616C756500696E646578202861
:10D940003020746F20322900736176650073617630
:10D950006520616E64207265626F6F74006E616D28
:10D96000653D76616C7565206F7220626C616E6BCF
:10D97000206F72202A20666F72206C6973740073A6
:10D98000686F772073797374656D20737461747533
:10D99000730052585F50504D005642415400494E5A
:10D9A000464C494748545F4143435F43414C005212
:10D9B000585F53455249414C004D4F544F525F53AD
:10D9C000544F5000534552564F5F54494C540053E6
:10D9D0004F465453455249414C004750530046412D
:10D9E000494C5341464500534F4E41520054454C1B
:10D9F000454D455452590043555252454E545F4D82
:10DA0000455445520033440052585F504152414CF6
:10DA10004C454C5F50574D0052585F4D535000528B
:10DA20005353495F414443004C45445F535452496A
:10DA30005000444953504C415900545249005155EB
:10DA40004144500051554144580042490047494D16
:10DA500042414C005936004845583600464C594919
:10DA60004E475F57494E470059340048455836588D
:10DA7000004F43544F5838004F43544F464C415485
:10DA800050004F43544F464C415458004149525066
:10DA90004C414E450048454C495F3132305F43436D
:10DAA000504D0048454C495F39305F44454700566A
:10DAB0005441494C340048455836480050504D5F59
:10DAC000544F5F534552564F004455414C434F50BD
:10DAD0005445520053494E474C45434F50544552CC
:10DAE00000435553544F4D00414552543132333465
:10DAF00000002710080423022001436C65616E6654
:10DB00006C696768742F2573536570203232203238
:10DB1000303134202F2031393A30323A3230202817
:10DB20002573290064356635666462005379737421
:10DB3000656D20557074696D653A202564207365A4
:10DB4000636F6E64732C20566F6C746167653A2046
:10DB50002564202A20302E31562028256453206247
:10DB6000617474657279290D0A004350552025644B
:10DB70004D487A2C20646574656374656420736510
:10DB80006E736F72733A200041434348573A202521
:10DB900073002E2563004379636C652054696D65BD
:10DBA0003A2025642C20493243204572726F7273EB
:10DBB0003A2025642C20636F6E6669672073697A4A
:10DBC000653A2025640D0A00417661696C61626CDA
:10DBD0006520636F6D6D616E64733A0D0A00257385
:10DBE0000925730D0A00556E6B6E6F776E20766196
:10DBF000726961626C65206E616D650D0A00437526
:10DC00007272656E742073657474696E67733A20FE
:10DC10000D0A0025732073657420746F200056610F
:10DC20006C75652061737369676E6D656E74206FC6
:10DC30007574206F662072616E67650D0A000D0AAB
:10DC4000456E746572696E6720434C49204D6F6460
:10DC5000652C207479706520276578697427207495
:10DC60006F2072657475726E2C206F722027686544
:10DC70006C70270D0A000D0A2320000D1B5B4B0062
:10DC80001B5B324A1B5B313B314800556E6B6E6F3C
:10DC9000776E20636F6D6D616E642C2074727920D5
:10DCA0002768656C702700082008004145545231F0
:10DCB00032333400526573657474696E6720746F13
:10DCC0002064656661756C747300736574202573D8
:10DCD000203D20004144584C333435004D505536DA
:10DCE000303530004D4D413834357800424D4132A9
:10DCF0003830004C534D333033444C4843004D5082
:10DD000055363030300046414B45004E6F6E650051
:10DD10004759524F00414343004241524F00475040
:10DD2000532B4D414700434A4D4355006C6F6F7074
:10DD300074696D6500656D665F61766F6964616EBB
:10DD40006365006D69645F7263006D696E5F63682F
:10DD500065636B006D61785F636865636B00727308
:10DD600073695F6368616E6E656C00696E7075746F
:10DD70005F66696C746572696E675F6D6F6465007C
:10DD80006D696E5F7468726F74746C65006D617834
:10DD90005F7468726F74746C65006D696E5F636F39
:10DDA0006D6D616E640033645F6465616462616EB1
:10DDB000645F6C6F770033645F6465616462616E99
:10DDC000645F686967680033645F6E65757472616B
:10DDD0006C0033645F6465616462616E645F746883
:10DDE000726F74746C65006D6F746F725F70776DB5
:10DDF0005F7261746500736572766F5F70776D5FD7
:10DE0000726174650072657461726465645F6172E9
:10DE10006D0064697361726D5F6B696C6C5F7377C1
:10DE20006974636800736D616C6C5F616E676C65CB
:10DE300000666C6170735F73706565640066697815
:10DE4000656477696E675F616C74686F6C645F644A
:10DE500069720073657269616C5F706F72745F31B3
:10DE60005F7363656E6172696F0073657269616C7F
:10DE70005F706F72745F325F7363656E6172696F3A
:10DE8000007265626F6F745F63686172616374656D
:10DE900072006D73705F62617564726174650063B6
:10DEA0006C695F6261756472617465007365726943
:10DEB000616C72785F70726F766964657200746508
:10DEC0006C656D657472795F70726F766964657286
:10DED0000074656C656D657472795F7377697463DE
:10DEE00068006672736B795F696E76657273696FCD
:10DEF0006E00766261745F7363616C650076626167
:10DF0000745F6D61785F63656C6C5F766F6C746174
:10DF1000676500766261745F6D696E5F63656C6CE6
:10DF20005F766F6C746167650063757272656E749D
:10DF30005F6D657465725F7363616C6500637572B4
:10DF400072656E745F6D657465725F6F666673652A
:10DF500074006D756C74697769695F637572726559
:10DF60006E745F6D657465725F6F75747075740043
:10DF7000616C69676E5F6779726F00616C69676E6B
:10DF80005F61636300616C69676E5F6D616700610B
:10DF90006C69676E5F626F6172645F726F6C6C0058
:10DFA000616C69676E5F626F6172645F70697463F0
:10DFB0006800616C69676E5F626F6172645F79614E
:10DFC00077006D61785F616E676C655F696E636C29
:10DFD000696E6174696F6E006779726F5F6C7066ED
:10DFE000006D6F726F6E5F7468726573686F6C64DA
:10DFF000006779726F5F636D70665F666163746FEF
:10E0000072006779726F5F636D70666D5F666163E2
:10E01000746F7200616C745F686F6C645F646561DB
:10E020006462616E6400616C745F686F6C645F66EB
:10E030006173745F6368616E6765007468726F74A2
:10E04000746C655F636F7272656374696F6E5F761F
:10E05000616C7565007468726F74746C655F636F72
:10E060007272656374696F6E5F616E676C6500796B
:10E0700061775F6465616462616E64007961775F96
:10E08000636F6E74726F6C5F646972656374696FDD
:10E090006E007961775F646972656374696F6E00A1
:10E0A0007472695F756E61726D65645F73657276B7
:10E0B0006F0072635F726174650072635F65787090
:10E0C0006F007468725F6D6964007468725F657870
:10E0D000706F00726F6C6C5F70697463685F7261FF
:10E0E0007465007961775F72617465007470615F57
:10E0F00072617465007470615F627265616B706FEC
:10E10000696E74006661696C736166655F64656CF5
:10E110006179006661696C736166655F6F66665FF1
:10E1200064656C6179006661696C736166655F74D2
:10E1300068726F74746C65006661696C73616665A2
:10E140005F6D696E5F75736563006661696C7361AD
:10E1500066655F6D61785F757365630067696D62A1
:10E16000616C5F666C616773006163635F686172B5
:10E170006477617265006163635F6C70665F66619E
:10E1800063746F720061636378795F646561646270
:10E19000616E64006163637A5F6465616462616E8D
:10E1A00064006163637A5F6C70665F6375746F6649
:10E1B00066006163635F756E61726D656463616C57
:10E1C000006163635F7472696D5F70697463680096
:10E1D0006163635F7472696D5F726F6C6C00626122
:10E1E000726F5F7461625F73697A65006261726FFA
:10E1F0005F6E6F6973655F6C7066006261726F5FFE
:10E2000063665F76656C006261726F5F63665F6113
:10E210006C74006D61675F6465636C696E617469DD
:10E220006F6E007069645F636F6E74726F6C6C65A3
:10E230007200705F706974636800695F706974630D
:10E240006800705F726F6C6C00695F726F6C6C005D
:10E25000705F79617700695F79617700705F7069DD
:10E260007463686600695F70697463686600645F00
:10E2700070697463686600705F726F6C6C660069C9
:10E280005F726F6C6C6600645F726F6C6C660070BE
:10E290005F7961776600695F7961776600645F79AD
:10E2A000617766006C6576656C5F686F72697A6F1E
:10E2B0006E006C6576656C5F616E676C6500705FA3
:10E2C000616C7400695F616C7400645F616C740000
:10E2D000705F6C6576656C00695F6C6576656C0077
:10E2E000645F6C6576656C00705F76656C00695F75
:10E2F00076656C00645F76656C000020202020202D
:10E3000020202020282828282820202020202020E5
:10E3100020202020202020202020208810101010D5
:10E320001010101010101010101010040404040429
:10E330000404040404101010101010104141414155
:10E34000414101010101010101010101010101013D
:10E35000010101010101101010101010424242424F
:10E36000424202020202020202020202020202020D
:10E370000202020202021010101020000000000031
:10E38000000000000000000000000000000000008D
:10E39000000000000000000000000000000000007D
:10E3A000000000000000000000000000000000006D
:10E3B000000000000000000000000000000000005D
:10E3C000000000000000000000000000000000004D
:10E3D000000000000000000000000000000000003D
:10E3E000000000000000000000000000000000002D
:10E3F0000000000000000000000000000000004BD2
:10E40000000000CB61636F73660000000000000035
:10E410007371727466000000000FC93F000F49401D
:10E4200000CB9640000FC9400053FB4000CB164183
:10E4300000ED2F41000F49410031624100537B4103
:10E44000003A8A4100CB9641005CA34100EDAF4108
:10E45000007EBC41000FC94100A0D5410031E2411E
:10E4600000C2EE410053FB4100F20342003A0A426F
:10E470000083104200CB164200141D42005C234270
:10E4800000A5294200ED2F4200363642007E3C4274
:10E4900000C74242000F4942A2000000F9000000FC
:10E4A000830000006E0000004E00000044000000E9
:10E4B0001500000029000000FC00000027000000FB
:10E4C00057000000D1000000F500000034000000FB
:10E4D000DD000000C0000000DB0000006200000062
:10E4E00095000000990000003C000000430000007F
:10E4F0009000000041000000FE00000051000000FC
:10E5000063000000AB000000DE000000BB00000064
:10E51000C500000061000000B700000024000000FA
:10E520006E0000003A000000420000004D000000B4
:10E53000D2000000E00000000600000049000000DA
:10E540002E000000EA00000009000000D1000000D9
:10E55000920000001C000000FE0000001D000000F2
:10E56000EB0000001C000000B100000029000000CA
:10E57000A70000003E000000E8000000820000004C
:10E5800035000000F50000002E000000BB00000078
:10E590004400000084000000E90000009C0000002E
:10E5A0007000000026000000B40000005F000000C2
:10E5B0007E000000410000003900000091000000D2
:10E5C000D600000039000000830000005300000066
:10E5D00039000000F40000009C00000084000000EE
:10E5E0005F0000008B000000BD000000F90000008B
:10E5F000280000003B0000001F000000F8000000A1
:10E6000097000000FF000000DE0000000500000091
:10E61000980000000F000000EF0000002F00000035
:10E62000110000008B0000005A0000000A000000EA
:10E630006D0000001F0000006D00000036000000AB
:10E640007E000000CF00000027000000CB0000008B
:10E6500009000000B70000004F0000004600000065
:10E660003F000000660000009E0000005F00000008
:10E67000EA0000002D0000007500000027000000E7
:10E68000BA000000C7000000EB000000E500000039
:10E69000F10000007B0000003D00000007000000CA
:10E6A00039000000F70000008A000000520000005E
:10E6B00092000000EA0000006B000000FB00000078
:10E6C0005F000000B10000001F0000008D0000008E
:10E6D0005D0000000800000056000000030000007C
:10E6E0003000000046000000FC0000007B0000003D
:10E6F0006B000000AB000000F0000000CF00000045
:10E70000BC000000200000009A000000F40000009F
:10E71000360000001D000000A9000000E30000001A
:10E7200091000000610000005E000000E6000000B3
:10E730001B000000080000006500000099000000B8
:10E74000850000005F00000014000000A000000031
:10E7500068000000400000008D000000FF00000085
:10E76000D8000000800000004D0000007300000091
:10E770002700000031000000060000000600000035
:10E780001500000056000000CA00000073000000E1
:10E79000A8000000C900000060000000E2000000C6
:10E7A0007B000000C00000008C0000006B00000037
:10E7B0000400000007000000090000000000C93F3D
:10E7C0000000F0390000DA370000A2330000842E88
:10E7D0000000502B0000C2270000D0220000C41F00
:10E7E0000000C61B000044176937AC316821223392
:10E7F000B40F14336821A2333863ED3EDA0F493F7A
:08E800005E987B3FDA0FC93F6F
:08E808006C97FF7F0100000086
:10E81000000100000000803F000000000000000038
:10E8200000000000000000000000000001000000E7
:10E83000000000000000000000127A00000000004C
:10E84000000000000102030406070809010300009C
:10E850000000803F0000803F0000803F000000007B
:10E860000102030401020304060708090204060862
:10E87000DC05DC05DC05DC05DC05DC05DC05DC0590
:10E88000B13300080300000000A24A0426DD00089E
:10E89000FAE2000800000000000000000000000094
:10E8A0000000000000000000000000000000000068
:10E8B0000000000017DD000800000000000000005C
:10E8C0000000000000000000000000000000000048
:10E8D0000000000000000000000000000000000038
:10E8E0000000000000000000000000000000000028
:0CE8F00000000000840000200100000077
:0400000508000000EF
:00000001FF
